:020000040800F2
:1000000000000220012F0108099300080B9300084B
:100010000D9300080F9300081193000800000000E2
:100020000000000000000000000000001393000822
:1000300015930008000000001793000819930008AA
:10004000452F0108452F0108452F0108452F0108BC
:10005000452F0108452F0108452F0108452F0108AC
:10006000452F0108452F0108452F0108B1760008EA
:10007000452F0108452F0108452F0108452F01088C
:10008000452F0108452F0108452F0108452F01087C
:10009000452F0108452F0108452F01084995000803
:1000A000452F0108452F0108452F0108452F01085C
:1000B00015950008452F0108452F0108452F010817
:1000C000452F0108452F0108452F0108452F01083C
:1000D000452F0108452F01085D960008452F0108AE
:1000E000452F0108452F01081D930008452F0108E1
:1000F000452F0108452F0108452F0108452F01080C
:10010000452F0108452F0108452F0108452F0108FB
:10011000452F0108452F0108452F0108452F0108EB
:10012000452F0108452F0108452F0108452F0108DB
:10013000452F0108452F0108452F0108452F0108CB
:10014000452F0108452F0108452F01084D93000850
:10015000452F0108452F0108452F0108452F0108AB
:10016000452F0108452F0108452F0108452F01089B
:10017000452F0108452F0108452F0108452F01088B
:08018000452F0108452F01087D
:1001880084B2050800000020080C0020080C00209C
:10019800A43C002008B5074B186809F053F80DF087
:1001A8004BFE054B054806221A70BDE8084001F0D1
:1001B800C4BB00BF10260020A4250020800F00200B
:1001C80008B5034801F0B9FB024B00221A7008BDBC
:1001D800D4170020A425002008B5054B01220020D3
:1001E8001A7005F053FD0348BDE8084001F0A5BBAF
:1001F800242C0020441500202DE9F041144C204601
:1002080003F0A3FE00201349134A03F055FC1349D9
:10021800134A0746002003F04FFC1249124A0646CB
:10022800002003F049FCD22105463A4623460A201D
:1002380003F05AFDD22132462346FA2003F054FD3A
:100248005A20D2212A462346BDE8F04103F04CBD8E
:1002580058130020F69E0508C9010008FF9E0508EE
:10026800E1010008079F05089D01000808B5054B36
:10027800012200201A7005F009FD0348BDE8084076
:1002880001F05BBB242C00204415002008B503486E
:1002980001F053FB024B00221A7008BDD41700204E
:1002A800A425002008B5054B07221A700DF0C4FDDF
:1002B8000348BDE8084001F040BB00BFA42500206A
:1002C800581300202DE9F041144C204603F03DFE60
:1002D80000201349134A03F0EFFB1349134A07465A
:1002E800002003F0E9FB1249124A0646002003F0F9
:1002F800E3FBD22105463A4623460A2003F0F4FCE4
:10030800D221324623465A2003F0EEFCAA20D221FD
:100318002A462346BDE8F04103F0E6BC800F0020E2
:10032800F69E050895020008109F0508AD02000812
:10033800199F050875020008014801F0FEBA00BFC0
:100348006C11002010B5094C204603F0FEFD00207A
:100358000749084A03F0B0FBD221024623464FF46E
:100368008270BDE8104003F0BFBC00BF8C160020AF
:10037800229F05084103000870B50C4C0C4D2068FD
:100388004FF6E076314602F0DBFE2068294602F09F
:1003980085FE6068314602F0D3FE6068294602F0A7
:1003A8007DFEBDE8704004F009B800BF080C0020CD
:1003B80011A5050838B52B4CFFF7DEFF002005F026
:1003C80065FC237A23B90A203221274A05F06CFDFF
:1003D800637A23B90A206421244A05F065FD214C7B
:1003E800A37A23B90A209621214A05F05DFDA37A54
:1003F8001C4DFBB16B7AEBB12B7ADBB100232B726E
:100408006B72AB721B4B286801221A704FF6E071B1
:1004180002F096FE2868184902F040FE68681749FD
:1004280002F03CFE0BF005FA03F0C8FF144804F094
:1004380009F80DE00B4C4FF47841206802F080FE7B
:100448002068104902F02AFE60680F4902F026FE73
:10045800FFF792FF00200BF0AFF90C48BDE83840D9
:1004680001F06BBA080C0020299F0508379F050882
:10047800469F0508A4250020549F050812A50508D5
:1004880080969800689F050814A50508D4170020D1
:1004980008B500200BF090F90248BDE8084001F0CB
:1004A8004CBA00BFD417002038B5FFF765FF0DF030
:1004B800DBFC3C213F220023DF2005F0D7FC4FF472
:1004C80080600EF00DFA124C3E223C21DF20002302
:1004D80005F0CCFC012323720E4B4FF6E07518682B
:1004E80008F0B0FE2068294602F02AFE20680A4972
:1004F80002F0D4FD6068294602F022FE60680749D0
:1005080002F0CCFD03F05AFF054B00221A7038BDEB
:10051800080C0020102600207A9F05088D9F0508EA
:10052800A425002038B5FFF727FF0DF09DFC6E21AC
:100538003F220023DF2005F099FC4FF486400EF09F
:10054800CFF9124C3E226E21DF20002305F08EFCED
:10055800012363720E4B4FF6E075186808F072FEBF
:100568002068294602F0ECFD20680A4902F096FD51
:100578006068294602F0E4FD6068074902F08EFDD4
:1005880003F01CFF054B00221A7038BD080C002030
:1005980010260020A09F0508B19F0508A42500206B
:1005A80010B5FFF7E9FE0DF05FFCA0213F22002304
:1005B800DF2005F05BFC4FF402400EF091F9114C7E
:1005C8003E22A021DF20002305F050FC0123A37266
:1005D8000D4B186808F036FE20684FF6E07102F0FF
:1005E800AFFD2068094902F059FD6068084902F02A
:1005F80055FD03F0E3FE64200AF0B8FF054B002226
:100608001A7010BD080C002010260020C29F050893
:1006180012A50508A42500202DE9F74F3A4D3B4EB9
:100628000024284603F091FC224623464FF6FF712A
:1006380037480094019402F047FD4FF6E07804270C
:10064800F06041462246234632480097019402F062
:100658003BFD23463060414622462F4800970194CF
:1006680002F032FD2D4970602D4A204603F024FA2D
:100678002C492D4A0746204603F01EFA2B492C4ADE
:100688008046204603F018FA2A492B4A814620461C
:1006980003F012FA29492A4A8346204603F00CFA45
:1006A80021468246F2682B46204603F01DFB5A215C
:1006B80032682B460A2003F017FB6E2172682B461E
:1006C8000A2003F011FB9B213A462B46FA2003F03F
:1006D8000BFB692142462B46FA2003F005FB372124
:1006E8004A462B46FA2003F0FFFAC82152462B4609
:1006F800AA2003F0F9FAF020C8215A462B4603B085
:10070800BDE8F04F03F0F0BAFC130020080C0020FD
:10071800D69F0508DE9F0508F19F050800A005087B
:10072800A905000808A005082D050008F89F050878
:10073800B104000810A005089904000817A00508CE
:10074800BD03000838B50C4C4FF6E0752068294603
:1007580002F0F6FC2068094902F0A0FC606829460E
:1007680002F0EEFC6068064902F098FC03F026FEF1
:10077800BDE8384003F022BE080C0020DE9F0508C3
:100788001EA0050870B52DED028B9FED248A88B058
:100798000A26F0EE488A03E0B0EE608AF0EE418A5D
:1007A8000CF09BFA8DED000ACDED010A9DE80300DF
:1007B80004AB83E80300F0EE680AB0EE480A9DED4A
:1007C800041ADDED051A8DED028ACDED038A0CF0D1
:1007D80027F8CDED010A8DED000A9DE8030002AD72
:1007E80085E80300013E6C46DDED020A9DED031A23
:1007F800D2D19FED0B0A0CF067FA8DED000ACDED12
:10080800010A9DE8030085E80300DDED030A9DED7C
:10081800020A08B0BDEC028B70BD00BF00000000EA
:10082800CDCCCC3D2DE9F74F564D574CDFF86491B0
:10083800DFF864814FF6E07005F0FCF9286811F0E4
:1008480063FA064668680F4611F05EFA3246CDE94B
:1008580000013B464946204616F0CCF822460023C4
:100868000520372105F020FB2869484F484E11F034
:100878004BFA824668698B4611F046FA5246CDE932
:1008880000015B463946204616F0B4F8224600239C
:100898000520692105F008FB286B11F035FA82461E
:1008A800686B8B4611F030FA5246CDE900015B4681
:1008B8004146204616F09EF8002305209B2122463B
:1008C80005F0F2FA31462A6C204616F093F82246D3
:1008D80000239B21A22005F0E7FA4FF4FC6005F005
:1008E800A9F9A86811F010FA8246E8688B4611F059
:1008F8000BFA5246CDE900015B464946204616F000
:1009080079F8224605205021002305F0CDFAA86980
:1009180011F0FAF98246E8698B4611F0F5F952466A
:10092800CDE900015B463946204616F063F82246B9
:1009380000230520822105F0B7FAA86B11F0E4F92D
:100948008246E86B8B4611F0DFF95246CDE900018B
:100958005B464146204616F04DF800230520B42199
:10096800224605F0A1FA31466A6C204616F042F894
:10097800A220B4212246002303B0BDE8F04F05F0C1
:1009880093BA00BF303A0020180C002043A0050895
:1009980066A0050831A0050855A0050808B500207F
:1009A80005F074F90A4B1B780B2B0BD8DFE803F022
:1009B8000A0A0A0A0A0A08060A0A0A0A054802E08E
:1009C800054800E00548BDE8084000F0B6BF00BF94
:1009D800A425002058130020800F0020D4170020E1
:1009E8002DE9F14F2D4C204603F0AFFA00202C4999
:1009F8002C4A03F061F82C492C4A8146002003F068
:100A08005BF82B492B4A0746002003F055F82A4982
:100A18002A4A0646002003F04FF82949294A054684
:100A2800002003F049F82849284A8046002003F0AE
:100A380043F82749274A8246002003F03DF8D2218F
:100A480083464A462346E62003F04EF928203A46D4
:100A58002346014603F048F946213246234628201A
:100A680003F042F964212A462346282003F03CF982
:100A7800822142462346282003F036F9524623466F
:100A88002820A02103F030F928205A46BE21234609
:100A980001B0BDE8F04F03F027B900BF44150020AE
:100AA8006BA00508A509000874A0050875120008C0
:100AB8007FA005085112000889A005082D1200081A
:100AC80094A00508091200089FA00508E511000870
:100AD800A9A00508C1110008023810B50A2800F2BB
:100AE8003C83DFE810F00B000F006400D2008A019D
:100AF8002001170231023A03A102F502BDE81040B5
:100B08000AF004BF00204FF6E0710BF05FF8632095
:100B18004FF6E0710BF05AF8B3204FF4F0610BF088
:100B280055F8C7204FF6E0710BF050F84FF6FF70FC
:100B380005F080F8DC2100237D20D34A05F0B4F9C4
:100B48004EF29C7005F076F8052001210023CF4A6B
:100B580005F0AAF9052052210023CD4A05F0A4F991
:100B6800B62100230520CB4A05F09EF94FF4F0602A
:100B780005F060F80121002340F21310C34A05F084
:100B880093F9002340F213105221C24A05F08CF960
:100B9800B621C14A40F21310002305F085F94EF240
:100BA8009C7005F047F80520A221BC4A68E00020A7
:100BB8004FF6E0710BF00AF831204FF6E0710BF0B8
:100BC80005F863204FF6E0710BF000F895204FF61A
:100BD800E0710AF0FBFFC7204FF6E0710AF0F6FF5C
:100BE8004EF29C7005F026F8052001210023AC4A3E
:100BF80005F05AF9052020210023AA4A05F054F9E6
:100C0800052052210023A84A05F04EF90520842129
:100C18000023A64A05F048F9B62105209D4A00237D
:100C280005F042F94FF4F06005F004F8012140F2B4
:100C3800131000239A4A05F037F940F213102021C7
:100C48009B4A002305F030F940F213105221914AD3
:100C5800002305F029F940F213108421954A002356
:100C680005F022F9B621944A40F21310002305F04A
:100C78001BF94FF6FF7004F0DDFF904A7D20DC2160
:100C88000023BDE8104005F00FB900204FF6E071D1
:100C98000AF09CFF27204FF6E0710AF097FF4F20DB
:100CA8004FF6E0710AF092FF77204FF6E0710AF0F4
:100CB8008DFF9F204FF6E0710AF088FFC7204FF69E
:100CC800E0710AF083FF4EF29C7004F0B3FF052038
:100CD800012100236F4A05F0E7F8052016210023BB
:100CE800774A05F0E1F805203E210023754A05F012
:100CF800DBF8052066210023734A05F0D5F88E211C
:100D080000230520714A05F0CFF80520704AB62166
:100D1800002305F0C9F84FF6FF7004F08BFF7D2023
:100D2800DC216C4AACE700204FF6E0710AF04EFF78
:100D380031204FF6E0710AF049FF63204FF6E07169
:100D48000AF044FF95204FF6E0710AF03FFFC720F4
:100D58004FF6E0710AF03AFF4EF29C7004F06AFF19
:100D68000520012100235C4A05F09EF8052020217A
:100D780000235A4A05F098F8052052210023584AC2
:100D880005F092F8052084210023564A05F08CF8D6
:100D9800B62105203F4A002305F086F84FF4F0609D
:100DA80004F048FF012140F2131000234E4A05F0D9
:100DB8007BF840F2131020214C4A002305F074F808
:100DC80040F213105221334A002305F06DF840F227
:100DD80013108421464A002305F066F8B621454AD7
:100DE80040F21310002305F05FF84FF6FF7004F08F
:100DF80021FF7D20DC21404A42E700204FF6E071C8
:100E08000AF0E4FE31204FF6E0710AF0DFFE6320BD
:100E18004FF6E0710AF0DAFE95204FF6E0710AF01D
:100E2800D5FEC7204FF4FC610AF0D0FE4EF29C704C
:100E380004F000FF052001210023304A05F034F8B2
:100E48000520202100232E4A05F02EF805205221E6
:100E580000232C4A05F028F88421002305202A4A7B
:100E680005F022F84FF4F06004F0E4FEB621052006
:100E7800264A002305F018F84FF6FF7004F0DAFE52
:100E88008720234ADC21FBE67FA00508B3A00508DC
:100E9800AEA0050861A60508B2A00508E0A00508EF
:100EA800CCA00508B7A00508C7A00508BCA0050880
:100EB800C1A00508C6A00508CBA0050889A005089B
:100EC800CFA00508D3A00508D7A00508DBA0050812
:100ED800DFA00508E3A00508EFA00508F3A00508B2
:100EE800F7A00508FAA0050803A10508FFA0050852
:100EF800FEA0050802A1050807A1050812A105081A
:100F0800D8A00508D0A0050822A1050878A70508DB
:100F1800A9A0050800204FF6E0710AF057FE6320EB
:100F28004FF4FC610AF052FE4FF6E071C7200AF058
:100F38004DFE4FF6FF7004F07DFE002004F07CFFAC
:100F4800A520D721854A9BE6042004F075FF0020E0
:100F58004FF6E0710AF03AFE31204FF6E0710AF0E0
:100F680035FE63204FF6E0710AF030FE95204FF60B
:100F7800E0710AF02BFEC7204FF6E0710AF026FE5A
:100F88004EF29C7004F056FE052001210023744A9D
:100F980004F08AFF052020210023724A04F084FF10
:100FA800052052210023704A04F07EFF0520842189
:100FB80000236E4A04F078FF0520B6216C4A00230E
:100FC80004F072FF4FF6E07004F034FE40F20B10AC
:100FD8000121684A002304F067FF40F22B1020210A
:100FE800654A002304F060FF40F223105221634A4F
:100FF800002304F059FF40F21B108421604A0023AB
:1010080004F052FFB6215F4A002340F2131004F0A7
:101018004BFF4FF6FF7004F00DFE002004F00CFFAC
:101028006E20D221584A90E0042004F005FF0020E9
:101038004FF6E0710AF0CAFD27204FF6E0710AF07A
:10104800C5FD4F204FF6E0710AF0C0FD77204FF63E
:10105800E0710AF0BBFD9F204FF6E0710AF0B6FD83
:10106800C7204FF6E0710AF0B1FD4EF29C7004F013
:10107800E1FD052001210023444A04F015FF052065
:1010880016210023424A04F00FFF05203E210023C9
:10109800404A04F009FF052066213F4A002304F076
:1010A80003FF05208E213D4A002304F0FDFEB621F2
:1010B8003B4A0023052004F0F7FE4FF6FF7004F0CA
:1010C800B9FD002004F0B8FE6420D221354A3CE086
:1010D800042004F0B1FE00204FF6E0710AF076FD1E
:1010E80043204FF6E0710AF071FD85204FF6E0715C
:1010F8000AF06CFD4FF6E071C7200AF067FD4EF26A
:101108009C7004F097FD05200121274A002304F074
:10111800CBFE05204521254A002304F0C5FE052005
:1011280087211F4A002304F0BFFEB621204A00236E
:10113800052004F0B9FE4FF6FF7004F07BFD002097
:1011480004F07AFE1B4A7D20D221002304F0ACFE75
:101158000420BDE8104004F06FBE10BD2AA50508A4
:1011680016A1050822A1050821A1050824A1050842
:1011780028A105082DA10508CCA0050834A105085B
:1011880038A105083DA1050843A1050849A105089E
:10119800FFA0050804A105084EA1050851A10508EE
:1011A800E0A0050854A105085DA1050812A10508DD
:1011B80061A60508D5A5050810B5064C06480623FE
:1011C800237000F0BAFB2078FFF786FCBDE81040DA
:1011D8000DF054BB242C00203017002010B5064C0D
:1011E80006480723237000F0A8FB2078FFF774FC5B
:1011F800BDE810400DF042BB242C00203017002021
:1012080010B5064C06480523237000F096FB20789D
:10121800FFF762FCBDE810400DF030BB242C002025
:101228003017002010B5064C06480423237000F040
:1012380084FB2078FFF750FCBDE810400DF01EBB82
:10124800242C00203017002010B5064C0648032334
:10125800237000F072FB2078FFF73EFCBDE81040D9
:101268000DF00CBB242C00203017002010B5064CC4
:1012780006480223237000F060FB2078FFF72CFC5F
:10128800BDE810400DF0FABA242C002030170020D9
:1012980038B5094C05464FF6E071206801F050FF5B
:1012A80020680DB1054900E0054901F0F7FEBDE8E9
:1012B800384003F083B800BF340C002061A1050852
:1012C80074A105081A4B10B51C78012C14BF102402
:1012D8000024002C14BFD820C82006F03BFA15497A
:1012E8000246154815F086FB002C14BFDC20CC20E4
:1012F80006F030FA0F490246104815F07BFB002C27
:1013080014BFE020D02006F025FA0A4902460C480E
:1013180015F070FB002C14BFE420D42006F01AFA54
:10132800044902460748BDE8104015F063BB00BFFA
:10133800F40D002066A00508E02500200426002002
:10134800162C0020CC25002010B5E82006F002FA63
:101358000F4C024621460F4815F04CFBEC2006F0D6
:10136800F9F9214602460C4815F044FBF02006F036
:10137800F1F921460246094815F03CFBF42006F035
:10138800E9F9024606482146BDE8104015F032BB8F
:1013980066A00508E025002004260020162C002061
:1013A800CC2500200E4A012310B513700D4A0024E5
:1013B80014700D4A204613700AF0FEF9204604F016
:1013C80065FC0A4B03221A700AF03AFD0BF021FA69
:1013D800074B08481C70BDE8104000F0AEBA00BFCB
:1013E800242C00204F0D00204D0D0020A4250020A6
:1013F800043800201012002038B50D4B0D4D002484
:101408001C700D4B28681C700C4B4FF6E0711C705B
:1014180001F096FE28680A4901F040FE02F0CEFF6E
:10142800204604F033FC0748BDE8384000F085BA90
:10143800AC0D0020340C00204F0D0020A425002006
:1014480016A50508D417002007B50E4B0E481A78C4
:10145800D2F1010238BF00221A700C4B05221A7013
:1014680000F06BFA022201238DE80C00B020602105
:10147800102232230DF0A6FB03B05DF804EB02F056
:101488009DBF00BFAC0D0020C8100020A42500207F
:101498002E4A002310B513702D4A13700CF0E6FF86
:1014A8000446002842D02B4C4FF6E071206801F02A
:1014B80047FE2068284901F0F1FD60684FF6E071A9
:1014C80001F03EFE6068254901F0E8FDA0684FF68E
:1014D800E07101F035FEA068214901F0DFFD02F05E
:1014E8006DFF4FF47A600AF041F820684FF6E0711A
:1014F80001F026FE20681B4901F0D0FD60684FF618
:10150800E07101F01DFE6068164901F0C7FDA06892
:101518004FF6E07101F014FEA068124901F0BEFD1B
:1015280002F04CFFBDE8104002F048BF0CF084FC0C
:10153800204604F0ABFB0C4B0C4804221A7000F058
:10154800FCF9BDE81040FFF7FDB800BFAC0D002066
:101558004F0D0020340C002087A105089BA1050829
:10156800ABA1050815A50508A4250020FC1300203B
:101578002DE9F04F6A4DDFF8F4916A4E85B00024EA
:101588004FF6FF78284602F0E0FC41462246234603
:1015980065480094019401F097FD042703904146A3
:1015A8002246234648460097019401F08DFD4146A6
:1015B80030602246234648460097019401F084FD96
:1015C800414670602246234648460097019401F040
:1015D8007BFDA8F50048B0604146224623465348A3
:1015E8000097019401F070FD4146F06022462346C1
:1015F8004F480097019401F067FD4146306122464B
:1016080023464C480097019401F05EFD2346706123
:101618004146224648480097019401F055FD474944
:10162800B061474A204602F047FA4649464A804692
:10163800204602F041FA4549454A8246204602F0D2
:101648003BFA4449444A0746204602F035FA4349E2
:10165800434A8146204602F02FFA4249424A8346CD
:10166800204602F029FA21468446039ACDF808C09C
:101678002B46204602F038FB052132682B46A02075
:1016880002F032FB692172682B46782002F02CFBAD
:101698007D21B2682B46782002F026FB2821F268CB
:1016A8002B46052002F020FB4B2132692B460520F2
:1016B80002F01AFB052072696E212B4602F014FB1A
:1016C8009121B2692B46052002F00EFBD2213A4641
:1016D8002B46052002F008FBD22142462B4660200B
:1016E80002F002FBD2214A462B46B02002F0FCFA57
:1016F800D22152462B464FF4807002F0F5FAB421FD
:101708005A462B46052002F0EFFADDF808C06020A3
:10171800B42162462B4605B0BDE8F04F02F0E4BAAA
:10172800A0140020340C0020BBA10508C5A10508A1
:10173800CCA10508D2A10508D8A10508DEA1050895
:1017480099140008E6A1050801140008EEA105088F
:1017580051140008F7A10508AD130008FFA10508FA
:101768005113000808A20508CD12000812A50508A3
:10177800544A00232DE9F0471370534ADFF860916B
:101788001370524B1D780127BD4214BF1025002548
:10179800B842044689F8007003D0022840F08C80D3
:1017A8000BE021464FF4747005F0BBFF0AF06EFAA7
:1017B800204605F0BBF920467CE0002D14BFD82058
:1017C800C82005F0C7FF0446002D14BFDC20CC203C
:1017D80005F0C0FF8046002D14BFE020D02005F0A2
:1017E800B9FF0646002D14BFE420D42005F0B2FF4F
:1017F80005460AF04BFA364B36491A68A242184693
:1018080002DB0B68434513DD334B04601E60334B2A
:10181800C1F800801D6009F08FFF314B01221A705A
:10182800304A0520B4210023BDE8F04704F03CBB52
:10183800944218D1984516D1274B1B689E4212D165
:10184800264B1B689D420ED14FF47470394689F8B7
:10185800007005F066FF244B00221A60234B4FF0FE
:101868007E521A6028E01E4B02251D7029464FF44F
:10187800747005F056FF164B1B6806EE906A1C1B29
:10188800F8EEE67A06EE904AB8EEE67A164B87EE60
:10189800277A284683ED007A0F4B1B6806EE903AAC
:1018A800B8EEE67A114BC7EE277AC3ED007A05F059
:1018B8003DF90020FFF7ECFC0AF0A7F9BDE8F04776
:1018C80002F07CBDAC0D00204F0D0020F40D00206F
:1018D80018260020302C00200C2C0020C8250020C1
:1018E800B501002011A20508A0250020D825002058
:1018F80008B500F0A5FEFEF77FFC00F04FF800F0F9
:101908006FF8FEF789FEFEF7DDFCFFF769F801F0D6
:10191800A7FAFFF72DFE01F079F8FEF713FD01F0A5
:101928009BF900F06DFB00F081FD00F013FE00F064
:101938005FFABDE8084000F02DBB10B5044628B991
:101948000F48104A104B532102F060FF0F4B1868E4
:10195800844213D010B1C36900219847002004F0D5
:1019680095F9002004F07CF94FF6FF7004F062F955
:10197800E369204601219847044B1C6010BD00BF55
:1019880025A20508E41F040841A20508500C002000
:101998000048D2E7D41700200CF028BD10B5084C39
:1019A800204602F0D2FA00200649074A02F084F8DD
:1019B800D22102462346FA20BDE8104002F094B92D
:1019C800380E00205FA20508A1190008024B034841
:1019D80001221A70FFF7B1BFA4250020A01400202F
:1019E8002DE9F743374D384F384E0024284602F08A
:1019F800ACFA2246234647F6FF7135480094019415
:101A080001F062FB4FF6FF788146414622462346A5
:101A180038460094019401F057FB41463060224655
:101A2800234638460094019401F04EFB414670600D
:101A38002246234638460094019401F045FB23468C
:101A4800B0604146224638460094019401F03CFBC0
:101A58002049F060204A204602F02EF81F49204A0B
:101A68000746204602F028F8214680464A462B467B
:101A7800204602F039F93C2132682B46192002F041
:101A880033F95A2172682B46192002F02DF9782172
:101A9800B2682B46192002F027F99621F2682B46E6
:101AA800192002F021F9D2213A462B46EC2002F007
:101AB8001BF99C20D22142462B4603B0BDE8F043D7
:101AC80002F012B91012002012A50508540C0020CB
:101AD80051A205085EA20508D519000867A20508E5
:101AE800A51C000870B5474E474C327847492DED84
:101AF800028B142592B005FB02420C320FA814F099
:101B080079FF33780D2B05FB03F504EB050332D879
:101B1800D3ED016A9B6807EE103A6359B8EEE68A7E
:101B280006EE903ADFED3A7AF8EEC78AB8EEE67A32
:101B380088EE278AC8EEA78AC7EE277A17EE900A9A
:101B480010F0E2F802460B466846324914F052FF9C
:101B580018EE100A10F0D8F802460B4605A82E49D0
:101B680014F048FF18EE900A10F0CEF802460B4623
:101B78000AA82A4929E093ED017A9B6807EE903A72
:101B8800635906EE903AF8EEE78AF8EEE67AB8EE90
:101B9800C78A17EE900A10F0B7F802460B46684657
:101BA8001F4914F027FF18EE100A10F0ADF802468E
:101BB8000B4605A81B4914F01DFF18EE900A10F0FB
:101BC800A3F80B46184902460AA8184C14F012FF4D
:101BD8002068174901F062FA20680FA901F05EFA3F
:101BE8006068694601F05AFAA06805A901F056FA3A
:101BF800E0680AA901F052FA02F0E0FB12B0BDEC6D
:101C0800028B70BD162600200000002070A2050877
:101C180000007A447BA205088CA205089DA205084D
:101C2800AEA20508BFA20508D0A20508540C0020E2
:101C38001BA5050808B5114B114A1B780D2B8CBF45
:101C480000210121117014225A430E4988588B181B
:101C58004FF47A720C495043086059684A430B495B
:101C68000A609A680A4B1A6009F066FD094B0A482F
:101C780001221A70BDE80840FFF75FBE1626002053
:101C8800F40D00200000002018260020302C002031
:101C98000C2C0020A4250020A0140020CAE700BFB7
:101CA8004FF6FF7070474FF6FF7070471FB5002959
:101CB80047D04FF2DE7003F0E9FF002004F0BCF8D3
:101CC8000F2003F0B7FF1F4C1F4A412101230A20B0
:101CD80004F0EAF8042004F0AFF8236828209621DD
:101CE800042B24DC0123194A04F0DEF803A90DF1C2
:101CF8000E02206804F060FB0F2003F09BFFBDF884
:101D08000C00BDF80E1014380F242822002380B2CE
:101D1800009403F0BFFFBDF80E10BDF80C0000944E
:101D2800143989B22822012303F0B4FF09E0084AD4
:101D3800012304F0B9F81E20A521064A012304F066
:101D4800B3F81FBD640C0020E1A20508F4A2050841
:101D580010A3050826A3050837B51E4C2368042BD5
:101D680005462BDC01A80DF1060104F023FBBDF8A4
:101D78000630BDF80420184904200DF079F82368CE
:101D8800002B04DA1548164A164B592105E0042B96
:101D980005DD1248124A144B5A2102F037FD04EBB4
:101DA8008302BDF8041001339180BDF8061023604A
:101DB800052BD18008D1201D04F07EFB00230B48A1
:101DC8002360FFF7BAFD03E028460121FFF76EFF05
:101DD8003EBD00BF640C00203DA3050882A3050892
:101DE800F61F0408A4A30508BBA30508E8150020EE
:101DF80037B50B4C204602F0A8F80A4B0A49009365
:101E080000250120094A0A4B019501F046FF2946A1
:101E180002462346284603B0BDE8304001F064BFBF
:101E2800B4120020B51C0008A91C0008AF1C00084B
:101E3800611D00084FF6FF7070474FF6FF7070473E
:101E480030B54FF6E07087B003F020FF002003F0B4
:101E5800F3FF0F2003F0EEFE00212C4A2C4C012347
:101E68000A2004F021F8002003F0E4FE042003F027
:101E7800E3FF0A201921274A012304F015F8252138
:101E8800254A01230A2004F00FF81F2003F0D2FE90
:101E980001230A203721214A04F006F82378002B71
:101EA80031D001231E2096211D4A03F0FDFF6288D0
:101EB8001C4902A814F09EFD01231E20A22102AA9B
:101EC80003F0F2FFA288184902A814F093FDAE218E
:101ED80002AA01231E2003F0E7FF0F2003F0AAFE49
:101EE8006088A188143880B20F2528220023009525
:101EF80003F0D0FEA18860880095143989B22822A1
:101F0800012303F0C7FE07B030BD00BFE9A30508F1
:101F18007C0C0020FBA305081BA405083BA40508AE
:101F28005EA4050870A405087DA4050801B187E72B
:101F3800704713B50DF1060101A804F0EFF9144B31
:101F480001221A705988BDF80420891A0E311C29FB
:101F580019460AD89C88BDF80600201A0E301C289D
:101F680003D899680131996001E000238B60084B20
:101F78009968012905DD00229A601A70FFF708FDAB
:101F880005E05A80BDF806209A80FFF759FF1CBD6E
:101F98007C0C002037B50B4C204601F0D6FF0A4BCD
:101FA8000A49009300250120094A0A4B019501F0CE
:101FB80074FE294602462346284603B0BDE8304051
:101FC80001F092BEE8150020351F00083D1E0008EC
:101FD800431E00083B1F000808B5064B00221A7074
:101FE800054B186814F09CF90448BDE80840FFF751
:101FF800A4BC00BFA4250020F0350020D417002081
:102008002DE9F04F514D524E85B00024284601F07D
:102018009CFF2246234647F6FF714E4800940194E0
:1020280001F052F84FF6FF770390394622462346CF
:1020380049480094019401F047F839463060224637
:10204800234646480094019401F03EF84FF00108F9
:102058007060224623464FF6E0714148CDF8008073
:10206800019401F031F82346B060394622463D48D4
:10207800CDF80080019401F027F83B49F0603B4A15
:10208800204601F019FD3A493A4A0746204601F030
:1020980013FD3949394A8046204601F00DFD38497B
:1020A800384A8146204601F007FD3749374A8246BB
:1020B800204601F001FD3649364A8346204601F0A4
:1020C800FBFC21468446039ACDF808C02B462046DF
:1020D80001F00AFE3C2132682B46142001F004FE70
:1020E8003C2172682B46EC2001F0FEFDB421B26859
:1020F8002B460F2001F0F8FDD2213A462B46E62068
:1021080001F0F2FD642142462B46052001F0ECFD6A
:102118004A462B460520872101F0E6FD52462B460C
:102128000520D22101F0E0FDD2215A462B4650204D
:1021380001F0DAFDDDF808C09B20D22162462B466B
:1021480005B0BDE8F04F01F0CFBD00BFDC0E0020A8
:10215800880C00208AA4050894A405080EA2050886
:1021680010A5050812A505085EA20508E11F0008CC
:10217800F89F0508C921000808A00508C922000819
:102188009DA40508D1230008A5A405088D230008EF
:10219800ADA405084923000808B50BF065FE4FF407
:1021A80041400CF09DFB044B186807F04BF8034BBB
:1021B80009221A7008BD00BF10260020A42500209F
:1021C80010B50C4CFFF7E8FF0B4A0023B42005219B
:1021D80003F06AFEA0684FF6E07100F0B1FFA06856
:1021E800064900F05BFF0BF03FFEBDE8104002F02F
:1021F800E5B800BF880C002018A50508B5A4050897
:10220800264B2DE9F7431888C00014F081F80546DD
:1022180028B90520B421224A2B4603F045FE214B5C
:10222800DFF878801D6000240BF01EFE26461E4F46
:10223800DFF8889023E009F0D7F83B68D9F8000068
:1022480045F8083C7B6845F8043C184B1B68C018E7
:1022580006F0F8FF164B186809F088F9B8F800007E
:1022680094FBF0F080B24FF4FC63009328210246FF
:10227800322303F06BFC04F59E7401360334B8F87E
:1022880000300835B342D6DA0A4B186806F0DAFF90
:10229800094B09221A70BDE8FE8300BFFC390020F3
:1022A800CEA40508F0350020BC3700209C2500206E
:1022B800C825002010260020A4250020F83500207D
:1022C80010B5094CFFF79CFFA0684FF6E07100F0CD
:1022D80037FFA068054900F0E1FE0BF0C5FDBDE839
:1022E800104002F06BB800BF880C0020DCA4050881
:1022F80010B5074C4FF6E071A06800F021FFA06808
:10230800044900F0CBFEBDE8104002F057B800BF0A
:10231800880C0020F6A4050810B5074C4FF6E071AC
:10232800A06800F00DFFA068044900F0B7FEBDE802
:10233800104002F043B800BF880C00200CA5050827
:1023480010B50C4C0B2323700B4B01221A70002084
:1023580002F06AFF0948FFF7F0FA2078FEF7BCFBA5
:10236800074B032093ED000A0BF08DFDBDE81040EC
:10237800D2E700BF242C0020500D00203017002089
:102388000C03002038B50C4D0C232B700B4B01248B
:102398001C70002002F048FF0948FFF7CEFA2878A1
:1023A800FEF79AFB074B204693ED000A0BF06BFDF6
:1023B800BDE83840B0E700BF242C0020500D0020B5
:1023C800301700200C03002010B50C4C0923237093
:1023D8000B4B01221A70002002F026FF0948FFF774
:1023E800ACFA2078FEF778FB074B022093ED000A41
:1023F8000BF049FDBDE810408EE700BF242C0020FB
:10240800500D0020301700200C0300200CF0B4B849
:10241800034A044800231370034A1370FFF78DBA68
:1024280004380020D4170020A42500202DE9F74304
:10243800384D394EDFF8FC800024284601F085FD30
:102448002246234647F6FF7134480094019400F071
:102458003BFE4FF6FF7781463946224623463048F1
:102468000094019400F030FE39463060224623463D
:1024780040460094019400F027FE394670602246D9
:10248800234640460094019400F01EFE2346B060A7
:102498003946224640460094019400F015FE214931
:1024A800F060214A204601F007FB2049204A0746F0
:1024B800204601F001FB214680464A462B4620462D
:1024C80001F012FC3C2132682B46282001F00CFC5C
:1024D8005A2172682B46192001F006FC7821B2684F
:1024E8002B46192001F000FC9621F2682B46192092
:1024F80001F0FAFBD2213A462B46EC2001F0F4FB1E
:102508000520D22142462B4603B0BDE8F04301F036
:10251800EBBB00BF24100020980C002026A505085E
:102528002EA505085EA205081924000839A5050886
:102538001524000812A50508034A0448002313704F
:10254800034A1370FFF7F9B904380020D4170020A4
:10255800A42500202DE9F743324E334DDFF8DC8007
:102568000024304601F0F1FC2246234647F6FF716D
:102578002E480094019400F0A7FD4FF6FF7781469E
:102588003946224623462A480094019400F09CFDCF
:10259800394628602246234640460094019400F0BC
:1025A80093FD3946686022462346404600940194CC
:1025B80000F08AFD2346A86039462246404600942A
:1025C800019400F081FD1B49E8601B4A204601F098
:1025D80073FA214607464A463346204601F084FBF3
:1025E8003C212A683346192001F07EFB5A216A688B
:1025F8003346192001F078FB7821AA683346192060
:1026080001F072FB9621EA683346192001F06CFB51
:10261800EC20D2213A46334603B0BDE8F04301F03E
:1026280063BB00BF78180020A80C002041A505084E
:102638004FA505085EA205084125000812A5050852
:1026480010B50B4C204601F080FC002001462246C4
:1026580000F09AFD00200749074A01F02DFAD2211F
:10266800024623464FF48270BDE8104001F03CBB9F
:10267800301700205CA50508A926000870B5C924F4
:102688000AE0A8B200223146013502F05DFCF02DC7
:10269800F7D10134EF2C02D00025A6B2F1E770BDC6
:1026A80010B51A4C2378092B08D1194A0023137046
:1026B800184A1370FFF7E2FF174823E00A2B0ED1E0
:1026C800164B186813F02CFE154A00231370114A94
:1026D8001370144A1370FFF7D1FF134812E000205B
:1026E80002F0A2FD114A00231360114A13800D4B1A
:1026F80002221A700F4B186806F0A4FD22780E4BC0
:102708000E481A70BDE81040FFF717B9A42500203D
:10271800500D00204F0D0020DC0E0020F035002069
:10272800510D002004380020241000209C0D0020AA
:10273800AA0D002010260020C22500206C110020C0
:10274800034B01224FF4FC601A7003F073BA00BF08
:102758004F0D0020044B054800221A70044B0C2230
:102768001A70FFF7EAB800BF4F0D00207818002054
:10277800A425002007B50A4A0023137004228DE817
:102788000C00C6201022232356210CF01BFA054BFF
:1027980005480A221A7003B05DF804EBFFF7CDB8BC
:1027A8004F0D0020A42500202410002007B50A4A58
:1027B8000023137004228DE80C0097201022232395
:1027C80056210CF0FFF9054B054809221A7003B091
:1027D8005DF804EBFFF7B1B84F0D0020A4250020E9
:1027E800DC0E002007B50B4B00221A7008220323C9
:1027F8008DE80C004920102223233D210CF0E2F93A
:10280800054B064801221A7003B05DF804EBFFF788
:1028180094B800BF4F0D0020A4250020A01400206C
:1028280008B501214FF080400EF01DFB0A4B002037
:1028380018700A4B18700A4B18700A4B08221A7045
:10284800094B187003F022FA084B094801221A7044
:10285800BDE80840FFF771B8C3250020AC0D002083
:102868004F0D0020A4250020242C0020083600202D
:10287800380E002070B51F4C1F4E20684FF6E075CB
:10288800294600F05DFC20681C4900F007FC6068E0
:10289800294600F055FC6068194900F0FFFBA06864
:1028A800294600F04DFCA068164900F0F7FB01F03E
:1028B80085FD4FF47A6008F059FE2068294600F03B
:1028C8003FFC2068314600F0E9FB6068294600F0CB
:1028D80037FC6068314600F0E1FBA068294600F04B
:1028E8002FFCA068314600F0D9FBBDE8704001F02C
:1028F80065BD00BFB80C002015A5050887A105080F
:102908009BA10508ABA105080C4B10B500241C7051
:102918000B4B01221A70204608F04EFF204603F0A8
:10292800B5F9084B0B221A7009F08AFA09F071FF01
:102938000548BDE81040FFF700B800BF4F0D002064
:10294800242C0020A4250020441500200F4A002331
:1029580010B513700E4A13700BF088FD044628B1A9
:10296800FFF788FFBDE8104001F028BD03F08EF99D
:1029780009F08CF9074B1C70074B07221A7009F0F5
:102988007FF90648BDE81040FEF7D7BFAC0D002020
:102998004F0D0020242C0020A425002058130020CF
:1029A80010B54FF0804001210EF05DFA114A002366
:1029B8001370114A1370114A13700BF057FD044637
:1029C80028B1FFF757FFBDE8104001F0F7BC03F04E
:1029D8005DF909F05BF906F08DFC094B1C70094B99
:1029E80006221A7009F04CF90748BDE81040FEF7B6
:1029F800A4BF00BFC3250020AC0D00204F0D002050
:102A0800242C0020A4250020800F00202DE9F04F61
:102A18006D4DDFF810928BB000244FF6FF782846F2
:102A280001F093FA414622462346684800940194EF
:102A380000F04AFB4FF6E076042704903146224620
:102A4800234663480097019400F03EFB3146059009
:102A5800224623465F480097019400F035FB414623
:102A680006902246234648460097019400F02CFB26
:102A7800594E414630602246234648460097019405
:102A880000F022FB234670604146224648460097E4
:102A9800019400F019FB5149B060514A204601F0F9
:102AA8000BF85049504A0746204601F005F84F49AF
:102AB8004F4A8046204600F0FFFF4E494E4A814665
:102AC800204600F0F9FF4D494D4A8246204600F065
:102AD800F3FF4C494C4A8346204600F0EDFF4B4932
:102AE8004B4A84462046CDF80CC000F0E5FF494922
:102AF8000790494A204600F0DFFF48490890484AB5
:102B0800204600F0D9FF21460990049A2B4620461A
:102B180001F0EAF82146059A2B46C82001F0E4F8AE
:102B28000A21069A2B46C82001F0DEF855213268A2
:102B38002B46782001F0D8F8692172682B46782056
:102B480001F0D2F87D21B2682B46782001F0CCF84C
:102B580005203A4628212B4601F0C6F8D2214246E4
:102B68002B46052001F0C0F8D2214A462B465620B4
:102B780001F0BAF8D22152462B46A62001F0B4F84B
:102B8800B4215A462B46052001F0AEF8DDF80CC0FA
:102B9800B42162462B46562001F0A6F8B421079AC4
:102BA8002B46A62001F0A0F8B421089A2B46F6205F
:102BB80001F09AF8099AF620D2212B460BB0BDE80D
:102BC800F04F01F091B800BFD417002061A50508A7
:102BD8006AA5050877A50508B80C002082A5050890
:102BE800ED2700088AA505081129000893A50508FE
:102BF800A92900089CA5050855290008A5A50508C8
:102C080029280008AEA50508B5270008B7A50508B6
:102C18007D270008C0A505085D270008C8A5050888
:102C28004927000812A5050807B5032308228DE8DF
:102C38000C004920102223233D210BF0C3FF044B35
:102C4800044801221A7003B05DF804EBFEF775BE64
:102C5800A4250020A01400202DE9F743314E324F5F
:102C6800324D0024304601F070F92246234647F6DB
:102C7800FF712F480094019400F026FA4FF6FF7870
:102C8800814641462246234638460094019400F086
:102C98001BFA414628602246234638460094019490
:102CA80000F012FA414668602246234638460094EE
:102CB800019400F009FA2346A860414622463846A6
:102CC8000094019400F000FA1A49E8601A4A204674
:102CD80000F0F2FE214607464A463346204601F0F8
:102CE80003F83C212A683346192000F0FDFF5A21D9
:102CF8006A683346192000F0F7FF7821AA6833463E
:102D0800192000F0F1FF9621EA683346192000F0F7
:102D1800EBFFEC20D2213A46334603B0BDE8F0433E
:102D280000F0E2BFC810002012A50508C40C00205E
:102D3800D0A505085EA20508312C00081C4B1A789E
:102D48001C4B10B51A7009F081F81B4B1B4A002464
:102D58001C6002202346CA2103F0A6F8204608F08A
:102D68002BFD174B1C80174B1C70174B1B78023B15
:102D7800052B1CD8DFE803F003070B13170FBDE87A
:102D88001040FEF773BABDE81040FEF75DBABDE823
:102D98001040FEF747BABDE81040FEF71FBABDE87D
:102DA8001040FEF72DBABDE81040FEF705BA10BD79
:102DB800C2250020A42500209C0D002011A505088F
:102DC8000436002004380020242C002008B5084BC5
:102DD800186806F037FA002002F058FF09F030F8BA
:102DE800044B05480B221A70BDE80840FEF7A5BD44
:102DF80010260020A425002044150020114B10B5F2
:102E080000241C70104B186806F01CFA204602F0CB
:102E18003DFF0E4B1B780B2B0ED8DFE803F00606A0
:102E28000D0D0D0D0A080D0D0D06094802E00948A3
:102E380000E00948FEF781FD084B1C70BDE8104012
:102E480008F0FEBF242C002010260020A425002016
:102E5800D417002058130020800F002004380020C9
:102E68002DE9F041144C204601F06FF80020134979
:102E7800134A00F021FE1349134A0746002000F0C8
:102E88001BFE1249124A0646002000F015FED22108
:102E980005463A462346E62000F026FF4B213246F7
:102EA8002346642000F020FF642069212A46234637
:102EB800BDE8F04100F018BF6C1100206BA00508B8
:102EC800052E0008D8A50508D52D0008E4A5050895
:102ED800452D000808B508B143682BB90348044AD2
:102EE800044B9B2101F092FC586908BDF1A5050827
:102EF8000820040813A6050808B5FFF7EBFF80684B
:102F0800123080B208BD08B5FFF7E4FF406806300C
:102F180080B208BD2DE9F84F04468846FFF7DAFF6E
:102F28006689E589074606F1030905F10F0AB8F134
:102F3800000F1FD01F2002F07DFE2046FFF7DCFFA8
:102F480083462046FFF7DFFF294603465FFA8BF2E8
:102F5800F0B202F0AFFE042002F06EFF0B364FF61F
:102F6800FF70033502F066FEB0B2A9B23A680123D9
:102F780002F09AFF3D69204641464A465346A84713
:102F8800BDE8F88F13B504460DF1060101A803F05A
:102F9800C5F92046FFF79EFF6389BDF80410BDF808
:102FA8000620C91AE389D21A0339C3680F3A2046A2
:102FB80098471CBDF7B5044614200D4616461F4613
:102FC80013F0A6F9089BC7600361064B0649074A38
:102FD80080E8700000930190054B002000F05DFE32
:102FE800FEBD00BF1D2F00080F2F0008012F00088D
:102FF8008D2F0008704708B508B143682BB90448FD
:10300800044A054BAD2101F001FC586908BD00BF19
:1030180032A605082020040813A60508F8B50546B9
:103028000E46FFF7E8FF836B04461BB1284631467E
:10303800984700E018466F8994F83C30ED890EB93E
:10304800034310D0208E02F0F5FD608E02F008FEDA
:1030580094F8350002F0F0FE94F8343038462946EA
:10306800224602F021FF002384F83C30F8BD08B561
:10307800FFF7C1FF90F83500BDE8084002F0F1BE47
:1030880038B5FFF7B8FF044613F03AFD054694F843
:10309800350002F0E1FE684380B238BD38B50D4610
:1030A800FFF7A9FF29462E22044613F059FD50B117
:1030B800204629462E2213F0A5FD002384F82E3041
:1030C800012384F83C3038BD2DE9F74307464020FA
:1030D8000E461546984613F01BF9044628B91148C0
:1030E800114A124B4E2101F091FB114B114A124922
:1030F8008DE818000020114B00F0CFFD39468146BD
:10310800FFF7CCFF9DF82830268684F835300B9BD6
:103118006586A363002384F8348084F83C304846ED
:10312800BDE8FE8332A605083820040850A6050825
:10313800253000087730000889300008FD2F000886
:1031480010B50C46FFF757FF0123048680F83C3082
:1031580010BD00BF4FF4A0707047C820704770477B
:10316800074B1B78022B07B508D1064B1B78022B9F
:1031780004D001A80DF1060103F0D0F80EBD00BF80
:1031880004380020242C002073B50A4B06460D464F
:103198001446009300200849084A094B019000F0A2
:1031A8007CFD294602462346304602B0BDE8704001
:1031B80000F09ABD673100085D31000863310008EE
:1031C8006931000813B502AB03E90600436843B14F
:1031D800027C0124082A9C7004D11B692146984767
:1031E80000E01C4620461CBD30B500282BD0058BBE
:1031F800002425E0036A1A7C012A05D15B681A8835
:103208008A421BD1187F30BD052A06D15B681A880F
:103218008A4213D193F82C0030BD032A06D15B688B
:103228001A888A420AD193F8250030BD062A05D1AA
:103238005B681A888A4201D1D87A30BD01340430DB
:10324800AC42D7D3002030BD08B18175012070474A
:10325800F8B504460D46D0B1E175D0F898309847D6
:10326800012D0DD12746002606E0F86900F1080275
:10327800436906CA98470136238B04379E42F4D324
:10328800D4F898302046294698470120F8BDF8BD63
:10329800F8B50546084617460E4613F031FC013FBF
:1032A800B84234BF04463C463CB128463146224623
:1032B80013F0A8FC00232B55F8BD2C70F8BDF7B50A
:1032C800044600200090019000296CD00E8B68E025
:1032D80000F1080351F823301D7C042D04D15D68EA
:1032E8002D88954247D0013000F1080351F823306A
:1032F8001D7C012D04D15D682D8895423BD001309D
:1033080000F1080351F823301D7C052D04D15D68B8
:103318002D8895422FD0013000F1080351F8233051
:103328001D7C032D04D15D682D88954223D0013082
:1033380000F1080351F823301D7C022D04D15D688B
:103348002D88954217D0013000F1080351F8233039
:103358001D7C072D04D15D682D8A95420BD0013064
:1033680000F1080351F823301D7C062D08D15D6853
:103378002D88954203D103F10801204615E001305C
:1033880000F1080351F823502B7C082B09D16F68F2
:103398003F88974204D105F1080120461A4605E006
:1033A8000130B04294D320466946082213F060FAEF
:1033B8002046FEBDF8B505460F461646002830D013
:1033C8004388032B2FD0202012F0A2FF04460028A8
:1033D8002BD040F80C5B39460C22FFF759FF182018
:1033E800E66112F095FF0646B8B102230374012383
:1033F80063760F4B446063600E4BA3600023237613
:103408006B8805EB830201339BB2012B50606B8004
:103418000CD16A685268137608E0204612F080FFE3
:1034280004E0064602E0002600E006463046F8BD05
:10343800849F0408229C040837B5456802AB03E959
:1034480006003DB3037C0124042B85F8314022D1CA
:10345800688E02F0EFFB95F8300002F0EDFC95F86D
:10346800343043B9BDF80200BDF80610AA1C234643
:1034780002F01AFD0FE0012B03D1084840F2395140
:1034880004E0022B07D1054840F24151044A054B9C
:1034980001F0BCF92C4620463EBD00BF63A60508D6
:1034A800F86A040861A60508F8B504460F461646EA
:1034B80010B3838A0A2B20D0202012F029FF05465A
:1034C800E8B14460102200F108003946FFF7E0FE39
:1034D8004FF6FF73A08A2B801F236B8000232B7667
:1034E800831D013080B20128EE6144F82350A08288
:1034F80007D1A3691876F8BDF8BD0020F8BD0120F2
:10350800F8BD0120F8BD2DE9F3471D464B1C984234
:1035180082460C461746BDF828600DDD95420BDC47
:1035280001320AF101035B1A521BC8B2D2B29BB234
:103538002946009602F0B6FBAAF1020A3046C4EB0F
:103548000A0A02F077FB4FF000084FF001091FFA52
:103558008AFA0BE0601C08EB050180B289B252467A
:103568000023009602F096FB09F101097B1B08F184
:10357800010899451FFA88F8ECD3BDE8FC87F8B52F
:10358800C7B2144638461E460D4602F095FB621E29
:1035980092B23846294602F08FFB304602F04AFBC9
:1035A800022606E0A21B92B23846294602F084FBA6
:1035B8000136A642F6D3F8BD73B504460E4600F1AF
:1035C8001E001546009200233C2280B21E3E02F0E7
:1035D80061FBB1B220463C220123009502F05AFB60
:1035E8007CBD73B504460E4601381546009200238B
:1035F800032280B2013E02F04DFBB1B22046032205
:103608000123009502F046FB7CBDF7B5089D2E7B93
:10361800EF7A1C463604AB7A06EB0726F618431AEF
:10362800687B06EB00602D1800200190121B0846ED
:103638002146009501F026FFFEBD30B5456885B0EE
:1036480004AB03E906007DB101242C736D68BDF855
:103658000800BDF80A109DF80C209DF80E30009562
:10366800FFF7D3FF204600E0284605B030BD2DE91E
:10367800F04385B004AB03E906004468BDF8086070
:10368800BDF80C70002C41D0012384F8263094F842
:1036980025300BB9A26800E06268FFB2BDF80A10D5
:1036A8009DF80E30009230463A46FFF7AEFF04F11F
:1036B8000C08022002F0C0FB404613F021FA054630
:1036C80000B1451E0F3F0024153E1FFA87F90DE093
:1036D80002F0BCFB02F0C0FB04FB106189B2484653
:1036E8002022002302F0FAFB0134E4B2AC42EFD30B
:1036F800002002F09FFAB8B2B1B24246012302F0AC
:10370800EDFB002002F098FB012000E0204605B008
:10371800BDE8F0832DE9F04385B004AB03E906006A
:103728004568BDF80860BDF80C70002D3CD0012339
:103738006B762B7EBDF80A10012B0CBF6A68AA684D
:103748009DF80E300092FFB23A463046FFF75DFF13
:103758000C35022002F070FB284613F0D1F90E3F19
:1037680081460024163E1FFA87F80DE002F06EFB32
:1037780002F072FB04FB106189B24046202200234C
:1037880002F0ACFB0134E4B24C45EFD9002002F062
:1037980051FAB8B2B1B22A46012302F09FFB0020C9
:1037A80002F04AFB012000E0284605B0BDE8F0839E
:1037B8002DE9F04F85B00546DDF840900291484666
:1037C8009046039313F09CF9DDF838A0DDF83CB07F
:1037D8000646294600242F4611E024B1B4420CBF06
:1037E8005B46534600E0039B01F10805ADB2009328
:1037F8002846029A4346FFF708FF01342946B44297
:10380800EBDD002002F016FA022002F015FB7D1D08
:1038180008F10508A8B21FFA88F14A46012305B045
:10382800BDE8F04F02F040BB70B5406886B006AB0B
:1038380003E9060000282ED0012380F82D30866881
:10384800164BF21A534243EB020390F82C205AB15C
:10385800002B134D134B144A08BF1D46134B00F1A0
:103868001C0418BF13460AE0002B0D4D0D4B0E4AE1
:1038780018BF1D460D4B00F10C0408BF1346BDF8D8
:103888001200BDF81410BDF8162000960195029498
:10389800FFF78EFF012006B070BD00BF68740408F2
:1038A800A47004084A760408867204082C78040870
:1038B80070B5446886B006AB03E9060004B301237B
:1038C8006377A668104B227FF11A4B4243EB010342
:1038D8000AB10BB904E01BB966680C4D0C4B01E04A
:1038E8000C4D0D4BBDF81200BDF81410BDF8162094
:1038F80000960C3401950294FFF75AFF012000E06E
:10390800204606B070BD00BFB47F0408F07B0408F1
:10391800D27D04088A810408608304082DE9F043F5
:1039280085B004AB03E906004468BDF80860BDF83B
:103938000A90BDF80C50BDF80E80002C00F08C8069
:103948000123A3740220676802F076FA4FF6FF702D
:1039580002F086F9002002F06DF9EDB25FFA88F8FE
:10396800A6F1160189B230462A4643460097FFF76A
:103978004CFE277A002F2ED1A28A234600E0013779
:10398800974204D29969097E04330029F7D002F0DE
:103998005DFA02F061FAA9F116091FFA89F90E21F8
:1039A80001FB10914FF6FF7208F101085FFA88F3E6
:1039B80089B2009248462A46FFF7A5FD022002F088
:1039C8003BFA1F2002F036F9A38A002B38D0103DAD
:1039D800E8B2303E2CE0E3685C68A28A2346013AEC
:1039E800002700E00137974204D29969097E043321
:1039F8000029F7D002F02AFA02F02EFA0E2101FB74
:103A080010914FF6FF7208F101085FFA88F389B246
:103A1800009248462A46FFF776FD022002F00CFA8B
:103A28001F2002F007F9A38A53B1103DE8B21A3EED
:103A38000637B1B254F827200123083202F04EFAB3
:103A4800002002F0F9F94FF6FF7002F009F91F2083
:103A580002F0F0F8012000E0204605B0BDE8F08350
:103A68002DE9F04105463620884614461F4612F0D7
:103A78004FFC0646E0B120F8025B41462E22FFF7D4
:103A880007FCBDF8183086F83440738618200123E7
:103A980086F8307086F8313012F03AFC044618B1D6
:103AA80004234660037404E0304612F039FC00E059
:103AB80004462046BDE8F081F8B5064624200F46A6
:103AC800154612F025FC0446D8B10F4B06808360DA
:103AD8000E4B39464360102200F10C00FFF7D8FB6B
:103AE80001260023182025622377667712F010FC40
:103AF800054610B14460067404E0204612F010FC3C
:103B080000E005462846F8BDB47F04080E7A04088C
:103B1800F8B506462C200F46154612F0F9FB044668
:103B2800E8B120F80C6B39461922FFF7B1FB0D4BB1
:103B3800A562A3600C4B6360002384F8253018202D
:103B4800012384F8263012F0E3FB054618B103235D
:103B58004460037404E0204612F0E2FB00E00546EE
:103B68002846F8BDC09804085E95040810B50446B8
:103B7800142012F0CDFB20B100234380014B0480B8
:103B8800036110BDBD33000838B50546442012F066
:103B9800BFFB0446C0B10E4B058243600D4B03606A
:103BA800012383740023037283820B4B0364182060
:103BB80012F0AEFB054618B107234460037404E015
:103BC800204612F0ADFB00E00546284638BD00BF90
:103BD800549104084A8D0408B13400082DE9F041D5
:103BE80005463420884614461F4612F091FB0646C7
:103BF80020B3144B05808360134B41464360102269
:103C080000F10C00FFF744FB214606F11C001022CE
:103C1800FFF73EFB002386F82C301820012337637A
:103C280086F82D3012F074FB044618B1052346605F
:103C3800037404E0304612F073FB00E004462046AB
:103C4800BDE8F08168740408C26E04082DE9F041EB
:103C5800044614200D461646984612F059FB0746AE
:103C6800B8B1069B048003610023C3720123456039
:103C7800068180F80A800373182012F049FB044675
:103C880018B106234760037404E0384612F048FB75
:103C980000E004462046BDE8F0812DE9F0410446E5
:103CA80018200D461646984612F032FB0746B8B162
:103CB80001238370069B04800361079B456086602F
:103CC800C0F80C804361182012F022FB044618B19A
:103CD80008234760037404E0384612F021FB00E033
:103CE80004462046BDE8F0812DE9F34198461B8B38
:103CF8001D2B05460C4617464FF0000000F2B48015
:103D0800B5F5A07F0090019000F2AE80F02900F296
:103D1800AB80127CADF80610511EADF80250072991
:103D280000F28A80DFE801F045595E04456A14769E
:103D38007B684E4A7A611A8893F834303A80013B9E
:103D4800DBB2012B7FD8ADF80240ADF806507AE01F
:103D580005F11602ADF8002004F11602ADF80420B2
:103D680002AE434A16E903007A6107F1080282E8C5
:103D7800030003F10802013348F82270A8F818304C
:103D88007B681A8A187A3A8000286CD1FFF7FCFE03
:103D98003849436859603849DF600126163D196083
:103DA80002461E72A8B2E1B24346FFF79DFF3046B5
:103DB8005AE0012A0CBF314B314B78687B6130F8EF
:103DC8000C3B3B8012F09CFE431CDB001A34ED18C0
:103DD800ADF80440ADF8005035E07B68294A1B680F
:103DE8007A6102E0284A7B687A611B8814353B8037
:103DF800ADF800501434ADF8044024E07B68234A41
:103E08007A611A883A801A899B7AAD18ADF8005001
:103E1800E418F0E77E681E4B7B61338838463B80A8
:103E280073689847013D4519ADF80050B3683846A6
:103E38009847013C0419DEE71648174A174B40F229
:103E48001A3100F0E3FC02AA12E9030007F10803A3
:103E580083E80300B8F8183003F10802013348F882
:103E68002270A8F818300120BDE8FC814134000810
:103E7800253900084089040836850408B93800083F
:103E8800313800081D370008773600084336000827
:103E9800CD31000863A60508086B040861A605086B
:103EA800F8B51646002834D01378002B2ED0028B94
:103EB800002327E0046A257C042D21D165682F881A
:103EC8008F421DD195F8313053B16F8E01F0D8FE75
:103ED80004F1080268866369204606CA98476F8617
:103EE800A81C31462E22FFF7D3F995F831307BB163
:103EF80004F108026369204606CA98470120F8BD04
:103F0800013304309342D5D30020F8BD1846F8BDDC
:103F18000120F8BD70B5B8B1068B0446002310E047
:103F2800256A287C04280AD16D682888884206D129
:103F38001046A91C2E22FFF7ABF9012070BD0133F2
:103F48000434B342ECD3002070BD38B5044620B326
:103F5800134BC361134BC0F89830134BC0F89C3017
:103F6800124B00257822C0F8A0308575C5750583E9
:103F7800294600F1200012F0BDFCD4F89830204604
:103F8800294698470A4A1388312B07D8094941F826
:103F9800234001331380012038BD38BD284638BD81
:103FA8005932000851320008F1310008C7320008C0
:103FB800D40C00201C1900202DE9F04104460028EB
:103FC80000F0B380078B02460025A8E0136A1E7C28
:103FD800042E00F08780012E23D1586803888B4275
:103FE80040F09B8005F1080712F09AF954F8270071
:103FF8004FF00008C0F8048012F092F9228B531E8B
:104008009D4208D00732238354F8221044F8271021
:1040180044F8228002E044F8278025833046BDE832
:10402800F081052E5ED0032E5CD0022E13D15B6882
:10403800186803888B4270D14388013B9BB2438048
:104048000BB912F06DF905F1080654F826305868D6
:1040580012F066F94EE0072E21D15E68338A8B4252
:104068005BD1002706E0BB1D013756F8230012F08C
:1040780057F9FFB2B38ABB42F5D80027B78205F1DA
:10408800080654F82630586812F04AF954F8260001
:1040980033E044F8267025830120BDE8F081062E20
:1040A8001ED1586803888B4237D105F1080612F0F3
:1040B80037F954F826000027476012F031F9228BAF
:1040C800531E9D4209D00833013A54F82310228325
:1040D80044F8261044F82370DEE744F826701AE006
:1040E800082E1AD1586803888B4216D112F018F995
:1040F80005F1080654F826000027476012F010F969
:10410800228B531E9D42C4D0073254F8221044F823
:10411800261044F822702383BEE701350432BD42DD
:10412800FFF454AF0020BDE8F081BDE8F08170B520
:10413800044600282AD0068B751E083600EB860632
:104148001EE056F8043D1A7C042A13D0012A11D027
:10415800052A0FD0032A0DD0022A02D15B681B68FA
:1041680009E0072A02D15B68198A05E0062A01D00E
:10417800082A04D15B6819882046FFF71DFF013D16
:10418800681CDED100232383012070BD70BDF0B50B
:1041980028B30023068B1A461EE0046A257C072DE7
:1041A80018D16468258A8D4214D1A78A002504EBAA
:1041B80083040DE004EB050C0435DCF818C09CF80A
:1041C80018C0BCF1010F03F1010301D1D8B2F0BD51
:1041D800BB42EFD301320430B242DED30020F0BD3F
:1041E80070B508B3048B00231BE0026A157C072D09
:1041F80015D15268158A8D4211D10023958A11462E
:104208001C46012007E013B99669307601E08E69F3
:10421800347601330431AB42F5D3012070BD01334C
:104228000430A342E1D3002070BD2DE9F04128B34A
:104238000023078B1A461EE0046A257C072D18D137
:104248006468258A8D4214D1B4F814C0002504EBA3
:1042580083040CE066190435B66996F81880B8F13D
:10426800010F03D106F10800BDE8F0810133634571
:10427800F0D301320430BA42DED30020BDE8F08129
:104288002DE9F04700282FD00023B0F818C01D46AC
:1042980027E0046A267C072E21D16468268A8E428C
:1042A8001DD1B4F81480002604EB830915E009EB4E
:1042B8000604A7693C7E012C0DD192F800A0BAF142
:1042C800000F08D007F1080011461022FEF7E0FFA2
:1042D8002046BDE8F087013304364345E7D301356E
:1042E80004306545D5D30020BDE8F087F0B5B0B1FE
:1042F800068B002510E0046A277C062F0AD1646823
:1043080027888F4206D123819DF814306260A372FA
:104318000120F0BD01350430B542ECD30020F0BDDA
:1043280010B500210446FEF793FF20460121BDE8A1
:104338001040FEF78DBF38B598B1048B02460023B4
:104348000CE0106A058804328D4206D100F108029B
:10435800436906CA9847012038BD0133A342F0D308
:10436800002038BD10B50C460021FEF771FF20462D
:104378000121BDE81040FEF76BBF13B502AC04E99C
:104388000C00BDF80230834206D8BDF800308342E5
:1043980034BF0020012000E00020BDF806308B4229
:1043A80006D8BDF804308B4234BF0021012100E05B
:1043B8000021002818BF0846C0B21CBD38B5114BF3
:1043C800114A1988002319E052F8045FA87D0128D2
:1043D80012D100240CE004F1080355F82300037CF3
:1043E800082B03D1436800211B6998470134A4B204
:1043F8002B8BA342EFD838BD01339BB28B42E3D15C
:1044080038BD00BFD40C002018190020704770B5C3
:10441800094CA5787DB9094B1E78012E0BD163682C
:10442800013363606268064B9A4204D9284601F05A
:10443800C5FCA670656070BDD40C00208401002006
:1044480040420F00054A9060134602E0996801391E
:10445800996091680029F9D1704700BFD40C0020F9
:10446800F0B585B001F058FF002800F0498100251B
:1044780002A80DF10A01ADF80850ADF80A5001F094
:104488004DFF03A80DF10E01ADF80C50ADF80E501C
:1044980001F090FFBDF80C10BDF808200091BDF8A0
:1044A8000E10BDF80A3001912C46964D9649082009
:1044B8000AF0DEFCA878012803D101F07FFCAC707B
:1044C80019E1924B5B78012B40F01581AB78002BFA
:1044D80040F011816B6029888D4A09E152F8046F18
:1044E800B07D012840F002810025FAE005F10803BB
:1044F800BDF8080056F82340BDF80A1004F1080377
:104508000CCBFFF73AFF002800F0E980237C013B41
:10451800062B00F29F80DFE803F00429159D1F9DFC
:104528004C006668012304F10805337795E8060016
:10453800636920469847002333772046636995E8E6
:10454800060086E0636893F8252012F1FF3218BF51
:10455800012283F8252077E0636893F82C2012F174
:10456800FF3218BF012283F82C206DE06268137EA9
:104578001568002B6ED16E882F462946184606E02E
:1045880051F804EFDEF804E001338EF81800B34266
:10459800F6D301231376002607E057F8040F00F13D
:1045A8000802436906CA984701366B889E42F4D3CD
:1045B80050E0656820892E68A37B227B0096A0F1D5
:1045C800160189B2FFF721F81420FFF73BFF2B7A79
:1045D800C3B9AF8A29461A461E4609E0886990F889
:1045E80018E00676BEF1010F08BF13460431013208
:1045F800BA42F3D301220BB9AB6924E0053355F86D
:10460800233020E06368DB685A680023908A1546E7
:1046180019461F4609E0AE6996F818E03776BEF1EC
:10462800010F08BF0B46043501318142F3D3411E07
:104638008B4203D1053052F8203003E004D207330F
:1046480052F8233001221A7604F1080206CA636977
:1046580020469847237C013B072B4CD8DFE803F022
:104668000410074B0A0D123A63681B6A34E063684A
:104678009B6A2DE063681B6B2AE063681B6927E06F
:10468800636824E063681A7A7AB9988A1946013807
:1046980000E00132824204D28C69247E0431002C6D
:1046A800F7D0063253F8223011E0DB685A68908A56
:1046B80011460138002300E00133834204D28C699B
:1046C800247E0431002CF7D0063352F82330DB69FE
:1046D800984710E06368DB68204698470BE001358F
:1046E800ADB2338BAB423FF601AF04E001339BB26E
:1046F8008B427FF4F3AE01F055FE0F20FFF7A2FEC8
:1047080005B0F0BDD40C002089A60508840100205E
:1047180018190020034B9A6812B19A68013A9A60F6
:10472800704700BFD40C00202DE9F3470120DFF8C3
:10473800D080DFF8D09001460BF034FF012400252B
:104748004FF4807602274046694600968DF804703B
:104758008DF805408DF806508DF807400BF07AFB70
:104768004046082122460BF0F5FB244BDFF89880E1
:104778001A6844F2A243B2FBF3FA0AF1FF3A204660
:1047880021461FFA8AFA0BF03DFFC8F804A04846F4
:104798004146A8F80050A8F80250A8F8085088F830
:1047A8000A500CF0CBFA7023A8F80C300423A8F8B0
:1047B80010300AF1FF3A6323642203FB0AF3B3FBC8
:1047C800F2F39BB2C8F8143008F10C014846A8F877
:1047D8000E40A8F81870A8F81A50A8F81C60A8F895
:1047E8001E500CF0C9FB484621460CF03CFB4846DD
:1047F80021460CF042FEBDE8FC8700BFD001002036
:104808000000024000000140E40C002083B50E4681
:104818000746154910201C4615460AF029FB1020AA
:1048280012490AF025FB102011490AF021FB10203B
:104838000E490AF01DFB002310200E4901930AF0CF
:1048480017FB334610200C493A460AF011FB10209A
:104858000A492A460AF00CFB1020094922460AF0A8
:1048680007FB019B0133E7E7C3A60508C8A60508AF
:10487800E8A60508F8A6050808A705081DA705085D
:104888002EA7050808B5164B1A6A01321A621A6A69
:10489800012A1A4603D0134840F21D210FE058623E
:1048A800194602E04B6A013B4B62506A0C4B0028E8
:1048B800F8D11A6A012A06D00A484FF40A710A4A3E
:1048C8000A4BFFF7A3FF1A6A013A1A621B6A2BB157
:1048D8000448054A064B40F22A21F2E708BD00BF0A
:1048E800E40C00203FA70508E6A2040869A705080C
:1048F8007AA7050810B5084C0221002220460BF0C3
:104908001EFB44F6FF70FFF7BDFF2046022101227F
:10491800BDE810400BF013BB000402400C4B0D49DE
:104928001A6844F2A2436428B2FBF3F3D4BF20EA26
:10493800E0706420013B9BB24B60013B584364220A
:10494800B0FBF2F080B2486103480C310CF097BA22
:10495800D0010020E40C00200000014010B5134BEA
:1049680093F828202AB11248124A134B4FF4427187
:104978000EE0012283F8282066234FF0C042013B55
:10498800DBB2108033B90A480A4A0C4B40F21231A4
:10499800FFF73CFF1488A4B28442F0D1084B198079
:1049A800024B002283F8282010BD00BFE40C002031
:1049B8003FA70508F0A204088BA7050861A605080B
:1049C8000000026010B5FFF7AFFE6420FFF7A6FFF6
:1049D80021210720FFF7C2FF3220FFF753FF0121F3
:1049E8000020FFF7BBFF3220FFF74CFF23210720F1
:1049F800FFF7B4FF3220FFF745FF00211020FFF733
:104A0800ADFF41F28830FFF73DFF33210720FFF764
:104A1800A5FF3220FFF736FF112046F63001FFF7D9
:104A28009DFF3220FFF72EFF4FF4C0610220FFF7F1
:104A380095FF3220FFF726FF122046F6EB41FFF7DD
:104A48008DFF3220FFF71EFF03204AF6A401FFF76F
:104A580085FF3220FFF716FF00210C20FFF77EFFAD
:104A68003220FFF70FFF0D2040F60C01FFF776FF0D
:104A78003220FFF707FF0E204FF42C51FFF76EFF8F
:104A88003220FFF7FFFEB0211E20FFF767FF32201C
:104A9800FFF7F8FE012042F63F31FFF75FFF3220B3
:104AA800FFF7F0FE05200021FFF758FF3220FFF73F
:104AB800E9FE00210620FFF751FF3220FFF7E2FE52
:104AC80016204EF61C71FFF749FF3220FFF7DAFE79
:104AD800172040F20311FFF741FF3220FFF7D2FE03
:104AE80000210B20FFF73AFF3220FFF7CBFE002111
:104AF8000F20FFF733FF3220FFF7C4FE41200021CB
:104B0800FFF72CFF3220FFF7BDFE42200021FFF700
:104B180025FF3220FFF7B6FE00214820FFF71EFFD1
:104B280040F23F143220FFF7ADFE21464920FFF73F
:104B380015FF3220FFF7A6FE00214A20FFF70EFFDF
:104B48003220FFF79FFE00214B20FFF707FF32209E
:104B5800FFF798FE44204FF46F41FFF7FFFE322025
:104B6800FFF790FE00214520FFF7F8FE3220FFF7FF
:104B780089FE21464620FFF7F1FE3220FFF782FE2C
:104B8800302040F20771FFF7E9FE3220FFF77AFE86
:104B980031204FF40171FFF7E1FE3220FFF772FE7A
:104BA80032204FF40171FFF7D9FE40F2025432204F
:104BB800FFF768FE21463320FFF7D0FE3220FFF7CB
:104BC80061FE342040F20751FFF7C8FE3220FFF79C
:104BD80059FE35204FF40171FFF7C0FE3220FFF770
:104BE80051FE36204FF40171FFF7B8FE3220FFF76F
:104BF80049FE21463720FFF7B1FEA4F500743220A4
:104C0800FFF740FE21463A20FFF7A8FE3220FFF7C3
:104C180039FE2F2041F2BE21FFF7A0FE3220FFF718
:104C280031FE21463B20FFF799FE3220FFF72AFE8E
:104C380000212320FFF792FE3220FFF723FE0021F8
:104C48002420FFF78BFE3220FFF71CFE25204FF4AF
:104C58000041FFF783FE3220FFF714FE00214F20AA
:104C6800FFF77CFE3220FFF70DFE4E200021FFF7F4
:104C780075FE3220BDE8104004E608B5124B93F8E3
:104C880029202AB11148124A124B40F222310FE072
:104C9800012283F82920222166234FF0C042013BDC
:104CA800DBB2118033B90948094A0B4B40F23B315A
:104CB800FFF7ACFD108880B22228F0D1024B002209
:104CC80083F8292008BD00BFE40C00203FA7050891
:104CD800FDA204088BA7050861A6050810B51E4BA0
:104CE800032826D8DFE800F0021A080E1C8841F2D3
:104CF800280246F628000AE01C8841F2080246F617
:104D0800080004E01C8841F2300246F6300049F2FF
:104D180041318C4214BF014611460BE0188846F613
:104D2800200249F24131884214BF11464FF48151A3
:104D380000E000211B8848F68912934205D049F209
:104D48002032934204D1032000E01120FFF706FE31
:104D5800BDE8104091E700BF86010020014B188094
:104D68000A208FE5000002604FF0C043188003F569
:104D780000331A881A88188880B270474FF0C043E9
:104D880022221A8003F5003382B01A8892B2ADF855
:104D980006201B889BB2ADF80630BDF8060080B22D
:104DA80002B07047072040F27311D7E507200021B1
:104DB800D4E582B0044BADF80600BDF8062092B2E7
:104DC8005A8502B0704700BFE40C002082B0044B43
:104DD800ADF80600BDF8062092B25A8002B07047BE
:104DE80086010020014B80B21880704700000260E5
:104DF8004FF0C04380B218807047024B80B21880D1
:104E0800704700BF000002604FF0C04380B21880B6
:104E18007047024B80B21880704700BF00000260E4
:104E280082B0044B0190019ADA62DA6A002AFCD156
:104E380002B07047E40C002070B54FF0C0452A243A
:104E48002C800A4C060AC0B226802080100AD2B2F2
:104E5800208022802B222A800A0A2280C9B21A0ABC
:104E6800DBB221802280238070BD00BF0000026079
:104E780010B50B4614460246FFF7DEFF4FF0C0435D
:104E88002C22A0B21A80BDE8104067E7114B1B889E
:104E980048F68912934210B504460BD049F22032E5
:104EA800934212D1C1F1EF01202089B2FFF756FDDC
:104EB800212006E0C1F1EF014E2089B2FFF74EFD37
:104EC8004F202146BDE8104048E502460B46BDE8A4
:104ED8001040B1E78601002008B5FFF7D7FF0F4B58
:104EE8001B78012B4FF0C0420D4B0FD12E211180A2
:104EF8001A881A881B8892B202F0FC0002F47842E1
:104F080042EAC000C3F3C423184308BD222111801C
:104F18001A881A88188880B208BD00BFEC190020CA
:104F28000000026070B5074D064601242146304650
:104F3800FFF7D2FF0134A4B2C82C25F8020FF5D12F
:104F480070BD00BF0638002010B5084B1B78012B38
:104F5800144602D1BDE810408AE7FFF797FFFFF734
:104F68008CFE2046BDE81040F8E600BFEC19002092
:104F780070B5074D064601242146013435F8022F45
:104F88003046A4B2FFF7E0FFC82CF5D170BD00BFD2
:104F98000638002070B505460E46FFF7C3FF01240A
:104FA8002146013428463246A4B2FFF7CDFFC82C6B
:104FB800F6D170BD2DE9F04104460D461646BDF800
:104FC8001880032B39D8DFE803F00B351927381977
:104FD80080B2294642460137FFF7B6FFBFB200E06C
:104FE8000027B742F3D1BDE8F081E01B80B2294623
:104FF80042460137FFF7A8FFBFB200E00027B742DB
:10500800F3D1BDE8F081E91B89B220464246013759
:10501800FFF79AFFBFB200E00027B742F3D1BDE81F
:10502800F081791989B2204642460137FFF78CFF93
:10503800BFB200E00027B742F3D1BDE8F08170B5F8
:10504800194B1A4A598E92F9004064180025A4B2E7
:105058008AB0AC4208BF0124C62C28BFC6241570EC
:105068000F264FF6FF721E865C865A8519202B463E
:10507800009221460A22FFF79DFF21463046FFF79E
:105088002BFF224603460A4902A811F0B3FC02AAE4
:1050980006A8084911F0AEFC3220D22106AA2B46F8
:1050A80000F002FF0AB070BDE40C0020591A00207D
:1050B800A0A70508A8A705082DE9F341BDF82050C9
:1050C8000C4690461F461A46002306460095FFF7F1
:1050D80071FF611E414430463A46002389B200956B
:1050E800FFF768FF30462146424601230095013EFE
:1050F800FFF760FFBF19B8B2214642460123089561
:1051080002B0BDE8F04155E72DE9F0410D46C5F183
:10511800F008411E5E18C2EB0802C5F1EF039BB20E
:1051280092B2B6B29A422CBF904698469A4234BF81
:1051380011461946864234BF3746074640F23F13A8
:10514800864238BF06469E4228BF1E46174B1B881C
:1051580048F68912B8F1EF0F28BF4FF0EF089342D5
:10516800044610D049F2203293421AD15020FFF75A
:10517800F5FB51204146FFF7F1FB52203946FFF776
:10518800EDFB53200AE041EA082189B24420FFF7E9
:10519800E5FB45203946FFF7E1FB46203146FFF79E
:1051A800DDFB20462946BDE8F0416FE68601002078
:1051B80000200146F0224FF4A073A5E770B580B235
:1051C80002FB03F489B292B29BB2FFF79DFF002065
:1051D800FFF784FD0025064E04E0708D80B2FFF7CE
:1051E800BDFD0135A542F8DBBDE87040E0E700BF32
:1051F800E40C002070B54FF0C0452A242C80094CDF
:10520800060A26802080080A208021802B212980F8
:10521800110A218022801A0A228023802C232B80C5
:1052280070BD00BF0000026070B5114B1B78012BE8
:10523800044607D1002040F23F110246EF23FFF752
:10524800D9FF04E0FFF7B4FF0020FFF747FDF02582
:1052580009E0013E2046B6B2FFF780FD002EF8D1E6
:10526800013DADB215B14FF4A076F2E770BD00BFB5
:10527800EC1900202DE9F04F1C463E4B87B01B78F7
:10528800039183469DF8441010980591012B039BC8
:10529800049092461FFA8BF09AB208D1411E531E11
:1052A8000919534489B29BB2FFF7A4FF09E01FFA1A
:1052B8008AF51146A3B22A46FFF726FF0020FFF71A
:1052C8000DFD0027DDF80C803E4640F23F1CA1464C
:1052D80039E0BBF1000F2EDB65452CDC0398002874
:1052E80029DBB8F1EF0F26DC220702D1002CC8BF5A
:1052F800013621492140002903DA013961F00F0103
:105308000131059A0AB1C1F10F01049830F816204D
:1053180003FA01F10A4012B26AB118494A8D0293A0
:1053280092B2A8B21FFA88F1CDF804C0FFF70CFEBC
:10533800DDF804C0029B013401354C45C9DB013658
:10534800013708F10108574503DA5D4600240123B7
:10535800F3E7084B1B78012B08D1002040F23F11DE
:105368000246EF2307B0BDE8F04F43E707B0BDE8BA
:10537800F04F1DE7EC1900200F000080E40C00201E
:105388002DE9F74F1F463B4BDDF830801B7816465A
:105398009DF83420012B044601920D4680B28AB252
:1053A80008D1411E531EC9199B1989B29BB2FFF738
:1053B80021FF09E01FFA86FE1146BBB27246FFF7CD
:1053C800A3FE0020FFF78AFC4FF0000BDA463DE011
:1053D800002C30DB09EB040340F23F1293422ADC35
:1053E800002D28DB0BEB0503EF2B24DC19F00F0F46
:1053F80004D1B9F1000FC8BF0AF1010A1E4B09EA2E
:105408000303002B03DA013B63F00F030133019A16
:105418000AB1C3F10F03012202FA03F338F81A2084
:1054280013401BB213B1154B588D01E0144A508834
:1054380080B2FFF793FC09F1010901E04FF0000980
:10544800B945C5DB0AF1010A0BF1010BB345F5DBE0
:10545800084B1B78012B08D1002040F23F1102466F
:10546800EF2303B0BDE8F04FC4E603B0BDE8F04F4A
:105478009EE600BFEC1900200F000080E40C00201D
:10548800860100202DE9F0411C4F069C3F789DF8CD
:105498001C60012F02FB03F580B28FB209D1411EB7
:1054A800CB1899B27B1E9A1893B23A46FFF7A2FE20
:1054B80007E092B29BB23946FFF726FE0020FFF7BD
:1054C8000DFC002709E034F8020B1EB1030A43EA79
:1054D800002080B2FFF742FC0137AF42F3DB074BF5
:1054E8001B78012B07D1002040F23F110246EF2321
:1054F800BDE8F0417EE6BDE8F04159E6EC19002030
:105508002DE9F0431F2093B0FFF78EFE4FF478404B
:10551800FFF78AFE4FF6E0754FF4FC60FFF784FE54
:105528002846FFF781FE0020514CFFF77DFE002042
:105538004FF6FF79014664220346A4F82A90CDF875
:105548000090FFF737FD00200A2164220346CDF8BA
:105558000090FFF72FFD00200146642201234FF43D
:10556800784765850095FFF725FD7720EF21C8224C
:1055780000234FF4FC6667850097FFF71BFDBD21EC
:105588003222012340F23F1066850096FFF712FD94
:10559800A02032220023782167850097FFF70AFDB3
:1055A800A0207821322201234FF01F08668500963B
:1055B800FFF700FDA020782132220223A4F82A80D8
:1055C800CDF80080FFF7F6FCA020782132220323D3
:1055D80065850095FFF7EEFC264B2749A3F8028066
:1055E80002AD3C22284611F043F9EB20C3210522E5
:1055F800302300950025A4F82A900195FFF7C0FEF6
:1056080032210A2096220B4667850097FFF754FD42
:1056180032213C2096220B4666850096FFF74CFD0A
:1056280032210B4696226E20A4F82A80CDF80080FD
:10563800FFF742FDFFF7BAFBFFF7B4FB3220FFF795
:105648006DF92846FFF76AF96420FFF767F90B4BF5
:1056580003F110028DE8240028465A681B68294681
:10566800FFF710FF1195119B01331193FBE700BF62
:10567800E40C00208601002012A30408D0C701080A
:105688002DE9F14FFFF750F84FF0C0456420FFF7C0
:1056980045F90127FFF72EF94FF028096D48FFF764
:1056A800F1F82F800520A5F8009003F0D3F9CF2357
:1056B8002B80694B002683221E801A8030221A8094
:1056C800ED222A804FF064080322A3F800801A8094
:1056D80012221A8081221A80E8222A8085221A80C2
:1056E80079221F801A80CB222A8039221A804FF013
:1056F800340C02242C21F72219801E80A3F800C044
:105708001C802A8020221A80EA222A80C0221E8039
:10571800C1211E802A8026221A8029801121198001
:10572800C5212980352119803E211980C72129806A
:10573800BE211980362129803A205521A3F80090EE
:1057480028801980B12129804FF0100BF2211E808A
:10575800A3F800B02980082119802A80E0221F8040
:105768004FF01F092A801A22A3F800904FF0180A58
:105778001A800F210A22A3F800A01A801980062196
:105788001980452119808721198032211980072124
:105798001A804FF0E10E19801C80052419801C80A6
:1057A8001E80A5F800E04FF0250E1E80A3F800E04B
:1057B8004FF0270EA3F800E01C80A3F800B04FF0CC
:1057C800090BA3F800B04FF0780B1880A3F800B0CD
:1057D8004FF04D0BA3F800B01C800D24A3F800A0D7
:1057E8001C8038241C8018802A20A3F80090EF24FD
:1057F80028802B201E801E801E801C8028803F2031
:105808001E801E801F801880B720A5F800C0288041
:105818001980B62129801A8082221A801122A3F8C1
:1058280000E040461E8029272A8003F013F94046ED
:105838002F8003F00FF90948FFF724F82C232F8055
:1058480030462B8040F23F113246234601B0BDE876
:10585800F04FCFE4400D03000000026040420F000B
:105868002DE9F041022098B0012100240AF09AFEA7
:10587800012502268048169616A98DF85D408DF8F8
:105888005E408DF85F408DF85C500AF0E3FA18200E
:1058980029460AF087FE284629460AF09BFE21463B
:1058A8000C2276480AF056FB0C22744829460AF066
:1058B80051FB04210C2271480AF04CFB05210C22F3
:1058C8006E480AF047FB07210C226C480AF042FB9D
:1058D80008210C2269480AF03DFB09210C2267487F
:1058E8000AF038FB0A2165480C220AF033FB0B2129
:1058F80062480C220AF02EFB0E210C225F480AF0A7
:1059080029FB0F210C225D480AF024FB07210C22F9
:105918005B480AF01FFB08210C2259480AF01AFBC1
:1059280009210C2256480AF015FB0A210C2254487A
:105938000AF010FB0B210C2251480AF00BFB0C213A
:105948000A464F480AF006FB0D210C224C480AF083
:1059580001FB0E210C224A480AF0FCFA0C224848A6
:105968000F210AF0F7FA4CF6B3734448169316A9B8
:105978008DF85C608DF85E408DF85F408DF85D5065
:105988000AF068FA16A94FF680733D4816938DF809
:105998005C608DF85E408DF85F408DF85D500AF0D0
:1059A80059FA40F6B830FEF76DFFFEF7A3FF40F650
:1059B800B830FEF767FF0F2311934FF48053102779
:1059C8000DF13C08099368464FF400231094129493
:1059D80014941594009401940294039704940694E3
:1059E800079408940A9405940B940C93CDF834808A
:1059F8000F95139509F0A7FF0523684611930F9695
:105A08001094129414941594CDF83880139509F0D5
:105A18009AFF294620460AF016F840F6B830FEF7F5
:105A280031FF2046FFF7A0F904461649164E3846BE
:105A3800224609F01DFA41F289239C4248F689184A
:105A4800124F01D044450ED1FEF7BCFF00233B7036
:105A5800A6F8008010200E4948F6891241F28923E1
:105A680009F006FA05E0FFF70BFE49F241333D70F5
:105A7800338018B0BDE8F08100040240000C0240F9
:105A880000100240ADA7050886010020EC1900208F
:105A9800C4A705084FF0C04336221A8003F5003327
:105AA800012814BF682048201880704770B5244B1F
:105AB80001228CB01A7000240AE0A9B21F223046D5
:105AC8000135FFF741FA642DF7D10134642C02D077
:105AD8000025A6B2F1E73220014602460346FFF749
:105AE800ABF94FF0C0432E221A8003F50033002093
:105AF8001A881C881D88A4B200F09CF8ADB2002357
:105B0800224600930F492B4603A810F073FF002389
:105B18000A20C82103AA00F0C7F904F0FC0204F423
:105B2800784444EAC20242EAD522074903A810F0A1
:105B380061FF0A20DC2103AA002300F0B5F9FEE783
:105B4800EC19002003A805081BA805082DE9F04F4B
:105B580040F23F19484534BF04464C46EF2B34BF4A
:105B680098464FF0EF084A4538BF9146EF2934BFB1
:105B78000D46EF25C4EB090AC5EB080785B0BAF155
:105B8800000FB8BFCAF1000A002FB8BF7F424FF616
:105B9800FF734C452CBF1A4601221FFA8AFA454565
:105BA80038BF0123BFB202930FFA8AF63BB29E4276
:105BB800BDF838B0019202DDC6F34F0607E00226B1
:105BC80093FBF6F67642B6B201E01E4603E00FFA02
:105BD8008AF35B420393144A1378022B2046294622
:105BE8005A4602D1FDF7FDFC01E0FFF7ADF94C453F
:105BF80001D1454514D0039A33B2934205DD019A89
:105C0800F31BA4189BB2A4B200E0334636B23AB2F2
:105C18009642DADA029A5344AD189BB2ADB2D4E791
:105C280005B0BDE8F08F00BF242C00200048704765
:105C3800F419002082B0064BADF80600BDF8062026
:105C480092B21A80188880B202B0FFF7B2B800BFCB
:105C5800F0190020014B188880B27047F019002015
:105C680082B0064BADF80600BDF8062092B21A8045
:105C7800188880B202B0FFF7A9B800BFF219002057
:105C8800014B188880B27047F2190020FFF7CCBA90
:105C9800FFF73ABA10B5BDF808400294BDE81040C5
:105CA800FFF788B910B5BDF808400294BDE8104068
:105CB800FFF702BAFFF782BA2DE9F04F4FEA420820
:105CC80000253D4C85B082468B46C8F1030817462F
:105CD8002E461FFA87F909EB0B0C228805EB0A03FD
:105CE8001FFA8CFC9BB26146184692B2CDF804C0EC
:105CF8000293FFF729F9C9EB0B0292B20392029BB8
:105D080022880399184692B2FFF71EF9DDF804C0FD
:105D18002288C5EB0A039BB26146184692B20293E9
:105D2800FFF712F9029B22880399184692B2FFF7EF
:105D38000BF905EB0B0292B2039209EB0A032288D6
:105D480003999BB2184692B20293FFF7FDF8029BA3
:105D58002288C5EB0B0C1FFA8CFC1846614692B2E0
:105D6800CDF804C0C9EB0A09FFF7EEF822880399B9
:105D78001FFA89F992B24846FFF7E6F82288DDF85B
:105D880004C092B248466146FFF7DEF8B8F1000F4A
:105D980004DA08EB860808F1060805E0F31B08F1A9
:105DA8000A0808EB8308013F01360135BE42ADB24F
:105DB8008FD905B0BDE8F08FF019002008B9FEF7BB
:105DC800F5BF012801D1FEF7EDBF704770470020ED
:105DD8000146F0224FF4A073FFF796B9704708B553
:105DE80005280CD8DFE800F0121403050709094854
:105DF80008BD094808BD094808BD094808BD094843
:105E0800094A0A4B40F24111FEF700FD084808BD57
:105E1800084808BD74010020640100205C010020CE
:105E28005401002026A805084EA3040861A6050809
:105E38007C0100206C01002010B50446FFF7CFFF5D
:105E4800014B18601C7110BD8C010020014B1879A2
:105E5800704700BF8C01002008B5FFF7C0FF80889D
:105E680008BD08B5FFF7BBFFC08808BDF7B51F46DA
:105E78000B4B0C4E1D681446EA882B68203C544393
:105E8800A4B2AE1B03EB440418BF0126AB888DE80F
:105E9800500017B1FFF7EEF901E0FFF771FAFEBD08
:105EA8008C0100207C0100202DE9F0410F46984626
:105EB80015460446084E08E0204643463946FFF793
:105EC800D5FF33689B88E418A4B215F8012B002A83
:105ED800F2D1BDE8F08100BF8C01002010B5044666
:105EE80008462146BDE81040DEE7094B70B5044678
:105EF80018790E461546FFF7B4FFC6F1F001091AE6
:105F080089B220462A460023BDE87040CCE700BF8E
:105F18008C010020704700BF044B1A680AB9044A74
:105F28001A601A681018186010467047180D00207B
:105F3800A43C00204FF0FF30704708B50248034AE0
:105F4800034B3721FEF762FC45A8050864A3040843
:105F580061A605080120704710B504460A480221C9
:105F68000AF0A6FD0028F9D0074821460AF069FD85
:105F7800054801210AF09CFD0028F9D00248BDE837
:105F880010400AF05BBD00BF0038004010B519484A
:105F980002210AF08DFD0028F9D0164800210AF0E8
:105FA80050FD144801210AF083FD0028F9D011485A
:105FB8000AF044FD0402A4B2002301E001339BB2BD
:105FC800002BFBD00B4802210AF072FD0028F9D003
:105FD800084800210AF035FD064801210AF068FD4D
:105FE8000028F9D003480AF029FD2043C0F3CB006C
:105FF80010BD00BF003800402DE9F0478AB00AAF55
:106008000A2001210AF0CEFA4FF4604347F8143D04
:10601800474EDFF824A1012400254FF0020830463E
:1060280039468DF81A508DF818808DF819808DF83A
:106038001B4009F00FFF30460D21052209F08AFFA9
:1060480030460E21052209F085FF052230460F2132
:1060580009F080FF21464FF480400AF0C7FA504605
:106068000AF0A2FB4FF48273ADF802304FF40073CC
:10607800ADF80A303823ADF80C305046072369468E
:10608800ADF81030ADF80050ADF80450ADF806503A
:10609800ADF80850ADF80E500AF0B8FB504621464E
:1060A8000AF04FFCA9468DF81A5030464FF4805537
:1060B800394605958DF818408DF819808DF81B40E4
:1060C80009F0C8FE3046294609F035FF4025394613
:1060D80018488DF818908DF819808DF81A908DF859
:1060E8001B40059509F0B6FE21464FF480400AF0A2
:1060F80089FA062103200AF013FD0C2307A88DF85E
:10610800213007958DF820908DF8224009F096FBF4
:1061180017238DF8243009A80F238DF825308DF822
:1061280026308DF8274002F0B3FE0AB0BDE8F087AC
:1061380000040240000C024000380040014B18786F
:10614800704700BF1C0D0020024B5A889B880280B4
:106158000B8070471C0D0020014B00221A707047FD
:106168001C0D0020F0B593B068460021482210F0BD
:10617800C1FB6D46002464484FF4805109F0DDFEF0
:10618800002301E001339BB2002BFBD09020FFF7E6
:10619800E3FE002301E001339BB2002BFBD0FFF7A5
:1061A800F5FE4FF480510746574809F0C4FE002316
:1061B80001E001339BB2002BFBD053484FF48051D0
:1061C80009F0BBFE002301E001339BB2002BFBD09A
:1061D800D020FFF7C1FE002301E001339BB2002B62
:1061E800FBD0FFF7D3FE4FF480510646464809F02E
:1061F800A2FE45F8047B01342E6244484021E4B2F3
:1062080009F087FE10B9092CB5D101E0092C78D125
:106218009DE80C00D218029B03980699D218049B9B
:10622800C018059BC018079BCB180899032490FB3E
:10623800F4F092FBF4F25B1893FBF4F3151AC11A0D
:106248009C1A002DB8BF6D420029B8BF4942002CE6
:10625800B8BF6442502D03DD502909DD502C50DCB5
:106268008D4205DAAC424FF0020405DB111806E056
:106278008C424FF0020401DAD11800E0C1180A9BE1
:10628800099A0C980F9DD2180B9BD2180D9BC01819
:106298000E9BC018109BEB18119D91FBF4F1032481
:1062A80092FBF4F290FBF4F05B1993FBF4F3161AEB
:1062B800C41A9D1A002EB8BF7642002CB8BF64429B
:1062C800002DB8BF6D42502E89B203DD502C09DD78
:1062D800502D16DCA64205DAB5424FF0020405DB64
:1062E800131806E0A5424FF0020401DAD31800E0C3
:1062F800C318074A93FBF4F39BB2938001235180A0
:10630800137013B0F0BD00BF00040240000C02403F
:106318001C0D002000000000FFF710BFF7B5054670
:106328000C4601A80DF10601FFF70EFF1B4BBDF847
:106338000660BDF8040093E80600724301FB0022E2
:1063480099685218164992FBF1F207EE102AF8EEF6
:10635800C77A40F23F17FCEEE77A17EE902A92B21E
:10636800B2F5207F28BF3A462A801D69DA685B6942
:106378006E4302FB0060C01890FBF1F107EE101AA3
:10638800F8EEC77AFCEEE77A17EE903A9BB2B3F5CF
:10639800F07F28BFEF232380FEBD00BF240D00201F
:1063A80040420F00FFF7D8BE014B187E704700BF70
:1063B800240D0020FFF7C8BE042808B505D90748F2
:1063C800074A084B7D21FEF721FA054B03EB8000B5
:1063D800038B0B80438B138008BD00BF66A805089C
:1063E8006AA3040884A8050808B5082001F08AF9FA
:1063F80042F69643C31A584240EB030008BD10B555
:106408000A2001F0A7F90C4C20600E2001F0A2F937
:106418006060122001F09EF9A060162001F09AF940
:10642800E0601A2001F096F920611E2001F092F92F
:1064380001236061237610BD240D002010B5FFF7FD
:10644800DBFD01F03DFA044601F046FA0749034630
:106458002246202008F00CFDFFF7C6FF28B101F006
:1064680049FA10B9BDE81040C9E710BDC0A8050831
:1064780010B5104C0A20216801F053F961680E200C
:1064880001F04FF9A168122001F04BF9E1681620DC
:1064980001F047F921691A2001F043F961691E20CA
:1064A80001F03FF9082042F69641BDE8104001F09E
:1064B8001BB900BF240D00202DE9F04F0346A7B0FB
:1064C800B0F800C01C898688DF885D89CDF810C0C7
:1064D800B249B0F802C0B3F80C90B3F80E80CDF80A
:1064E80024C00FFA84FB30B201220FFA87FE0BEBAF
:1064F800000C0A7629B20FFA89FACDF888C001EBA8
:106508000E0C0FFA88F2CDF890C00AEB0B0CCDF800
:1065180030C002EB010CCDF858C0B3F810C05B8A4C
:10652800CDF800C00FFA8CFC06910CEB00010A9123
:1065380002930CEB0A011BB2239103EB0E010E919F
:1065480099182591049900FA81F058445044604400
:10655800DDF824C006990EFA8CFEDDF810C01FFA8B
:1065680080FB1CFB0CF08E4416FB0600964414FBC3
:106578000400009A19FB09009E4412FB02001FFA4E
:106588008EFA0BF09FFBDDF824C0029ACDE91201C8
:106598001CFB0CF017FB070015FB050018FB080097
:1065A80012FB02000BF08EFBDDF824C0029ACDE945
:1065B800140104991CFB01F317FB063615FB04664E
:1065C800009B18FB096612FB03600BF07BFBDDE9FF
:1065D8001423CDE90001DDE912010BF0E9FB0446C3
:1065E8000D46DDE9000102460B460BF0E1FB0246D1
:1065F8000B46204629460BF027FACDE918015846E4
:106608000BF070FBCDE91001DDE91023DDE9000195
:106618000BF0CEFBCDE9060150460BF063FB80463C
:1066280089464246DDE912014B460BF0C1FBDDE924
:106638001023CDE91C01DDE914010BF0B9FB0022A0
:1066480006460F46564BDDE918010BF0B1FB4246F2
:1066580004460D464B46DDE906010BF0A9FB024650
:106668000B460BF0F3F902460B46204629460BF081
:10667800EDF9424604460D464B46DDE91C010BF098
:1066880097FB02460B46204629460BF0DDF9DDE96B
:10669800102304460D46304639460BF089FB024666
:1066A8000B46204629460BF0CFF9DDF828C0CDE986
:1066B80002014FEA8C10DDF830C000EB0C20DDF849
:1066C80010C0A0241CFB04000BF0FCFADDF838C055
:1066D800CDE90A014FEA8C10DDF858C000EB0C2018
:1066E800DDF824C01CFB04000BF0ECFACDE90C012A
:1066F80050460BF0E7FADDE91023CDE91601DDE994
:106708000C010BF055FB4246CDE91E014B46DDE975
:106718000A010BF04DFB4246CDE920014B46DDE96D
:1067280000010BF045FB32463B460BF08DF9CDE9F5
:106738000E0158460BF0C6FADDE91C23CDE91A0113
:10674800DDE906010BF080F9DDF88CC0C024CDE945
:10675800060104FB0CF0DDF888C0302505FB0C00B1
:10676800DDF810C078261CFB06000BF0ABFADDF84C
:1067780094C0824604FB0CF0DDF890C005FB0C00C9
:10678800DDF824C01CFB06008B460BF09BFADDE904
:10679800102306460F460BF00BFB03E0240D0020E8
:1067A800000014404246CDE904014B465046594684
:1067B8000BF0FEFADDE9142380468946DDE90A017B
:1067C8000BF0F6FADDE9002304460D46DDE90C017D
:1067D8000BF0EEFA02460B46204629460BF034F938
:1067E8000022A14B0BF0E4FADDE9202304460D4614
:1067F800DDE91E010BF028F902460B46DDE916011A
:106808000BF0D6FA02460B46204629460BF01EF935
:10681800002204460D46954BDDE90E010BF0C8FA3F
:1068280002460B46204629460BF010F9DDE9022303
:106838000BF0E8FB88A3D3E900230BF0B9FA0BF0BF
:1068480051FD8B490860DDE91223DDE90C010BF0ED
:10685800AFFADDE9002304460D46DDE90A010BF035
:10686800A7FA02460B46204629460BF0EDF800220F
:106878007D4B0BF09DFADDE91E2304460D46DDE94C
:1068880020010BF0E1F802460B46DDE91A010BF096
:106898008FFA02460B46204629460BF0D7F800220D
:1068A80004460D46714BDDE906010BF081FA0246FC
:1068B8000B46204629460BF0C9F8DDE902230BF008
:1068C800A1FB65A3D3E900230BF072FA0BF00AFDD4
:1068D800674A5060DDE90E23DDE90A010BF068FA2A
:1068E800DDE9062304460D46DDE90C010BF060FAEC
:1068F80002460B46204629460BF0A8F8002204461B
:106908000D465A4BDDE918010BF052FA02460B46C8
:10691800204629460BF09AF8DDE902230BF072FBBA
:106928004DA3D3E900230BF043FA0BF0DBFC504BEB
:1069380059469860DDE9142350460BF039FADDE931
:10694800002304460D46304639460BF031FA02461C
:106958000B46204629460BF077F80022424B0BF0F5
:1069680027FA424604460D464B46DDE904010BF082
:106978006BF802460B46DDE916010BF019FA0246E0
:106988000B46204629460BF061F835A3D3E90023CE
:1069980004460D46DDE90E010BF00AFA02460B46E5
:1069A800204629460BF052F8DDE902230BF02AFBBA
:1069B80029A3D3E900230BF0FBF90BF093FCDFF8D4
:1069C800B0C0DDE91223CCF80C00394630460BF094
:1069D800EFF9DDE9002304460D46504659460BF011
:1069E800E7F902460B46204629460BF02DF800220F
:1069F8001D4B0BF0DDF9DDE9042304460D46404646
:106A080049460BF021F802460B46DDE91A010BF066
:106A1800CFF902460B46204629460BF017F810A37B
:106A2800D3E9002304460D46DDE906010BF0C0F961
:106A380002460B46204629460BF008F8DDE90223FA
:106A48000BF0E0FA04A3D3E900230BF0B1F90BF043
:106A580049FC074908610DE00000000080842E41D0
:106A68000000000000C0824000001440000089407F
:106A7800240D0020DDE90E23504659460BF098F905
:106A8800DDE9062304460D46304639460BF090F9F9
:106A980002460B46204629460AF0D8FF11A3D3E93F
:106AA800002304460D46DDE918010BF081F9024682
:106AB8000B46204629460AF0C9FFDDE902230BF000
:106AC800A1FA0AA3D3E900230BF072F90BF00AFC30
:106AD800034A506127B0BDE8F04FC9E4AFF3008026
:106AE800240D00200000000000C0824000000000CB
:106AF80080842E41AFF30080064A074B1A60074A8C
:106B0800074B1A60074B42F210721A60064B642258
:106B18001A60704740420F001826002080C3C90140
:106B2800302C00200C2C0020C8250020012810B58E
:106B380003D041D3022838D123E0204B204C1B78C6
:106B4800012B204B0ED11968C82000F0EAFD2168FE
:106B5800CC2000F0E6FD1C4BD020196800F0E1FDC8
:106B6800D4201EE01968D82000F0DBFD2168DC2065
:106B780000F0D7FD144BE020196800F0D2FDE420A6
:106B88000FE0104BE820196800F0CBFD0C4BEC200F
:106B9800196800F0C6FD0C4BF020196800F0C1FD23
:106BA800F4200A4B196800F0BCFD04F037FE18B950
:106BB800BDE8104004F043BE10BD00BFF40D002036
:106BC800302C0020182600200C2C0020C82500207E
:106BD80010B5224B1B78012B02D0022B3DD128E0A7
:106BE8001F4B204C1B78012B0FD1C82000F0B2FDA1
:106BF8002060CC2000F0AEFD1B4B1860D02000F0C8
:106C0800A9FD1A4B1860D4200EE0D82000F0A2FD90
:106C18002060DC2000F09EFD134B1860E02000F09F
:106C280099FD124B1860E42000F094FD104B186099
:106C380010BDE82000F08EFD0A4B1860EC2000F033
:106C480089FD094B1860F02000F084FD074B18609F
:106C5800F42000F07FFD064B186010BDB501002040
:106C6800F40D002018260020302C00200C2C0020C9
:106C7800C825002008B504F0D1FD10B1BDE80840D2
:106C8800A6E7BDE8084037E7064B07495960C02129
:106C9800002219721E211A70D9601A745A611A7664
:106CA800DA617047201A002040787D0110B5032171
:106CB800FF22C02001F0D4FB1F4C1021802220604D
:106CC800C02001F0CDFB112180222060C02001F0FE
:106CD800C7FB122180222060C02001F0C1FB1321D4
:106CE80080222060C02001F0BBFB1421802220609C
:106CF800C02001F0B5FB152180222060C02001F0E2
:106D0800AFFB802220601621C02001F0A9FB206083
:106D1800C0201721802201F0A3FB80222060B72128
:106D2800C02001F09DFB054B00221A745A611A76A7
:106D3800DA6101221A7010BDF0250020201A002007
:106D480038B5C0200321FF2201F08AFB0B4D002437
:106D58002B19615D5A78C020023401F081FBC82CE0
:106D6800F6D1B121AC22C02001F07AFBC02003216A
:106D7800002201F075FB002038BD00BF96A304086F
:106D88002DE9F34706460F4692461D461AB90C1FD1
:106D9800E401914635E005EE902A06EE903AB8EE09
:106DA800657AF8EE667AFC01C7EE277AA4F50074D6
:106DB8009FED5C7A67EE877A17EE900A0AF0A4FFD7
:106DC80041EC100B0DF0B4F859EC108B49464046D5
:106DD8000BF0B0FA24184FEACA100AF073FFCDE995
:106DE800000128460AF06EFF4B4642460AF0E0FFD3
:106DF80002460B46DDE900010AF026FE0BF09AFA7E
:106E08008146002E14BF4FF022084FF01A08C5F330
:106E180007224146C02001F023FB08F10101EAB234
:106E2800C02001F01DFBC4F3014208F10201C0209B
:106E380001F016FBC4F3072208F10301C02001F09A
:106E48000FFBE2B208F10401C02001F009FBC9F30D
:106E5800034305F4702243EA123208F10501C02009
:106E680001F0FEFA08F10601C9F30722C02001F07B
:106E7800F7FA08F107015FFA89F2C02001F0F0FA89
:106E8800C020B121A02201F0EBFA07EE107A264CBF
:106E9800F8EEC77A0EBBD4ED015A06EE90AAB8EE0A
:106EA800657A05EE905AB8EE666AF8EE656A0123CF
:106EB800C6EE266A237477EEA67A67EE277A17EE6F
:106EC800900A0AF021FF41EC100B0DF031F851EC5B
:106ED800100B0BF02FFA606120E005EE90AAD4EDBC
:106EE800016AB8EE656A05EE905AB8EE667AF8EE71
:106EF800656A0123C6EE266A237677EEA67A67EEE0
:106F0800277A17EE900A0AF0FFFE41EC100B0DF0FD
:106F18000FF851EC100B0BF00DFAE0610020BDE802
:106F2800FC8700BF00000043201A00200022012334
:106F380026E7012838B50D4604D002280CBF3C24AA
:106F48002C2400E034242146C02001F003FB05F086
:106F5800070200F00F0040EA02122146C020BDE8F7
:106F6800384001F07DBA2DE9F3470A9C1D460746D3
:106F78008A461646524B01E06D0864089C42FBD8CD
:106F88002DB906F10076043EF601A94634E006EE76
:106F9800905AB8EE667A06EE904AF8EE667AF601EE
:106FA800C7EE277AA6F500769FED467A67EE877AD0
:106FB80017EE900A0AF0A8FE41EC100B0CF0B8FF8F
:106FC80059EC108B494640460BF0B4F93618E801E5
:106FD8000AF078FECDE9000120460AF073FE4B4620
:106FE80042460AF0E5FE02460B46DDE900010AF0DA
:106FF8002BFD0BF09FF98146022F9BBF324BDB190B
:107008004FF0000893F8C880C4F307224146C02017
:1070180001F026FA08F10101E2B2C9B2C02001F07C
:107028001FFA08F10201C9B2C6F30142C02001F0FB
:1070380017FA08F10301C9B2C6F30722C02001F00C
:107048000FFA08F10401C9B2F2B2C02001F008FA3F
:1070580004F47024C9F3034308F1050143EA143228
:10706800C9B2C02001F0FCF908F10601C9B2C9F3A0
:107078000722C02008F1070801F0F2F95FFA89F247
:107088005FFA88F1C02001F0EBF9BAF1010F0CBFEB
:107098002F220F220DB942F04002012F06D002D351
:1070A800022F0AD105E0C020102104E0C0201121E0
:1070B80001E0C020122101F0D3F90020BDE8FC87CF
:1070C800FFFF0F000000004396A3040807B5012343
:1070D80000930023FFF747FF0EBD00280CBFFF22D7
:1070E800002208B5C020032101F0BAF9002008BD2C
:1070F80008B5C020B121AC2201F0B2F9002008BDCA
:1071080008B50420012109F04DFA4FF480700121DF
:10711800BDE8084009F076BA07B5022300930323B7
:107128008DF804300348002369468DF8073008F0CD
:1071380091FE0EBD0008024030B5124D8BB0002400
:1071480006A8069407940894099408F051F8009446
:107158008DF804408DF80540029403940494284661
:10716800012469468DF8144008F013F828460B21CD
:107178002246062308F088F82846214608F052F8E7
:107188000BB030BD0020014010B50021044601229B
:10719800302001F065F9C0B9012001F05BFC002C3A
:1071A800B8BF4034E4B210212246302001F058F92B
:1071B800012001F04FFC30201121224601F050F946
:1071C8000120BDE8104001F045BC10BD10B50021FC
:1071D80004460122302001F043F9C0B9012001F032
:1071E80039FC002CB8BF4034E4B2122122463020CA
:1071F80001F036F9012001F02DFC30201321224640
:1072080001F02EF90120BDE8104001F023BC10BDAB
:1072180038B5012205460C463020002101F020F93E
:10722800F0B9012001F016FC25EAE5725F2AA8BF33
:107238005F223B21D2B2302001F012F9012001F087
:1072480009FC24EAE4725F2AA8BF5F22D2B2302088
:107258003C2101F005F90120BDE8384001F0FABBF6
:1072680038BD302810B504460ADC10F17F0F02DB68
:10727800002802DB05E06FF07E0404F5807400E06E
:107288003024002130200A4601F0EAF8A8B901208C
:10729800E4B201F0DFFB41212246302001F0E0F8A2
:1072A800012001F0D7FB30204221224601F0D8F816
:1072B8000120BDE8104001F0CDBB10BD282810B555
:1072C800044609DC10F1180F02DB002802DB04E099
:1072D8006FF017047F3400E02824002130200A468C
:1072E80001F0BEF8A8B90120E4B201F0B3FB5321C4
:1072F8002246302001F0B4F8012001F0ABFB302029
:107308005421224601F0ACF80120BDE8104001F0FC
:10731800A1BB10BD08B530200021012201F0A0F862
:1073280060B9012001F096FB30203321402201F0A2
:1073380097F80120BDE8084001F08CBB08BD10B5E6
:1073480030200021012201F08BF8044660B90120A9
:1073580001F080FB30203321224601F081F8012022
:10736800BDE8104001F076BB10BD10B530200021FB
:10737800012201F075F80446A0B9012001F06AFB6A
:1073880034212246302001F06BF8012001F062FB25
:1073980030203721224601F063F80120BDE8104073
:1073A80001F058BB10BD4020EEE640200EE708B5BE
:1073B80000210122302001F053F8012001F04AFB9E
:1073C80030203421024601F04BF8012001F042FB45
:1073D80030203721024601F043F80120BDE808407B
:1073E80001F038BB08B500210122302001F038F83F
:1073F800012001F02FFB302034210C2201F030F85D
:107408000120BDE8084001F025BB00000000000095
:107418002DE9F04F984B994A1968994B002914BFE8
:1074280091469946974B2DED048BC3F80090964BE7
:107438000025002287B01A80AA46AB46A8465AE023
:10744800A2004046CDF804C002920AF05DFC07464F
:10745800584601F100460AF057FC02460B463846EA
:1074680031460AF0F1FA39F9243007EE103AF8EE0D
:10747800C77A064617EE900A0F460AF045FC024600
:107488000B46304639460AF0E1FA0AF073FF074620
:1074980050460AF039FC0446284601F100460AF035
:1074A80033FCCDE90401DDE90423204631460AF026
:1074B800CBFA029A09EB02030446B3F9023007EE4D
:1074C800103AF8EEC77A0D4617EE900A0AF01CFC3F
:1074D80002460B46204629460AF0B8FA0AF04AFF47
:1074E800DDF804C0684A0CF1010CC3465546A2F801
:1074F80000C08246B846644BB3F800C00FFA8CF45B
:10750800B32C9DDD58460AF0FFFBCDE90201404649
:107518000AF0FAFB002206460F465C4BDDE9020141
:107528000AF046FC02460B46304639460AF08EFA07
:107538000022574B0AF066FD0AF01CFF4CA3D3E962
:10754800002309EE900ADDE902010AF031FC00226D
:107558004F4B0AF057FD0AF00DFF09EE100A2846B6
:107568000AF0D2FB044650460D460AF0CDFB002235
:1075780006460F4620462946444B0AF019FC0246A7
:107588000B46304639460AF061FA0022404B0AF0B1
:1075980039FD0AF0EFFE36A3D3E9002308EE900A7E
:1075A800294620460AF004FC0022394B0AF02AFD3D
:1075B8000AF0E0FE08EE100A69EE287A58EE297AF9
:1075C80017EE900A0AF0A0FB68EE097A48EEA97A4D
:1075D800044617EE900A0D460AF096FB45EC104B50
:1075E80041EC110B0CF0A8FD51EC100B0AF0C2FE97
:1075F80028EE088A08EEA88A07EE100A254B264CC2
:10760800F1EE477AC3ED007A18EE100A0AF07CFB17
:1076180041EC100B0CF09EFE29EE099A51EC100B70
:1076280009EEA99A0AF0A6FE206019EE100A0AF0DF
:107638006BFB41EC100B0CF08DFE51EC100B0AF0BB
:1076480099FED4ED007A07EE100A87EE877A134B7D
:107658001860134BFDEEE77A83ED007A114BC3ED0A
:10766800007A07B0BDEC048BBDE8F08FAFF3008063
:10767800912B50E67AB6EB3F481A0020CA22002028
:107688002A1D0020441A0020501A00200000E03F64
:1076980000005940342C00204C2C0020402C0020A5
:1076A8003C2C00204C1A002010B5084C204608F04D
:1076B8001EF8074B1860FFF7ABFE064B0649012280
:1076C80020461A80BDE8104008F092B810600240C9
:1076D800481A0020400D002020800010014B186837
:1076E800704700BF4C1A002038B505460C460135D6
:1076F800C1F3072101F0BCF9A8B2E1B201F0B8F971
:1077080000B238BD38B5044600F0ECFF0134054638
:10771800A0B200F0E7FFEDB2C0B240EA052000B227
:1077280038BD37B50B0E8DF804300B0C8DF80530CD
:107738000B0A8DF806308DF80710002400E0284663
:1077480001AB451CE15C013401F092F9042CADB2A7
:10775800F5D13EBD37B5002400E02846451C00F0B1
:10776800C1FF01ABADB2E0540134042CF5D19DF852
:1077780005009DF80430000440EA03609DF80730D6
:1077880018439DF8063040EA03203EBD37B5002374
:107798000193002400E02846451C00F0A3FF01AB3C
:1077A800ADB2E0540134042CF5D19DED010A3EBD83
:1077B8007047000038B50446642001F04BF925787D
:1077C8006068AD00EDB2257008F0A9FB237A40FA95
:1077D80003F000F003000543104B257005F00F057A
:1077E8005A5D6378D218D2B2D3B20132D2B2022A29
:1077F800637001D80022A2705BB2012B03DD012364
:10780800A3700023637094F90130013303DAFF2376
:10781800A3700023637094F9020038BD62A40408C1
:10782800F7B504200121234F08F0BCFE02AD012169
:107838004FF48040012408F0E5FE00264FF4B073B1
:107848003846694645F8083D8DF804608DF80740CC
:1078580008F000FB1020214608F0A4FE78236946B2
:10786800154800938DF804608DF8074008F0F2FA87
:107878000420214608F096FE21464FF4804008F087
:10788800C1FE1C233846694600938DF804608DF8C4
:10789800074008F0DFFA0220214608F083FEB023F3
:1078A80006488DF8046069468DF80740009308F093
:1078B800D1FAFEBD00080240001002400004024058
:1078C800802108B5034808F024FBD0F1010038BF37
:1078D800002008BD0004024008B54FF48071044838
:1078E80008F017FBD0F1010038BF002008BD00BF29
:1078F8000008024008B5FFF7E3FF08B1FFF7ECFF07
:10790800C0B208BD70B500283AD01E4B1A7880184E
:107918001D4AC0B292F90020187040B282421B4A38
:1079280002DD11780139197093F9001092F90020DD
:1079380091FBF2F402FB14141549E4B21C700A8896
:10794800144B1A80144B154A18881080144A92F95F
:10795800000064B2013094FBF0F200FB1240114CBD
:107968002688114C258800FB065008800F49088896
:107978000F49098802FB00121A800E4B01221A7067
:1079880070BD00BFDE39002009360020E535002033
:10799800143A00202A360020DC390020DC37002089
:1079A800163A002038370020783A0020A43A002000
:1079B800BA370020E4350020F0B5264A264C0023CB
:1079C8001370264A25681678254A12680FE0D45C99
:1079D8002F197F7817F0040F07D0302C02D12023FD
:1079E800135431E01B4A137003E00133DBB29E42AB
:1079F800EDDA184B1B788342194B16D9A9B11A68CE
:107A0800164C3121115430210BE01A681518125CFC
:107A18002E2A19D0303AD2B2092A88BF29700130EB
:107A2800C0B222788242F0DA0EE01B681A5C79B1A3
:107A38002E2A0DD05118C9B2392903D82F2998BF39
:107A4800302100E039211954BDE8F040FCF7B6BCFC
:107A5800F0BD00BF440D002024030020983B002007
:107A6800003A002010B5642000F0F4FF8C48FFF7BE
:107A7800A1FE8C4B1B7804460C2B00F2E780DFE854
:107A880013F00D000D00E5007400740037008A0043
:107A9800E5008A008D00A700E500CE00FFF71CFF77
:107AA80018B10120F9F764FED0E07F4B18887F4BAE
:107AB8001B88C01A7E4B1B8890FBF3F07D4B1A88FD
:107AC8007D4B1B88D31A7D4A128893FBF2F3DBB2F5
:107AD800C0B2032B00F29F80DFE803F0020406081F
:107AE800774A3FE0774A3DE0774A3BE0774A39E01A
:107AF800FFF7F2FED8B100210A22754810F0CAF843
:107B0800744B002118600A22734810F0C3F8734BB5
:107B180018600420FEF790F996200521704A00238A
:107B2800FEF7C2F90020FEF787F906F011FF5E4B59
:107B380018885E4B1B88C01A5D4B1B8890FBF3F0BE
:107B48005C4B1A885C4B1B88D31A5C4A128893FBDF
:107B5800F2F3DBB2C0B213B1012B5CD101E05C4A95
:107B680000E05D4A5F4B1A6055E000286ED05E4B1E
:107B78001A7806DD0132D2B20F2A1A7008D91022FB
:107B880005E0013AD2B2102A1A7001D900221A70FF
:107B9800F9F7A8FF5AE0554B187057E0FFF79CFE1D
:107BA800A0B1002152480FF0C1FF524B042083EDD1
:107BB800000AFEF741F9B42005214F4A0023FEF7D9
:107BC80073F9FAF795FB0020FEF736F9484A16E0F4
:107BD800FFF782FE90B1002148480FF0A7FF484BFD
:107BE800042083ED000AFEF727F996200521424A72
:107BF8000023FEF759F90020FEF71EF93F4A394BDA
:107C08001A60294B1888294B1B88C01A284B1B88D7
:107C180090FBF3F0C0B22146FFF7CEFE16E0FFF767
:107C28005BFE08B107F06CF8364B1A68A41814F517
:107C3800967FB8BF344A1C60B8BF1A601B68B3F59A
:107C4800967F03DD2F4B4FF496721A602F48FFF78B
:107C5800B1FD144B1B78013B0A2B60D8DFE803F019
:107C6800065F5F5F5C15155F11111500FFF74AFE8F
:107C7800FFF726FE002852D00220BDE81040F9F791
:107C880077BD234B1B78022B46D10028214B01D10D
:107C9800187010BD01DD012200E0FF221A7010BD2E
:107CA80094010020A4250020143A0020783A0020EE
:107CB80038370020DC390020BA370020A43A0020E9
:107CC800E025002004260020162C0020CC250020CA
:107CD800803A0020B0010020F0390020AC010020DB
:107CE800FBA80508003A0020162600200C3A0020C0
:107CF800FC3500200C0300200BA9050820360020C5
:107D080008030020103A0020D4FEFFFFA001002045
:107D180004380020591A0020BDE81040F2E510BDD3
:107D280010B58CB01E490F2268460EF0A1FD1D4902
:107D38000F2204A80EF09CFD1B490F2208A80EF084
:107D480097FD00210822302000F08AFB012000F076
:107D580081FE002404AB1DF80420E15C302000F013
:107D68007FFB0134012000F075FE0F2CF2D10021B9
:107D78000922302000F074FB012000F06BFE002483
:107D880008AB1DF80420E15C302000F069FB0134E9
:107D9800012000F05FFE0F2CF2D10CB010BD00BF27
:107DA80074A4040883A4040892A4040810B58CB031
:107DB8001E490F2268460EF05BFD1D490F2204A8DC
:107DC8000EF056FD1B490F2208A80EF051FD0021A8
:107DD8000822302000F044FB012000F03BFE002484
:107DE80004AB1DF80420E15C302000F039FB0134BD
:107DF800012000F02FFE0F2CF2D1002109223020A3
:107E080000F02EFB012000F025FE002408AB1DF831
:107E18000420E15C302000F023FB0134012000F055
:107E280019FE0F2CF2D10CB010BD00BFA1A404089C
:107E3800B0A40408BFA4040810B58CB01E490F22D2
:107E480068460EF015FD1D490F2204A80EF010FD1E
:107E58001B490F2208A80EF00BFD00210822302034
:107E680000F0FEFA012000F0F5FD002404AB1DF837
:107E78000420E15C302000F0F3FA0134012000F026
:107E8800E9FD0F2CF2D100210922302000F0E8FA98
:107E9800012000F0DFFD002408AB1DF80420E15CA0
:107EA800302000F0DDFA0134012000F0D3FD0F2C62
:107EB800F2D10CB010BD00BFCEA40408DDA40408A4
:107EC800ECA4040807B50220012108F06BFB01238C
:107ED80000938DF8043002238DF805300448002300
:107EE80069468DF806308DF8073007F0B3FF0EBDF0
:107EF8000004024010B5084C01210022204608F079
:107F08001EF840F2FF4000F0A5FD012120460A4678
:107F1800BDE8104008F013B80004024008B5FFF7A8
:107F2800E9FF00210A46302000F09AFA012000F00B
:107F380091FD01210A46302000F092FA012000F05C
:107F480089FD00210122302000F08AFA012000F08A
:107F580081FD01210822302000F082FA012000F082
:107F680079FD02210122302000F07AFA012000F088
:107F780071FD00210A46302000F072FA012000F05D
:107F880069FD1B21CD22302000F06AFA012000F0A3
:107F980061FD04210322302000F062FA012000F084
:107FA80059FD06210922302000F05AFA012000F07C
:107FB80051FD07210822302000F052FA012000F07C
:107FC80049FD08217022302000F04AFA012000F013
:107FD80041FD1E213020B02200F042FA012000F0BD
:107FE80039FD05219122302000F03AFA012000F0F5
:107FF80031FD0D210322302000F032FA012000F07B
:1080080029FD0E210022302000F02AFA012000F07C
:1080180021FD14218022302000F022FA012000F0F6
:1080280019FD0B218822302000F01AFA012000F0F7
:1080380011FD0C218222302000F012FA012000F0FC
:1080480009FD12218822302000F00AFA012000F0F0
:1080580001FD13218C22302000F002FA012000F0EB
:10806800F9FC00210A46302000F0FAF9012000F05E
:10807800F1FC3D210222302000F0F2F9012000F04D
:10808800E9FCFFF74DFEFFF791FEFFF7D5FE302024
:108098000021012200F0E4F9012000F0DBFC3D2181
:1080A8006422302000F0DCF9012000F0D3FC032129
:1080B8000022302000F0D4F9012000F0CBFC04218C
:1080C8000022302000F0CCF9012000F0C3FC002190
:1080D8000122302000F0C4F9012000F0BBFC0C2183
:1080E8000822302000F0BCF9012000F0B3FC0D217B
:1080F8000822302000F0B4F9012000F0ABFC0E217A
:108108000822302000F0ACF9012000F0A3FC0F2178
:108118000822302000F0A4F9012000F09BFC002187
:108128000A46302000F09CF9012000F093FC02225E
:108138004021302000F094F9012000F08BFC302021
:108148004121002200F08CF9012000F083FC3F213E
:10815800D422302000F084F9012000F07BFC0021BB
:108168000122302000F07CF9012000F073FC10217E
:108178000F22302000F074F9012000F06BFC11216F
:108188000F22302000F06CF9012000F063FC12216E
:108198000022302000F064F9012000F05BFC13217C
:1081A8000022302000F05CF9012000F053FC092186
:1081B8003C22302000F054F9012000F04BFC002153
:1081C8000122302000F04CF9012000F043FC30205F
:1081D8003421024600F044F9012000F03BFC302035
:1081E8003721024600F03CF9012000F033FC36212B
:1081F8000322302000F034F9012000F02BFC392153
:108208000322302000F02CF9012000F023FC3B2150
:108218003C22302000F024F9012000F01BFC3C2116
:108228000A46302000F01CF9012000F013FC002160
:108238000A46302000F014F9012000F00BFC51210F
:10824800C022302000F00CF9012000F003FC52217C
:108258003020002200F004F90120BDE8084000F0B9
:10826800F9BB00BF2DE9F04F454E464D93B00121B3
:108278004FF4001008F096F9304607F039F94FF03E
:10828800C0630293404B0393404B002404934FF484
:10829800B4794FF400334FF480684FF400674FF41B
:1082A800005A4FF4807B304602A90C93019309973A
:1082B800CDF8189005940794CDF82080CDF828A023
:1082C800CDF82CB00D9407F09FF92246304630497E
:1082D80007F0F5F93046012107F0FBF901210A46BC
:1082E8004FF0402008F0CCFB284607F001F9294A56
:1082F800019B0392284A0C9304922846402202A923
:10830800059209970294CDF818900794CDF820802B
:10831800CDF828A0CDF82CB00D9407F075F92246B9
:1083280028461E4907F0CBF92846012107F0D1F964
:1083380042F2107701220221194808F0A1FB3846C1
:1083480000F088FB3046012107F099F90121284601
:1083580007F095F9384600F07DFB0B238DF8443083
:1083680011A801238DF845408DF846408DF8473017
:1083780000F08EFD384600F06DFB13B0BDE8F08FBD
:1083880010600240886002400C400040CA22002071
:108398002A1D00200C3C0040FA1F00205A1A002019
:1083A800003C004002481021012207F0DFB900BF5D
:1083B8001060024013B50220012108F0F3F84FF4D1
:1083C80010730E4C009302238DF804308DF805309D
:1083D80001238DF806302046002369468DF80730C2
:1083E80007F038FD20460621042207F0B3FD204699
:1083F8000921042207F0AEFD1CBD00BF00040240A5
:1084080030B5154D85B001214FF4001008F0EEF895
:10841800284607F0B5FD0023ADF804304BF6FF738E
:10842800ADF806303323ADF808304FF48063ADF86B
:108438000A304FF48043ADF80C3004AC074B2846A3
:10844800012144F8103D07F03DFE2846694607F033
:10845800C5FD05B030BD00BF00540040801A0600BD
:1084680073B54FF4961306460D461446019304E07F
:10847800019B5A1E0192002B57D031484FF400310E
:1084880007F038FF0028F3D12D48012107F026FE18
:108498004FF48053019304E0019B5A1E0192002B74
:1084A80045D02748274907F010FF0028F4D0244872
:1084B8003146002207F02AFE4FF48053019304E06E
:1084C800019B5A1E0192002B33D01D481E4907F00C
:1084D800FCFE0028F4D01A48294607F09AFE4FF40B
:1084E8008053019303E0019B5A1E01921BB3144869
:1084F800164907F0EAFE0028F5D01148214607F092
:1085080088FE4FF49613019303E0019B5A1E0192D3
:108518009BB10B480E4907F0EDFE0028F5D008483E
:10852800012107F0E7FD002008E0012006E0022015
:1085380004E0032002E0042000E005207CBD00BF29
:10854800005400400100030082000700800007007B
:108558000400001037B54FF4961304460D460193F6
:1085680005E0019B5A1E0192002B00F09B805648A3
:108578004FF4003107F0BEFE0028F2D15248012125
:1085880007F0ACFD4FF48053019305E0019B5A1EA0
:108598000192002B00F088804B484C4907F095FE6B
:1085A8000028F3D048482146002207F0AFFD4FF4D9
:1085B8008053019304E0019B5A1E0192002B75D051
:1085C8004148434907F081FE0028F4D03E48294637
:1085D80007F01FFE4FF48053019304E0019B5A1EDD
:1085E8000192002B64D038483A4907F083FE0028EE
:1085F800F4D03548012107F071FD4FF48053019301
:1086080004E0019B5A1E0192002B53D02E482F499B
:1086180007F05BFE0028F4D02B482146012207F022
:1086280075FD4FF48053019304E0019B5A1E01929B
:10863800002B41D0244C2849204607F05BFE002837
:10864800F3D02046002107F069FD20460121238B45
:1086580007F050FD4FF48053019304E0019B5A1E2C
:108668000192002B2AD018481C4907F043FE002825
:10867800F4D0154807F0CFFD4FF480530193124A08
:1086880003E0019B591E0191D3B113889B05F8D4CF
:10869800012104460C4807F041FD0B48104907F03A
:1086A80043FE0EE001240CE002240AE0032408E063
:1086B800042406E0052404E0062402E0072400E080
:1086C800082420463EBD00BF0054004001000300BE
:1086D8008200070004000010020000104000001093
:1086E8000004001013B54FF496130446019305E0F7
:1086F800019B5A1E0192002B00F0AF8060484FF496
:10870800003107F0F7FD0028F2D15D48012107F09C
:10871800E5FC4FF48053019305E0019B5A1E01923A
:10872800002B00F09C805648564907F0CEFD0028E3
:10873800F3D05348A021002207F0E8FC4FF48053FF
:10874800019305E0019B5A1E0192002B00F08980DD
:108758004B484D4907F0B9FD0028F3D0210A484895
:1087680007F057FD4FF48053019304E0019B5A1E14
:108778000192002B77D04248444907F0BBFD0028FE
:10878800F4D0E1B23E4807F044FD4FF48053019322
:1087980004E0019B5A1E0192002B66D038483B49E1
:1087A80007F0A8FD0028F4D03548012107F096FC11
:1087B8004FF48053019304E0019B5A1E0192002B51
:1087C80055D02F482F4907F080FD0028F4D02C48B9
:1087D800A121012207F09AFC4FF48053019304E091
:1087E800019B5A1E0192002B43D0254C2849204654
:1087F80007F080FD0028F3D02046002107F08EFC0A
:1088080020460121238B07F075FC4FF48053019318
:1088180004E0019B5A1E0192002B2CD018481D49D8
:1088280007F068FD0028F4D0154807F0F4FC4FF471
:1088380080530193124A03E0019B591E0191E3B151
:1088480013889905F8D4012104460D4807F066FC01
:108858000B48114907F068FD10E001240EE00224DE
:108868000CE003240AE0042408E0052406E00624BA
:1088780004E0072402E0082400E0092420461CBD87
:1088880000540040010003008200070004000010AB
:1088980002000010400000100004001013B54FF44F
:1088A80096130446019305E0019B5A1E0192002B82
:1088B80000F0AF8060484FF4003107F01BFD00283E
:1088C800F2D15D48012107F009FC4FF48053019370
:1088D80005E0019B5A1E0192002B00F09C8056482F
:1088E800564907F0F2FC0028F3D05348A021002293
:1088F80007F00CFC4FF48053019305E0019B5A1ECE
:108908000192002B00F089804B484D4907F0DDFCAF
:108918000028F3D0210A484807F07BFC4FF4805325
:10892800019304E0019B5A1E0192002B77D0424824
:10893800444907F0DFFC0028F4D0E1B23E4807F0D4
:1089480068FC4FF48053019304E0019B5A1E019286
:10895800002B66D038483B4907F0CCFC0028F4D0FF
:108968003548012107F0BAFB4FF48053019304E026
:10897800019B5A1E0192002B55D02F482F4907F012
:10898800A4FC0028F4D02C48A121012207F0BEFB4A
:108998004FF48053019304E0019B5A1E0192002B6F
:1089A80043D0254C2849204607F0A4FC0028F3D0E2
:1089B8002046002107F0B2FB20460121238B07F057
:1089C80099FB4FF48053019304E0019B5A1E0192D6
:1089D800002B2CD018481D4907F08CFC0028F4D037
:1089E800154807F018FC4FF480530193124A03E02E
:1089F800019B591E0191E3B113889C05F8D401210C
:108A080004460D4807F08AFB0B48114907F08CFC17
:108A180010E001240EE002240CE003240AE0042400
:108A280008E0052406E0062404E0072402E0082400
:108A380000E0092420461CBD00540040010003004A
:108A4800820007000400001002000010400000101F
:108A58000004001082B0002304E0019B013301935D
:108A6800009B01330093009B8342F6D302B070470A
:108A780037B54FF4805304460D46019304E0019B3B
:108A88005A1E0192002B6DD03C484FF4003107F07C
:108A980031FC0028F3D13948012107F01FFB4FF4BE
:108AA8008053019304E0019B5A1E0192002B5BD076
:108AB8003248334907F009FC0028F4D02F48A02198
:108AC800002207F023FB4FF48053019304E0019B3D
:108AD8005A1E0192002B49D028482A4907F0F5FB75
:108AE8000028F4D0210A254807F093FB4FF480535F
:108AF800019304E0019B5A1E0192002B38D01F48B5
:108B0800214907F0E2FB0028F4D0E1B21B4807F046
:108B180080FB4FF48053019303E0019B5A1E01929E
:108B280043B31648184907F0D0FB0028F5D013487E
:108B3800294607F06EFB4FF49613019303E0019B5F
:108B48005A1E0192C3B10D48104907F0D3FB002803
:108B5800F5D00A48012107F0CDFA0D48FFF77AFF52
:108B680000200AE0012008E0022006E0032004E0DB
:108B7800042002E0052000E006203EBD005400402D
:108B880001000300820007008000070004000010B5
:108B9800A0860100F7B54FF4805304460D461646EB
:108BA800019304E0019B5A1E0192002B74D04048A7
:108BB8004FF4003107F09EFB0028F3D13C48012117
:108BC80007F08CFA4FF48053019304E0019B5A1E7E
:108BD8000192002B62D03648364907F076FB002810
:108BE800F4D03348A021002207F090FA4FF48053C4
:108BF800019304E0019B5A1E0192002B50D02C488F
:108C08002D4907F062FB0028F4D0210A284807F014
:108C180000FB4FF48053019304E0019B5A1E01921C
:108C2800002B3FD02248254907F04FFB0028F4D0FD
:108C3800E1B21F4807F0EDFA4FF48053019304E0C6
:108C4800019B5A1E0192002B2ED019481B4907F090
:108C58003CFB0028F4D000244FF4961710E0295D5F
:108C6800134807F0D6FA019703E0019B5A1E0192B8
:108C7800E3B10F48124907F03DFB0028F5D0013455
:108C8800E3B2B342EBD30A48012107F033FA0D48A7
:108C9800FFF7E0FE00200AE0012008E0022006E0DD
:108CA800032004E0042002E0052000E00620FEBDC9
:108CB8000054004001000300820007008000070004
:108CC80004000010A086010013B50520012107F05B
:108CD80069FC184C4FF4E053009302238DF80430DC
:108CE8008DF805302046002369468DF806308DF84A
:108CF800073007F0AFF820460A21062207F02AF9C4
:108D080020460C21062207F025F9062220460B21D1
:108D1800A4F5006407F01EF94FF4004320466946A5
:108D2800009307F097F820460F21062207F012F962
:108D38001CBD00BF000802401FB50446FFF7C2F87B
:108D4800FFF75EFBFFF7EAF8FFF7BEFF01214FF4DC
:108D5800004007F04BFC02940F4C1023ADF8023092
:108D6800204600236946ADF80430ADF80C30ADF864
:108D78000030ADF8063007F068FD69464FF0402036
:108D880007F037FE2046012107F0E7FD4FF04020AD
:108D9800012107F0E2FD1FBD003C004082B0002326
:108DA80004E0019B01330193009B01330093009B76
:108DB8008342F6D302B0704707B50420012107F0BB
:108DC800F1FB01214FF4804007F01CFC4FF40073C5
:108DD800009300238DF804300348012369468DF879
:108DE800073007F037F80EBD000802400D4B07B5F5
:108DF8001A680D484FF47A73B2FBF3F20B4B013A41
:108E08005A600B4AF02182F8231000229A60072248
:108E18001A60084B084A00930121084B01F0ECFF47
:108E28000EBD00BFD00100201C26002010E000E08D
:108E380000ED00E0EC020020D00200203802002003
:108E4800054B1A6812B11A68013A1A60034B1A687E
:108E580001321A60704700BFDC250020F42500208D
:108E680082B0044B0190019A1A601A68002AFCD15A
:108E780002B07047DC250020704700BF40F0BE609C
:108E8800024B40F42020D860704700BF00ED00E09E
:108E9800C37810B503B3164B4278DB688478DB439C
:108EA800C3F30223C3F10401C9B202FA01F10F228C
:108EB80042FA03F2C9B222400A430E4B017812016A
:108EC800CB18D2B283F8002303780122590903F0A2
:108ED8001F0302FA03F307E003780122590903F09C
:108EE8001F0302FA03F32031024A42F8213010BD71
:108EF80000ED00E000E100E021F0604121F07F0199
:108F0800014B08439860704700ED00E0044B1A6974
:108F180009B1104301E022EA00001861704700BF60
:108F280000ED00E0044B1A6804280CBF42F004026C
:108F380022F004021A60704710E000E0014B93ED44
:108F4800000A70473C2C0020014B93ED000A704743
:108F5800342C0020014B93ED000A7047482C002068
:108F6800014B93ED000A7047382C0020014B93ED1C
:108F7800000A70474C2C0020014B93ED000A704703
:108F8800402C00200000000010B5FDF78FFE0020E7
:108F9800012324210246FDF7F3FE114B1C78002023
:108FA800012C05D10146FDF7C4FF2046002104E04D
:108FB8000721FDF7BEFF01200721FDF7BAFF632255
:108FC8001221C020FFF74CFA02200121FDF7B1FF62
:108FD800FEF78EF80120BDE81040FEF77EB800BF0E
:108FE800F40D00200D4B1B78062B05D10C4B0D4AB8
:108FF800196812688A181A600B4B1B78012B084BEA
:10900800196805D1094A914207DD01321A60704793
:10901800074A914201DD01321A607047A4250020F9
:10902800102C00209C250020F40D00207FD1F00892
:10903800FF27ED080E4B1B78062B05D10D4B0E4A6A
:10904800196812688A1A1A600C4B1B78012B094B95
:1090580005D10B4A1968914208DC1A6070471A68F2
:10906800B2F57A2FDCBF4FF47A221A60704700BF3E
:10907800A4250020102C00209C250020F40D0020A1
:1090880020A107002DE9F04F694B6A4C1B688DB091
:1090980019220A9068485343B0FBF1F01C190D4699
:1090A80008F010FE41EC100B0AF042FF51EC100BD7
:1090B80009F040F910F0010F804618BF00F1FF38A1
:1090C80005FB08F008F0FEFD064620460F4608F0AE
:1090D800F9FD02460B463046394608F093FF044630
:1090E8000D4645EC104B0AF023FF57EC106B204659
:1090F80032463B46294608F0A7FCCDE9020139462D
:10910800304609F017F946A3D3E900230B90DDE9AF
:10911800020109F0C9F8002858D1012000264FF0B3
:109128001509314607464FF0000A4FF0000B03E0DF
:1091380030463946069E049FA7FB0A23541807FBAE
:109148000B333E4A43F100050023A242AB41CDE96F
:1091580004453ED3A6FB0A23141806FB0B333748F5
:1091680043F100050021A042A941CDE9064530D3CD
:10917800DDE902012CA3D3E90023049C069D09F034
:1091880093F840BBDDE9022300202D4908F03AFF9F
:1091980082468B464BEC10AB0AF0CAFE5046594645
:1091A80053EC102B8DED080B08F04EFCCDE90201B5
:1091B800DDE9080109F08CFB09F1FF395FFA89F94B
:1091C80082468B46B9F1000FB2D104E00125002494
:1091D80001E035463C460B9A0A9BD1B25BB918466A
:1091E80022462B46FDF7CCFD0A9801230093014641
:1091F8004246034609E022462B460120FDF7C0FD02
:1092080001200090014642460023FDF7ACFEFDF721
:109218006FFF01200DB0BDE8F04FFDF75EBF00BF46
:10922800956479E17FFDA53DBBBDD7D9DF7CDB3DEA
:10923800103A002040787D0100E9A435FFFF0F00B7
:109248000000F03F224A234B1278012A10B518601B
:1092580009D1214A904201DD01321A601F4A1B6878
:1092680093420DDC0AE01E4A904201DD01321A6089
:109278001B68B3F57A2F03DC4FF47A22154B1A607A
:10928800144B184A1968184B184C1B68CB18934292
:10929800236018DC0020FFF7F5FE01202168FFF7A6
:1092A800F1FE0B4B1C780020012C05D10146FDF77F
:1092B80040FE2046002104E00721FDF73AFE012088
:1092C8000721FDF736FE034B1A68094B1A6010BDDB
:1092D800F40D0020102C00207FD1F00820A10700F9
:1092E800FF27ED0880D1F008282C00202C2C002026
:1092F800F8350020014B1868A4E700BF10260020AD
:109308007047FEE7FEE7FEE7FEE7704770477047E5
:1093180002F022B910B5094CA37A4BB1084B1A6870
:1093280022F006021A6000F013F8204600F041FE11
:109338004FF48020BDE8104006F0E8BA1C26002053
:1093480010ED00E0014801F003B800BF1C26002022
:10935800364BD3F8882042F47002C3F88820344B87
:109368001A6842F001021A6000229A60196821F016
:10937800847121F4803119602E495960196882B0CE
:1093880021F480211960DA60009201921A6842F48F
:1093980080321A601A6802F400320192009A01328F
:1093A8000092019A1AB9009AB2F5A06FF2D1204B37
:1093B8001B6813F4003318BF01230193019B012B91
:1093C8002ED11B4B1A6C42F080521A641A4A11684B
:1093D80041F4804111609A689A609A6842F40042A8
:1093E8009A609A6842F4A0529A60144A5A601A68BD
:1093F80042F080721A6019680D4A8901FBD5104B3A
:1094080040F205611960936823F003039360936841
:1094180043F002039360936803F00C03082BFAD11E
:10942800024B4FF000629A6002B0704700ED00E016
:1094380000380240103000240070004008544007F3
:10944800003C0240184B194A996801F00C010429A4
:1094580003D0082903D0164B19E0164B17E05968BA
:109468005A6811F4800F596814BF124B104B02F060
:109478003F02B3FBF2F30C4A5268C2F30142C1F354
:109488008811013252004B43B3FBF2F3074A1360D1
:10949800054B9A68054BC2F303129A18196812799A
:1094A80021FA02F21A60704700380240D001002009
:1094B8000024F40000127A0037B51C23012400258B
:1094C80001A88DF804308DF805508DF806408DF808
:1094D8000740FFF7DDFC2046214607F087F80A49D8
:1094E80040F2E1434B6040F24F130B800D814D80F9
:1094F8004FF0804007F022FC4FF080402146224682
:1095080007F0E1FF3EBD00BF502C002008B54FF02A
:109518008040012107F0ECFF60B101214FF080404D
:1095280007F0F1FFFEF79EFA034B044A11781A7808
:109538008A181A7008BD00BFC32500200C3A002005
:1095480008B5402006F0D4F930B1FCF70BFE4020F6
:10955800BDE8084006F0DAB908BD0000014608B5C4
:10956800044808F08FF90348402108F038FA002829
:10957800F9D008BD00440040F0B589B04FF4E1339C
:109588000120019300232B4CADF808301E460146FC
:10959800ADF80A30ADF80C30ADF810300C23ADF84A
:1095A8000E3006F0FFFF4FF40030012107F01EF8DF
:1095B80020680221072206F0CDFC072260680321FB
:1095C80006F0C8FC0125022704232068059305A995
:1095D8008DF81A608DF81B508DF818708DF8197079
:1095E80006F038FC08236068059305A98DF8187003
:1095F80006F030FCA06801A908F09AF82A4640F263
:1096080025510D4808F0D2F9262307A88DF81C30FB
:109618008DF81D608DF81E608DF81F50FFF738FC1F
:10962800A068294608F001F9044A054B1A6009B0F8
:10963800F0BD00BFE401002000440040659500082B
:109648009C3B0020024B9868002108F0EEB800BF50
:10965800E401002010B5094C40F22551204608F0DD
:10966800C8F950B1A288D2B2112A02D1044B012103
:109678001970044B19884A401A8010BD00440040F4
:10968800550D0020600D00207047704773B501200C
:10969800014606F087FF264C4FF4D8530093022367
:1096A80003268DF804302046002369468DF80630DD
:1096B8008DF807308DF8056006F0CCFB20460821B0
:1096C8000A2206F047FC204609210A2206F042FC3D
:1096D80020460B210A2206F03DFC0A2220460C21D6
:1096E80006F038FC01254FF4806320466946009354
:1096F8008DF806508DF807508DF8056006F0AAFB26
:109708000A210A46204606F025FC29464FF48040E7
:1097180006F078FF8020294606F050FF4FF0805071
:10972800294606F09FFF284606F0F0F87CBD00BFEA
:109738000000024007B54FF4C060FFF79FFB4323CA
:109748008DF804300322012301A88DF805308DF827
:1097580006208DF80730FFF79BFB0EBD7823584392
:109768000723B0FBF3F0002301338342FCD9704791
:109778004FF47A735843F1E737B50023104C01933F
:1097880005460320FFF7EAFFEB681A69013C0192DE
:1097980013D0019A002AF4DA019A42F001020192E8
:1097A800019A1A61064A1969013A019102D0019990
:1097B800C907F8D40320FFF7D1FF00203EBD00BF42
:1097C800410D030010B5C47874B900EB820003336F
:1097D8009B10D0F8D000224603E051F8044C013227
:1097E800046004319A42F8D1002010BD033230B52C
:1097F8009210D0F8D0400B46002003E025680130D5
:1098080043F8045C04339042F8D101EB800030BD8A
:109818000122F0B50023827040220129C3708280A2
:109828000CD108230370042343704FF4A073C38042
:1098380002230372C1724FF0A04309E041B90C231F
:109848000370062343704FF4A063C3801F4BC1729B
:1098580003F500620261C3604678044601461A4671
:10986800002508E002F5106C02F530620A65C1F8BF
:1098780014C001353A460431B54202F12007F1D34C
:1098880003F58062426103F58862C0F8CC2006784F
:1098980003F5A0650146002203E0C1F88C500132AF
:1098A80020350431B242F8D31946002202E0C4F848
:1098B800CC1001320434B24201F58051F7D303F5DC
:1098C8006063C0F80C310020F0BD00BF0000044008
:1098D80038B5037AC2680025012B044625D1936B5D
:1098E800417A65F3104309B143F480139363D36855
:1098F80023F4800323F0500343F010036FF3C303F2
:109908006FF3C7136FF351436FF3D343D36020460C
:10991800FFF732FFE378012B3ED1052363F34405BB
:10992800E36845F020059D6036E0D36843F04003C6
:10993800D360FFF721FF237A627A032B14BF4FF419
:1099480034134FF43C130AB143F48013E268142033
:109958009363FFF70DFFE268217AD368032908BFF4
:1099680043F48033D360237A032B15D1156B01237D
:1099780063F39B656FF3D7552D2345F0805563F34B
:1099880016451563C820FFF7F3FEE36845F40005A4
:109998001D63C820FFF7ECFEE378012B07D1E368CD
:1099A8009D68052262F3440545F020059D6000206E
:1099B80038BDC3689A6842F001029A600020704777
:1099C800C3689A6822F001029A600020704707B5C0
:1099D80000230193019B43F020030193019B61F352
:1099E8008A130193019BC2681361064B1169013BFD
:1099F800019102D001998806F8D40320FFF7AEFE42
:109A080000200EBD410D030007B500230193019B03
:109A180043F010030193019BC2681361064B11695F
:109A2800013B019102D00199C906F8D40320FFF740
:109A380095FE00200EBD00BF410D030008B5C268A9
:109A4800D36801296FF35D736FF39E7302D143F0FE
:109A5800005302E009B943F080433220D360FFF796
:109A680087FE002008BDC368586900F001007047F0
:109A7800C3685B6913F0010F14BF00200120704711
:109A8800C368586900F001007047C3685A6998694B
:109A980010407047C3685868704703691A6861F3D3
:109AA80001021A607047C268002393614FF0FF33C8
:109AB8005361536053610B4B9361C3789169002BD9
:109AC80014BF4FF400634FF4016343F4701343F47D
:109AD800405343F0080321EA03010B43936100203C
:109AE800704700BF00080080F8B5D0F80C3100229C
:109AF8001A60036915461A6865F3CC221A60C37A9E
:109B0800012B04461BD10321FFF7C7FFE36880211F
:109B18004FF4800261F30F0259629A62C02262F325
:109B28000F0561F31F454FF4A072C3F8045162F3A7
:109B38000F056FF31F45C3F80851C3F80C511021E6
:109B48002046FFF744FF2046FFF75EFF2269002307
:109B58004FF0FF311361204653611E469161FF2586
:109B6800D361214610E082691768C7F3076707F0D9
:109B78008007FFB2002F14BF4FF0904700271760EF
:109B8800013316610430956062789342EBD3002369
:109B98001D46FF2010E04A6D1668C6F3076606F0FA
:109BA8008006F6B2002E14BF4FF0904600261660CD
:109BB800013315610431906062789342EBD32369D5
:109BC8001A6942F480721A61E278012A04D1054ABE
:109BD800402161F359421A632046FFF764FF0020D1
:109BE800F8BD00BF0301010003699B68C3F341038B
:109BF800013B022B9ABF024AD05C0320704700BF8A
:109C080030A5040810B5036981699C680A68C4F323
:109C18004100022802D06FF30A0202E0032060F339
:109C28000A020A605A6842F480725A60002010BD25
:109C380030B54D780B780022012D00EB830405D157
:109C480005FA03F3A46963F30F0205E0012505FA99
:109C580003F3646D63F31F422368C3F3072505F01C
:109C68008005EDB26DB98D6865F30A03CD78C988B2
:109C780065F3934361F3995343F0805343F40043EE
:109C880023600369D9690A43DA61002030BD30B521
:109C98004D780B780024012D224600EB830105D175
:109CA80005FA03F3896963F30F0205E0012505FA54
:109CB80003F3496D63F31F4203696FF3CF340C60FC
:109CC800D96921EA0202DA61002030BDF8B54F787F
:109CD8000B78012F00EB830349D19E694C693568E5
:109CE80033692A4664F3120314B967F3DC430BE0C3
:109CF8008F68E419013CB4FBF7F7CC7867F3DC43D1
:109D0800012C08BF64F35E733361C378012B06D15D
:109D18000B780C6900EB83039B695C610CE0CB78E2
:109D2800012B09D04B693BB103690C785E6B0127A5
:109D380007FA04F434435C63CB78012B07D1036939
:109D48009B68DB0554BF45F0005245F080520B7804
:109D580000EB830342F004429B691A60CB78012B25
:109D680038D10A788B8AC968FFF72CFD32E05E6D1E
:109D78004F6935688C6833692A462FB964F3120332
:109D8800012464F3DC430AE03F19013FB7FBF4F711
:109D9800BF05BF0D67F3DC437C4364F312033361F3
:109DA800C378012B05D10B780C6900EB83035B6D3D
:109DB8005C61CB78012B06D14B7913B145F0005289
:109DC80001E045F080520B7800EB830042F004423A
:109DD800436D1A600020F8BD73B54D78012D3DD153
:109DE80083694A691E681C690094E4B242B962F347
:109DF80006048DF800409DF8024065F3C4040EE0A7
:109E08008D68AA4286BF4D6165F3060462F30604B5
:109E18008DF800409DF80240012262F3C4048DF8D9
:109E28000240009A1A61C278012A05D10A780C69A1
:109E380000EB82029269546146F004421A60C378CA
:109E4800002B34D14B69002B31D003690A78586B49
:109E5800012101FA02F202435A6328E00B784E69A5
:109E68008C6800EB83035B6D1A681D690095EDB281
:109E780006B14C6164F306059DF802408DF8005068
:109E8800012565F3C4048DF80240009C1C61C37869
:109E9800012B05D10B780C6900EB83035B6D5C61CA
:109EA8000B7800EB830042F00442436D1A600020F7
:109EB8007CBD4B78012B0B7800EB83000AD18269BB
:109EC8001368C3F3076101F08001C9B221B143F0FF
:109ED800804301E0426D136843F4001313600020CF
:109EE80070474B78012B0B78C97800EB83000CBFC7
:109EF8008269426D02391368C9B26FF3555301295B
:109F080098BF43F0805313600020704703699A6933
:109F1800D8691040000C704700EB810102694B6D55
:109F28009B6850691840704703699869DB69184055
:109F380080B2704782B000230093C0238DF80330AD
:109F48000122002362F3C4038DF8023018238DF830
:109F58000030009A436D1A61C278012A06D100F5D3
:109F6800B96058611A684FF080221A6002B07047D1
:109F7800D0F8143110B50446D3B103699A68D207F2
:109F880016D5827A42B1D0F80C21D0F80C116FF3B3
:109F980041026FF300020A605A6842F001025A60F7
:109FA8000520FFF7E5FB23695A6822F001025A6091
:109FB80010BD837A63B103699B68D90708D5D0F8C7
:109FC8000C31D0F80C216FF341036FF300031360D9
:109FD8007047012310B5002280F812310446034669
:109FE800FF2104E058698160186D01328160607852
:109FF80004338242F6D3236900221A615A61DA6176
:10A008004FF0FF329A612046FFF7FEFC20461021F0
:10A01800BDE81040DBE44B78012B0B7800EB8300A4
:10A028000FD183691868C0F3074000F02003DBB242
:10A03800CBB900F00200C0B200280CBF30202020AD
:10A048007047436D1868C0F3074000F02003DBB287
:10A058005BB900F00200C0B200280CBF4FF44050BA
:10A068004FF400507047102070474FF480507047ED
:10A078004B78012B0B7810B500EB83030AD19C6950
:10A08800102A236802D1BDE8104012E7202A0CD01C
:10A09800302A0FE05C6DB2F5805F236802D143F48B
:10A0A80000131BE0B2F5005F02D143F0006315E036
:10A0B800B2F5405F0FD1C3F3074202F02002D2B2DB
:10A0C80022B100234B71BDE810400AE743F08063DA
:10A0D80043F0802302E00AB962F3CF33236010BD56
:10A0E800F8B50446FFF794FB0122002384F81221F7
:10A0F80084F8133128271646194640250CE007FB3B
:10A1080003F000F58C7022182354D3805670D17058
:10A118009560D1605161013362789342EFD3002397
:10A128002826194640250CE006FB03F000F55C7074
:10A1380022182354D3805170D1709560D160516139
:10A14800013362789342EFD32046FFF739FC20466B
:10A15800FFF7BEFB00212046FFF770FC2046FFF703
:10A16800C3FC2046BDE8F840FFF723BC70B5CDB26C
:10A178000C464FF0280601F07F0106FB010115F09F
:10A18800800F14BF01F58C7101F55C7104F07F0438
:10A19800ED090C704D708A60CB7005B1CC80022B34
:10A1A80001D100230B71FFF743FD002070BD10B5EE
:10A1B800CAB201F07F034FF0280404FB030312F036
:10A1C800800F14BF03F58C7303F55C7301F07F01F6
:10A1D800D20919705A701946FFF759FD002010BDB1
:10A1E80038B501F07F0528246C4304F55C74011927
:10A1F8004B6100238B614B70EBB20355CA60C47886
:10A20800012C08BF0A6113B9FFF7E6FD01E0FFF76B
:10A218005DFD002038BD70B501F07F042825654339
:10A2280005F58C7541190126E4B2CA600A6100225D
:10A238004E7044558A614B6114B9FFF7CDFD01E0BA
:10A24800FFF744FD002070BDCAB212F0800F10B5B0
:10A258004FF0280306D001F07F0403FB040303F545
:10A268008C7303E003FB010303F55C73D20901243B
:10A2780001F07F0119709C705A701946FFF719FE9A
:10A28800002010BDCAB212F0800F10B54FF028039D
:10A2980006D001F07F0403FB040303F58C7303E08D
:10A2A80003FB010303F55C730024D20901F07F016D
:10A2B80019709C705A701946FFF713FE204610BD9E
:10A2C80008B50B0604D501F07F01FFF780FB01E01C
:10A2D800FFF79AFB002008BD0369002261F30A1208
:10A2E80019680A431A60704703695A6803206FF3B4
:10A2F80041025A60FFF73CBA03695A68032042F0EA
:10A3080002025A60FFF734BA11F0800F4FF02803A9
:10A3180006D001F07F0103FB010101F58C7103E018
:10A3280003FB010101F55C71FFF775BE11F0800FA9
:10A338004FF0280306D001F07F0103FB010101F56E
:10A348008C7103E003FB010101F55C71FFF790BE1E
:10A358002DE9F74F0446FFF78BFB002800F03F82FA
:10A368002046FFF792FB0546002800F03882C0F32C
:10A37800074000F00800C0B2002861D02046FFF76F
:10A38800C5FDA146824627464FF00008DFF86CB3AA
:10A398002E4650E01AF0010F46D05FFA88F21146B7
:10A3A80020460092FFF7B8FD10F0010F0546009A0D
:10A3B80020D07B6D01259D60E178A94207D11B69FA
:10A3C800D9F87813C3F31203CB1AC9F88833DBF82A
:10A3D800003020461B6811469847E378012B09D1C5
:10A3E800B8F1000F06D194F81131052B02D120469F
:10A3F800FFF7A0FD05F00203DBB213B17B6D022568
:10A408009D6005F00403DBB213B17B6D04259D60EC
:10A4180005F00805EDB23DB1DBF8003020469B6839
:10A4280098477B6D0820986008F101084FEA5A0A9E
:10A43800043709F12809BAF1000FABD135460120DC
:10A44800C5F3074303F00403DBB2002B00F0AF8031
:10A458002046FFF769FD264683464FF00008019520
:10A468009FE01BF0010F00F0978023695FFA88F9DD
:10A4780019695D6B04EB890225FA09F59269ED010A
:10A488009268EDB20D431540EA071CD55A6B0120BE
:10A4980000FA08F122EA01025A63B369974A986000
:10A4A800136805465B68204649469847E378AB42FF
:10A4B80009D1B8F1000F06D194F81131042B02D15B
:10A4C8002046FFF737FD05F00403DBB213B1B3698B
:10A4D80004259D6005F00803DBB213B1B3690825B4
:10A4E8009D6005F01003DBB213B1B36910259D60C0
:10A4F80005F02003DBB213B1B36920259D6005F098
:10A508004003DBB213B1B36940259D6005F0020337
:10A51800DBB213B1B36902259D6025F07F0515F004
:10A52800FF0F39D0282505FB084505F58C75C2466F
:10A53800AB696A69C3EB020CAB689C4528BF9C46B3
:10A548000CF1030CB3694FEA9C0C9B696746A04663
:10A5580014E0AA68E9681C1B944228BF1446A3B2F9
:10A5680040464A46FFF72EF9EB681B19EB60AB69CA
:10A57800E71C1C19AC61B3699B69BF089BB2BB425D
:10A5880005D9AC696B699C4201D2002BE1D1B36952
:10A59800802544469D60D04608F101084FEA5B0BD0
:10A5A8000436BBF1000F7FF45CAF019D012005F07C
:10A5B8000203DBB213B1E36802225A61C5F30763F1
:10A5C80003F08003DBB2CBB1A37A43B1D4F80C31EA
:10A5D800D4F80C216FF341036FF300031360236970
:10A5E8005A6822F001025A60444B1B6820469B6956
:10A5F8009847E3684FF000425A610120C5F30723EA
:10A6080003F00803DBB2F3B13C4B1B6820465B69DF
:10A6180098472369E2689B684FF400615161A27A08
:10A6280082B1DB070ED5D4F80C311A6842F001026A
:10A638001A601A6842F003021A60314B1A6942F034
:10A6480006021A61012005F00803DBB243B12B4B67
:10A658001B682046DB689847E36808225A61012096
:10A6680005F01003DBB2002B33D0E3689A6922F0BF
:10A6780010029A611F6A282607F00F0306FB03469B
:10A68800C7F34343022B06F55C7602D0062B1AD19A
:10A698000EE047F6F0733B40ABB1C7F30A1720460C
:10A6A800F1683A46FFF7A2F8F368DB19F36007E0B0
:10A6B80004F5B96120460822FFF798F8C7F30A178E
:10A6C800B369DF19B761E3689A6942F010029A61C9
:10A6D8000120C5F3072303F01003DBB2002B39D0A8
:10A6E80023695A68002622F001025A603146204642
:10A6F800FFF76DF923463246FF2108E0800200206B
:10A7080000ED00E058698160186D01328160607861
:10A7180004338242F6D3236901274FF0FF3267F3EF
:10A728000F069A6167F31F460F22DE615A612F22D6
:10A738001A611A686FF30A121A602046FFF7FAFBCB
:10A74800E3684FF480525A61264B1B6820461B6908
:10A7580098473846C5F3072303F02003DBB2EBB173
:10A768002046FFF74FFAE3682046DE68FFF73CFA19
:10A77800032806D10023A3704FF40073A380092394
:10A7880004E00123A3704023A380052363F38D26EF
:10A79800E3684FF40052DE6001205A61C5F30743B5
:10A7A80003F01003DBB24BB10E4B1B682046DB698C
:10A7B8009847E3684FF480125A610120C5F30745B2
:10A7C80005F02005EDB255B1064B1B6820461B6A03
:10A7D8009847E3684FF400125A610120FFE7BDE88B
:10A7E800FE8F00BF8002002043230B800048704783
:10A7F800F001002038B51F4B1A68511C052A196052
:10A8080035D11979002201291A6030D09968B1F53B
:10A81800006F08BF9A60174B9968DC68A1421A4616
:10A8280002D100221A7122E086BFC1F500631361CC
:10A83800C1EB0404D0F8EC3598BF14611569B3F87E
:10A8480039300C4C9D428AB204D95918ED1AA160CE
:10A85800256104E06918A1600021ABB221610549B6
:10A8680001240C7104498A188121FFF7D4FC0020C7
:10A8780038BD00BF640D0020EF2C002038B5282318
:10A888000A4D03FB01010A4BB1F888131B69044602
:10A8980028469847D4F8EC352046B3F840300121D3
:10A8A8002A46FFF79DFC002038BD00BFA72C0020DA
:10A8B8006C02002070B50B7813F0600506460C4654
:10A8C80025D0202D1FD1CD88B5B113F0800F487841
:10A8D80008D0214B21499B682A469847E2881F499E
:10A8E800304625E01E4B1D4958641E4B30465D61BD
:10A8F8002A4600F022FB1DE0174B48789B68294642
:10A908002A46984725E000F077FB022521E04B789E
:10A918000A2B11D00B2B14D0062B1AD14B881B0AEB
:10A92800212B03D1CA883A2A28BF3A220E49304639
:10A9380000F0EAFA00250CE00C49012200F0E4FAE4
:10A9480007E08B781BB9074A1D46936101E000F0C8
:10A9580053FB284670BD00BF6C020020E72C002086
:10A96800F0010020640D0020020200207C0D002070
:10A9780010B581210446FFF71AFC01212046FFF794
:10A9880016FC82212046FFF712FC024B5B689847B1
:10A99800002010BD6C02002038B5D0F8EC35044614
:10A9A800B3F8392081210223FFF7E0FBD4F8EC3516
:10A9B8000121B3F8402020460223FFF7D7FB82216C
:10A9C800082203232046FFF7D1FB094B022200256A
:10A9D8001A715D71074B1B689847D4F8EC35064A25
:10A9E800B3F8403020460121FFF7FAFB284638BD6E
:10A9F800B00200206C020020A72C002010B5074CE4
:10AA0800606CFF2807D0064B064A9B6806495269C6
:10AA18009847FF236364002010BD00BFF0010020A9
:10AA28006C020020640D0020E72C002038B5104986
:10AA38000B79012B19D10C690CB90C7115E0D0F800
:10AA4800EC358D68B3F839309C42AAB203D95D1948
:10AA58008D60E41A03E0A3B22C198C6000240C6109
:10AA6800044952188121FFF7D6FB002038BD00BFEA
:10AA7800640D0020EF2C0020002070470020704754
:10AA88000023F0B5084A094E1D4609E01468C75C62
:10AA9800375501340133B4F5006F146008BF1560F1
:10AAA8008B42F3D10020F0BD700D0020EF2C002068
:10AAB800104B114AD3F800C000232DE9F0410F4F85
:10AAC80016461D460DE0146810F8038007F8048048
:10AAD8000134802C08BF2C4614603468644505D0C6
:10AAE80001338B42EFD10020BDE8F0810220BDE8A0
:10AAF800F08100BF7035002084350020F03400203C
:10AB080021280FD1084B1A680A701A68120A4A706D
:10AB18005A888A70DA78CA701A790A715A794A7129
:10AB28009B798B71002070476402002007B502AB47
:10AB3800012103F8010D1846FFF7A2FF0EBD002101
:10AB480000E00131435C002BFBD199E798E70B4B00
:10AB58000B491A68096891420BD00A498A5C02704D
:10AB68001A680132802A1A6005D100221A60012071
:10AB78007047002070470120704700BF70350020E3
:10AB880084350020F0340020204B1A68204B1B68C5
:10AB98009A42F0B509D135E00133802B08BF002374
:10ABA8009A4203D11A4B1A602CE01A4CE15C002936
:10ABB800F2D00A29F0D00D29EED0154C1549134DC5
:10ABC80023600E460023CF182268BA5CC25422685C
:10ABD80001339F18802F08BF53422F689A18974255
:10ABE80010D0B25C1AB10A2A01D00D2AEBD100228A
:10ABF800C254074A116859187F29116003D980394E
:10AC0800116000E000231846F0BD00BF8435002025
:10AC180070350020F0340020704700BFD0F8E435CC
:10AC280010B51B6904469847032384F812310020A5
:10AC380010BD08B5042380F81231D0F8E435DB687C
:10AC48009847002008BD08B5D0F8E035DB6903B1A6
:10AC58009847002008BD08B5D0F8E0351B6A98472A
:10AC6800002008BD08B5D0F8E0355B6A9847002099
:10AC780008BD002110B5402204460B46FFF776FABE
:10AC88008021402200232046FFF770FA012384F830
:10AC98001231D4F8E435A0785B689847002010BDDD
:10ACA80013B56946044600F085F99DF8001001F0D7
:10ACB8001F03012B07D0022B0AD073B9204669461F
:10ACC80000F026FA0FE02046694600F007FA0AE08D
:10ACD8002046694600F0A2F905E021F07F01C9B2DB
:10ACE8002046FFF7B1FA00201CBD38B504460029FC
:10ACF8003DD190F81131022B42D1D0F83421D0F84F
:10AD080020319A4211D9C178D21A0129C0F83421C8
:10AD180004D1D0F82411CB18C0F8243192B22046BF
:10AD2800D4F8241100F000F92AE0D0F83821B2FB59
:10AD3800F3F503FB152565B99A420AD3D0F83C31DF
:10AD48009A4206D229462A4600F0EEF8C4F83C5149
:10AD580016E0D4F8E035DB682BB194F81221032A09
:10AD680001D120469847204600F00FF908E0D0F8B6
:10AD7800E0355B6923B190F81221032A00D1984786
:10AD8800002038BD10B5044659BB90F81131032B8B
:10AD980030D1D0F88C23D0F878339A4214D9C178BE
:10ADA800D21A0129C0F88C2304D1D0F87C13C91811
:10ADB800C0F87C139A4228BF1A4692B22046D4F8AB
:10ADC8007C1300F0CAF815E0D0F8E0351B6923B110
:10ADD80090F81221032A00D19847204600F0C6F8BF
:10ADE80008E0D0F8E0359B6923B190F81221032AD6
:10ADF80000D19847002010BD2DE9F041069F044678
:10AE0800164698460D46FEF741FC20462946C4F8EA
:10AE1800E085C4F8E475C4F8E865FFF761F9D4F88B
:10AE2800E4351B6898472046BDE8F041FEF782BC30
:10AE380000207047D0F8E03510B504461B689847E5
:10AE4800D4F8E4359B689847002010BD08B5D0F8C1
:10AE5800E0355B689847002008BD000012230B808E
:10AE680000487047B002002004230B800048704758
:10AE7800C202002010B5044C04480A46214600F0DE
:10AE880075FA204610BD00BF88350020CFA90508F7
:10AE98000A4608B50248034900F068FA014808BDA7
:10AEA800E2A90508883500200A4608B50248034982
:10AEB80000F05CFA014808BDF0A9050888350020B3
:10AEC80008B50A4608B9044800E00448044900F0F7
:10AED8004DFA034808BD00BFFBA9050808AA0508E4
:10AEE8008835002008B50A4608B9044800E0044837
:10AEF800044900F03BFA034808BD00BF15AA05083D
:10AF080036AA05088835002010B513460C46C0F847
:10AF18003821C0F83421022280F81121002122466C
:10AF2800FFF779F9002010BD10B50C461346002133
:10AF38002246FFF770F9002010BD10B513460C46E5
:10AF4800C0F89023C0F88C23032280F81121002137
:10AF58002246FFF745F9002010BD10B50C461346F0
:10AF680000212246FFF73CF9002010BD00210423F0
:10AF780010B50A46044680F811310B46FFF74BF925
:10AF88002046FEF7D7FF002010BD0021052310B58D
:10AF98000A46044680F811310B46FFF721F920468E
:10AFA800FEF7C8FF002010BD282303FB0100B0F8FE
:10AFB8008803704790F8C8350B7090F8C9354B7006
:10AFC80090F8CB2590F8CA3503EB02234B8090F814
:10AFD800CD2590F8CC3503EB02238B8090F8CF2554
:10AFE80090F8CE3503EB02239BB2CB80C0F83C31FE
:10AFF800012380F81131704710B591F90030002B0A
:10B00800044601DBCB880BB9802100E00021FFF763
:10B018001BF92046BDE81040FEF78CBF38B50D4639
:10B0280004466B780979012B10D027D3032B51D113
:10B0380090F81231022B28D0032B47D16B889BB98B
:10B0480091B1802910D0FFF7FFF80DE090F8123188
:10B05800022B1AD0032B39D16B88002B3AD149B176
:10B06800802907D0FFF70EF9D4F8E03520469B6811
:10B07800294698472046FFF779FF2BE090F81231D0
:10B08800022B02D0032B21D106E019B3802921D04D
:10B098002046FFF7D9F81DE011F0800F4FF0280384
:10B0A80006D001F07F0103FB010393F81A2103E0A6
:10B0B80003FB010191F87223074B02B101221A60C8
:10B0C800204605490222FFF71FFF03E020462946D4
:10B0D800FFF792FF002038BD800D002038B590F8AA
:10B0E8001231032B04460D460CD10B79012B09D8DC
:10B0F800D0F8E0359B689847EB883BB92046FFF7C6
:10B1080035FF03E020462946FFF776FF002038BDCB
:10B1180073B54B7804460D46092B00F21C81DFE815
:10B1280013F0D10008011A01E4001A0172000A00A4
:10B138001A01C00092004B881A0A013A062A00F246
:10B148000A81DFE812F007001A0027000801080149
:10B1580008010801D4F8E835A0781B680DF106014C
:10B168009847EB88402B014603D094F81231012B05
:10B178003AD10823ADF8063036E0D4F8E035A078A7
:10B188009B6A0DF106019847022343700146C4F8F3
:10B19800EC0529E0DBB2052B00F2DD80DFE803F0E7
:10B1A80003080D12171CD4F8E835A0785B6817E07F
:10B1B800D4F8E835A0789B6812E0D4F8E835A07890
:10B1C800DB680DE0D4F8E835A0781B6908E0D4F80E
:10B1D800E835A0785B6903E0D4F8E835A0789B6986
:10B1E8000DF1060198470146BDF80630002B00F026
:10B1F800B680EA88002A00F0B2809A4228BF1A4630
:10B20800ADF806205CE08B88002B40F0A480CB884A
:10B21800002B40F0A08094F812214B88032A00F0FC
:10B228009A8003F07F05204684F813512946FFF7DA
:10B2380053F82046FFF79AFE0DB1022300E00123E0
:10B2480084F812318BE08978464E0129317100F279
:10B25800828094F81231022B02D0032B7BD108E0B4
:10B26800002962D00121032384F8101184F81231D7
:10B2780013E041B9022384F8123184F810112046F2
:10B28800FFF7E4FD51E094F81011012920464DD054
:10B29800FFF7DCFD317984F810112046FFF7CAFD6D
:10B2A80043E0CA88012A56D194F81231022B02D001
:10B2B800032B50D102E020462B4913E004F5887196
:10B2C80020460FE094F81231023B012B43D8D4F802
:10B2D80014312449002B0CBF0123032341F80C3FF0
:10B2E80020460122FFF710FE39E04B88012B29D0B8
:10B2F800022B34D18B8813F0FF0F30D121691B0A40
:10B30800013B4A68042B0FD8DFE803F0030507095F
:10B318000B00012306E0022304E0032302E00423D8
:10B3280000E0052363F306124A602046FFF71EFE7D
:10B3380015E094F81231023B012B0CD84B88012BF5
:10B348000DD10023C4F81431D4F8E03520469B68A9
:10B3580029469847E9E720462946FFF74DFE002091
:10B368007CBD00BF800D0020880D002030B5C8B11D
:10B378000023DDB20133C41814F8014C002CF8D1B5
:10B388006B1C5B0013800B7003234B70022305E0DA
:10B39800CA545A1CD2B202338C54DBB210F8012BB7
:10B3A800002AF5D130BD00BF70477047704770471D
:10B3B800704770477047000008B5FCF781FA094BE1
:10B3C8005A78187002435A701AB19A7801329A70F2
:10B3D80030B99B78034A012B02D90023537093702C
:10B3E80008BD00BF900D00202DE9F84F394B1A78A1
:10B3F800394B2DED028B22B91A68802392FBF3F3A7
:10B4080000E01B68354A5361354B1A8892B2002A0E
:10B41800FBD0334B00221A80FDF790FD10EE105A36
:10B42800FDF792FD284610EE104A06F06DFC8046A6
:10B438002046894606F068FC41EC100B41EC180BDD
:10B4480008F01EFD57EC106BB0EE480AF0EE680AE3
:10B4580008F016FE32463B46404649465BEC10ABC8
:10B4680006F0A6FC06F086FF9FED1E8A07EE100A7E
:10B47800DFED1D7A57EE087A184C52465B46C4ED4C
:10B48800007A4046494606F093FC06F073FF07EE43
:10B49800900A27EE888A84ED018AFDF767FD84ED1E
:10B4A800020AFDF769FD84ED030AFCF717F90F4B53
:10B4B80062691B68D31A0E4A07EE100A1268F8EE82
:10B4C800C77A93FBF2F3C4ED047A2383BDEC028BB5
:10B4D800BDE8F88FF40D0020102C0020BC370020A8
:10B4E800400D00200000F04200008C421026002091
:10B4F8009C25002007B50420012105F053F84FF4DE
:10B508006043009301238DF8043002238DF8053041
:10B518000448002369468DF806308DF8073004F09A
:10B5280099FC0EBD00080240084B1A684FF47A7364
:10B53800B2FBF3F2064B013A5A60064AF02182F850
:10B54800231000229A6007221A607047D001002059
:10B5580010E000E000ED00E0034B5A6812B15A68B1
:10B56800013A5A60704700BF900D0020024B5860A6
:10B578005A68002AFCD17047900D002030B585B07C
:10B5880004460D4601A85C490A220BF071F95B4B91
:10B598001B78032B10D8DFE803F00205080B01A87D
:10B5A800574907E001A8574904E001A8564901E0B6
:10B5B800564901A80BF046FA04AA131913F80C3CD3
:10B5C8005D19EDB22F2D01D80A3502E0392D01D9C8
:10B5D8000A3DEDB204AB1C194FF6FF7004F80C5C81
:10B5E800FAF728FB0020FAF727FC0DF103050F24D2
:10B5F800204623345A21002315F8012FA4B2FAF764
:10B6080035FCB4F5A57FF3D164205A212C22002300
:10B61800FAF72CFC0023CD205A212C22FAF726FC1D
:10B628000020FAF707FB354B1B78032B62D8DFE8BD
:10B6380003F002284B5601A931480BF003FA0A22FD
:10B6480000212F480CF026FB314A324B1278186043
:10B65800012A06D1304A904201DC01321A602F4A91
:10B6680006E0B0F5FA5FBCBF4FF4FA521A602C4AF4
:10B678001B689342C4BF274B1A602A4B1A682A4B8F
:10B6880020E001A91F480BF0DDF90A2200211D481E
:10B698000CF000FB1E4A254B12781860012A06D1CF
:10B6A8001D4A904201DC01321A601C4A06E0B0F5DE
:10B6B800FA5FBCBF4FF4FA521A60194A1B689342EA
:10B6C80018DD1A4B1A6015E001A90F480BF0BAF9FA
:10B6D8000D4800210A220CF0DDFA154B09E001A9FA
:10B6E8000A480BF0AFF9094800210A220CF0D2FAF7
:10B6F800104B186005B030BD57AA05080F2600206A
:10B70800E025002004260020162C0020CC2500204F
:10B71800F40D0020182600201FA1070080D1F00892
:10B7280050DA110010260020102C0020302C0020A8
:10B738000C2C0020C825002010B50D4B0D4C1A68A4
:10B748000D4821460BF056F90C4B0D481A68214656
:10B758000BF050F90B4B0C481A6821460BF04AF9CC
:10B768000A4B0B481A682146BDE810400BF042B955
:10B778001826002066A00508E0250020302C0020AF
:10B78800042600200C2C0020162C0020C8250020A0
:10B79800CC2500209FED010A704700BF0000000083
:10B7A8009FED010A704700BF000000009FED010AED
:10B7B800704700BF0000000018B1012801D1034BF9
:10B7C80000E0034B1868FDF73DBD00BF00260020D0
:10B7D8001026002010B9034B18687047024B1868F0
:10B7E800704700BF182600201026002010B9034B10
:10B7F80018687047024B1868704700BF302C00204B
:10B808000026002008B54FF49570FBF77BFF40F247
:10B818006523C31A584240EB030008BD08B5C6208B
:10B82800FBF770FF40F28D13C21A504240EB020042
:10B8380008BD4FF4957040F26521FBF755BFC6204F
:10B8480040F28D11FBF750BFDCE760EEA00AB7EEBF
:10B85800007AF0EE606A70EE077A40EE006A47EE12
:10B86800A70A36EEC77A08B5C7EE200A10EE900A86
:10B8780006F04AFA0022084B06F09AFA0022074B13
:10B8880006F0E4F806F076FD07EE900AFDEEE77A9A
:10B8980017EE900A9F3008BD000059400000E03FB5
:10B8A80038B52DED028BF7EE008AB0EE608A70EEA7
:10B8B800288A10EE900A28EE088A06F025FA08EE83
:10B8C800A88A00220F4B06F073FA044618EE100AF5
:10B8D8000D4606F019FA02460B462046294606F0A0
:10B8E80091FB0022084B06F0B1F806F043FD07EE85
:10B8F800900AFDEEE77A17EE900A7730BDEC028BDE
:10B9080038BD00BF000069400000E03F2DE9F04F5E
:10B91800894F2DED068B97E80F0091B00CAC1037CE
:10B9280084E80F000FCF05AE0FC697E807004FF663
:10B93800FF7386E807009F2077216422F7F71FFE30
:10B94800A020772164224FF6FF73F7F718FE9E2098
:10B95800772164224FF6FF73F7F711FE9F207621B7
:10B9680064224FF6FF73F7F70AFE4FF6FF7378214C
:10B9780064229F20F7F703FE0020F9F71AFA9F20A8
:10B9880077216522FAF798F90C349F2077216422F1
:10B99800FAF792F90DF12C0A0394F7EE009A4FF09A
:10B9A8000F0B00E04D460AF1040AF7EE008A9AED03
:10B9B800009A0024B0EE68AA01E0B846354618EEB1
:10B9C800900A06F0A1F95AA3D3E9002306F0F0F98A
:10B9D80006F0D0FC08EE900A38EEE98AB0EE490A83
:10B9E800F0EE480AFFF731FFB0EE490AF0EE480AD8
:10B9F8000646FFF755FFB2B2074683B22CB9104688
:10BA080019460F22F9F7A0FA06E0A8B21FFA88F142
:10BA1800CDF800B0FAF79AF80134B4F5967FCCD196
:10BA28003D46F7EE008A002401E045464E4618EEF2
:10BA3800900A06F069F93EA3D3E9002306F0B8F9A5
:10BA480006F098FC08EE900A39EEE88AB0EE490A4A
:10BA5800F0EE480AFFF7F9FEB0EE490AF0EE480AA0
:10BA68008146FFF71DFF1FFA89F2804683B22CB981
:10BA7800104619460F22F9F767FA05E0B0B2A9B2E5
:10BA8800CDF800B0FAF762F80134B4F5967FCCD15E
:10BA9800039B9A4586D104AD0DF12C0B4FF0000A9B
:10BAA80001E0B846B146043595ED009AF7EE008AF4
:10BAB800002401E0B846B14618EE900A06F024F9D1
:10BAC8001BA3D3E9002306F073F906F053FC08EE34
:10BAD800900A38EECA8AF0EE490AB0EE480AFFF733
:10BAE800B4FEB0EE480AF0EE490A0646FFF7D8FE63
:10BAF800B2B2074683B22CB9104619462246F9F766
:10BB080023FA07E01FFA89F01FFA88F1CDF800A0A0
:10BB1800FAF71CF80134B4F5C87FCBD15D45C0D124
:10BB280011B0BDEC068BBDE8F08F00BFAFF300800D
:10BB3800295C8FC2F528F03F34A50408121A06EED6
:10BB4800902A081AB8EEE67A06EE900AF8EEE67A37
:10BB580008B5C7EE277A17EE900A06F0D5F807A3BE
:10BB6800D3E9002306F024F90022034B05F06EFF09
:10BB780006F0B8FB08BD00BF0000E03F0000000071
:10BB880000F073408A1A06EE902A081AB8EEE67A90
:10BB980006EE900AF8EEE67A08B5C7EE277A17EEB1
:10BBA800900A06F0B1F807A3D3E9002306F000F9DC
:10BBB8000022034B05F04AFF06F094FB08BD00BFC6
:10BBC8000000E03F0000000000E0684070B5064655
:10BBD8000D460024610704D5A0B231462A46F9F77C
:10BBE800B3F90134B4F5A07FF4D170BD70B5064641
:10BBF8000D460024600704D5A1B230462A46F9F75D
:10BC0800A3F90134C82CF5D170BD114B11481B782C
:10BC18001149124A0068012B114B09D112680860BA
:10BC28001A60104B1A68104B1A60104B1A680CE017
:10BC38001268D2011A600B4B1A680B4BD2011A60BA
:10BC48000A4B1A68C0010860D201094B1A60704794
:10BC5800F40D00201826002010260020302C00208B
:10BC6800002600200C2C00209C250020EC2500201C
:10BC7800282C0020014B1868FDF7E4BA1026002094
:10BC880008B5FFF7C2FFBDE80840F3E770B500212B
:10BC98000A222748274D284E284C0BF0FBFF00218D
:10BCA8000A22286026480BF0F5FF00210A2230609E
:10BCB80024480BF0EFFF00210A22206022480BF0F5
:10BCC800E9FF224B326818602B682149D31A06EE27
:10BCD800903A2368B8EEE67A06EE903AF8EEE67AFD
:10BCE800C7EE277AFCEEE77A17EE903A9AB20B8005
:10BCF800531C07EE903AB8EEE77ADFED167A67EE56
:10BD0800277A154BFCEEE76A16EE901A8AB206EE11
:10BD1800902AB8EEE67A198077EEC77AF5EEC07AFF
:10BD2800F1EE10FA01DD01321A80BDE87040A7E794
:10BD3800E025002018260020302C00200C2C0020A4
:10BD480004260020162C0020CC250020C825002021
:10BD5800FC3900200000803D903A00200022F0B518
:10BD68001346202603254FF02C0C00E02646303ED3
:10BD7800F6B217460132092E10F8014B0AD897FB84
:10BD8800F5F605FB16772FB9CE1801F803C07470C5
:10BD9800023301E0CC540133092AE7D12022CA54E6
:10BDA800CB1848225A707A229A700022DA70F0BDB5
:10BDB800F0B51F46144B1E78012E8DB005460C4673
:10BDC80020D0A6F1030CDCF1000646EB0C06CEB938
:10BDD8000E4908A80AF00EFE08A86946FFF7BEFF3C
:10BDE8000B496A4604A80AF005FEBDF84800F9F7B1
:10BDF80021FF3846F9F734FF2846214604AA33467E
:10BE0800FAF752F80DB0F0BDA425002066A0050889
:10BE1800A8A7050810B501210446F9F7BBF8014B9E
:10BE28001C8110BD900D002008B50021C620FBF72D
:10BE38005BFC4FF495700021BDE80840FBF754BC4B
:10BE4800014B9F221A817047900D00200020014667
:10BE5800C82240F23F13F9F7B1B907B50DF1070051
:10BE6800FEF775FE9DF807000EBD08B5FFF7F5FF54
:10BE78000028FBD108BD30B5044687B010EE100A83
:10BE88000D4605F041FF02460B4601A805490AF098
:10BE9800B1FD2046294601AA0023FAF705F807B0A4
:10BEA80030BD00BF61AA050808B5084803F034FA98
:10BEB8000648022103F001FB0028F9D0034803F0EB
:10BEC80057FA07EE900AB8EE670A08BD002001404D
:10BED80010B52DED028B9FED098A1924FFF7E4FFB9
:10BEE800013CE4B238EE008A002CF7D19FED040A39
:10BEF80028EE000ABDEC028B10BD00BF0000000058
:10BF0800ACC868392DE9F04F2DED068B8E4B8F4C60
:10BF18008F495D695F68C1B00646324638A893ED1F
:10BF2800038AD3ED04AAD3ED028A93ED00AA93ED18
:10BF3800069A0AF05FFDA06805F0E6FE02460B4689
:10BF480028A884490AF056FDE06805F0DDFE02469F
:10BF58000B462CA880490AF04DFD1AEE900A05F010
:10BF6800D3FECDE90801DDE908237C4930A80AF0B1
:10BF780041FD284605F0C8FECDE90401DDE90423AA
:10BF8800774934A80AF036FD18EE900A05F0BCFE91
:10BF98008046894642464B46724910A80AF02AFD57
:10BFA80018EE100A05F0B0FE82468B4652465B46F4
:10BFB8006D4914A80AF01EFD1AEE100A05F0A4FE39
:10BFC800CDE90A01DDE90A23684918A80AF012FD3B
:10BFD800384605F099FE54A3D3E90023CDE90601BC
:10BFE80005F0E6FE02460B461CA861490AF002FD70
:10BFF80049EC118B4BEC10AB08F09EF84AA3D3E93F
:10C00800002351EC100B05F0D3FE02460B4624A882
:10C0180058490AF0EFFC19EE100A05F075FE0246C1
:10C028000B4620A854490AF0E5FCD4ED047AFDEE4D
:10C03800E77A0CA817EE902A50490AF0DBFCB5EE17
:10C04800C08AF1EE10FADFED4E9A37D5304605F08A
:10C0580049FE37A3D3E9002305F0AAFEF1EE487A9A
:10C06800044617EE900A0D4605F04EFE02460B46B2
:10C078002046294605F09CFE02460B462EA1D1E932
:10C08800000105F0BFFF06F075F99FED3E7A07EE57
:10C09800900AF4EEC77AF1EE10FAC6BFC7EEA97A95
:10C0A800394C3A4CF4EEE97AF1EE10FA38DD9FEDAE
:10C0B800347A374D374CC7EE877A76E020A3D3E938
:10C0C80000235046594605F073FE044630460D4697
:10C0D80005F008FE16A3D3E9002305F069FE024621
:10C0E8000B462046294605F08DFF06F043F907EE7A
:10C0F800900AB7EE007AF4EEC77AF1EE10FA46BF6E
:10C1080067EEA97A244C254CF4EEE97AF1EE10FAA0
:10C118004ADD9FED1B7A224D224CC7EE877A44E018
:10C128001B4D42E0AFF300806666666666A64C402B
:10C138001F85EB51B81E1940000000A2941A6D42E9
:10C148000000000080842E41AC390020BC3700205C
:10C1580083AA05088DAA050898AA0508A3AA0508B0
:10C16800ADAA0508B7AA0508C3AA0508CFAA0508F5
:10C17800DAAA0508E5AA0508F0AA0508FCAA050830
:10C1880000007A440024744972AA05086FAA0508B9
:10C1980013AA05087BAA050878AA050875AA050840
:10C1A8007EAA050880AA0508954D17EE900A05F0A5
:10C1B800ABFD2A46CDE900013CA8924902940AF059
:10C1C80019FC914B1A68914B1B689642CCBF002210
:10C1D80001229E428E4BD8BF0022DA608D4B1B781D
:10C1E800082B40F09C800220F9F726FE4FF6FF70DE
:10C1F800F9F736FD1F20F9F71DFD19210023864A9E
:10C208002D20F9F751FE4FF6FF70F9F729FD0020B0
:10C218000024F9F70FFD0F20B42132464FF6FF73C3
:10C228000094FFF7C5FD0F206E2128AA2346F9F7D1
:10C238003BFEB0206E210DEB00022346F9F734FED9
:10C248000F20382118AA2346F9F72EFEB0203821EE
:10C258001CAA2346F9F728FE0F205C2130AA2346A2
:10C26800F9F722FEB0205C2134AA2346F9F71CFE18
:10C278000F204A2110AA2346F9F716FEB0204A21BA
:10C2880014AA2346F9F710FE0F209B2120AA234663
:10C29800F9F70AFE0F2084213CAA2346F9F704FE89
:10C2A800B020842124AA2346F9F7FEFD5B4B1B68C6
:10C2B800B3F57A7FCCBF4FF4FC604FF47840F9F7C0
:10C2C800CFFC0023A0209B210CAAF9F7EDFD544BCD
:10C2D8001B78012B08D14FF4FC60F9F7C1FC4FF42F
:10C2E8008C7002214F4A07E04FF6E070F9F7B8FC6E
:10C2F8004D4A4FF48C7002210023F9F7D5FD002038
:10C30800F9F7AEFC4FF4FC60F9F794FCFFF7E0FD99
:10C318000F20DC21FFF7AFFD1F20F9F7A1FC3D4BF3
:10C328001B789A1FD2B2012A02D90B2B40F0258222
:10C338003E4B1B78023B052B00F21F82DFE813F00F
:10C3480006007E00E2003B01DE015801DFED387A8D
:10C358002AEE27AA1AEE100A05F0D6FC9DED060B68
:10C368008046894607F08CFD404653EC102B494621
:10C3780005F01EFD1EA3D3E9002305F067FB05F0B9
:10C38800B1FF9DED060B044607F07AFE404653ECDC
:10C39800102B494605F00CFD02460B4616A1D1E9C3
:10C3A800000105F051FB05F09DFF4FF6E073009387
:10C3B800054600230520DC213246FFF7F9FC144B23
:10C3C800DB6853B11B4B18881B4B4FF4784719880F
:10C3D8000097A2B2ABB2F9F7B9FB164B1C60164B2B
:10C3E8004FF6E0701D60F9F725FCC6E1AFF3008059
:10C3F8000000000000E063400000000000C05D4055
:10C408007EAA050809AB0508302C00201826002054
:10C41800900D0020A425002016AB05084C1A00201A
:10C42800F40D002081A9050885A90508242C002001
:10C438000000C842F83700209C3A0020A04B18683A
:10C44800A04B9FEDA19A19683246FFF777FBF4EEEF
:10C45800498AF1EE10FAC8BFF0EE498AF5EE408A33
:10C46800DFED9A7AF1EE10FA48BFF0EE678AF4EE43
:10C47800C98AF1EE10FA04461ED8F4EEE78AF1EE06
:10C4880010FA19DBFDEEE88A002018EE902A4FF426
:10C49800FA71FFF777FB8E4BDB68054653B18D4B7E
:10C4A80018888D4B4FF6FF7719880097A2B2ABB268
:10C4B800F9F74CFB884B1D60B4EE498ADFED827AB0
:10C4C800F1EE10FAC8BFB0EE678ADFED847AB4EEF9
:10C4D800678AF1EE10FA48BFB0EE678AB4EEC98AEF
:10C4E800F1EE10FA00F24981B4EEE78AF1EE10FAA3
:10C4F800C0F24381BDEEC88A794818EE102A4FF47D
:10C50800FA71AEE06E4B18686E4B32461968FFF749
:10C5180015FBF5EEC0AAF1EE10FA044627DDDDE9B9
:10C52800080159A3D3E9002305F0B4FEF8B158A3D4
:10C53800D3E90023DDE9080105F03AFC0B46024681
:10C548006849002005F080FA05F0CCFE604BDB68F6
:10C55800054653B15F4B18885F4B4FF6FF77198834
:10C568000097A2B2ABB2F9F7F1FA5B4B1D60DDE9B7
:10C57800040149A3D3E9002305F0AAFE002800F02E
:10C58800FC80DDE9040140A3D3E9002305F082FE25
:10C59800002800F0F28042A3D3E90023DDE904017A
:10C5A80005F006FC02460B4600204F4905F04CFA00
:10C5B80005F098FE57E0424B1868424B324619681E
:10C5C800FFF7BCFA38A3D3E900230446DDE90A01E2
:10C5D80005F07EFE50B19DED0A0B07F035FE0022F6
:10C5E80051EC100B414B05F0E3FBB1E0C825B2E07C
:10C5F8002FA3D3E90023DDE9060105F0D9FB2EA31B
:10C60800D3E9002305F0FEFC05F0B4FE2C4B08EE40
:10C61800100A18682B4B32461968FFF78FFADFEDBE
:10C62800347A4AEE677A2A4BFDEEE77ADB6817EE32
:10C63800905A044625EAE57553B1264B1888264BCF
:10C648004FF6FF7719880097A2B2ABB2F9F77EFAD6
:10C65800BDEEC88A204B18EE102A1D606FF0B3009B
:10C66800B421FFF78FFA1A4BDB68054653B1194B13
:10C678001888204B4FF4FC6719880097A2B2ABB218
:10C68800F9F764FA1B4B75E09A9999999999B93F0A
:10C698000000000000409F409A9999999999B9BF64
:10C6A8000000000000408F4089B5F81400E3693F9E
:10C6B80000000000008076401F85EB51B81E19402D
:10C6C80018260020302C00200000FA43000000004B
:10C6D800900D0020F83700209C3A00200000FAC393
:10C6E8000CFEFFFF0000694000005940000054C0E4
:10C6F80000004843E83500200000C8425FED027A98
:10C70800B4EE679AF1EE10FAC8BFB0EE679AB4EECD
:10C71800E79AF1EE10FA30D8214B1868214B3246CF
:10C728001968FFF70BFA044619EE100A05F0ECFA3F
:10C7380041EC100B07F088FD00221B4B51EC100B4D
:10C7480005F036FB02460B460020184905F07CF937
:10C7580005F0C8FD0546164BDB6853B1154B188824
:10C76800154B4FF6FF7719880097A2B2ABB2F9F7CD
:10C77800EDF9114B1D600F4B1C60104B1B78022B01
:10C7880009D043B14FF6FF7300930520DC213246F0
:10C798000023FFF70DFB41B0BDEC068BBDE8F08F21
:10C7A80018260020302C0020000059400000694065
:10C7B800900D0020F83700209C3A0020242C0020FF
:10C7C80010B54FF4C770FAF79DFFDB2805D14FF479
:10C7D800C870FAF797FF84B219E041F2E1042146E4
:10C7E80044F20100FAF780FF44F20100FAF78AFFE9
:10C7F800A04214BF80244FF4007421B24FF4C870D3
:10C80800FAF772FF4FF4C770DB21FAF76DFF204685
:10C8180010BD024B00221A60704700BF043600208A
:10C8280070EEA10A88B030EE010A08B0704770EEC9
:10C83800E10A88B030EE410A08B07047F0EE407A5D
:10C8480020EEA10A60EE810A47EEA10A88B017EE31
:10C85800810A08B07047D0B561EEA17A41EE017A3D
:10C868002DED048B17EE900A88B0B0EE409AF0EEEA
:10C87800609AF0EE418AB0EE618A05F045FA00222E
:10C88800002306460F4605F0FBFCE8B969EE887AF6
:10C8980049EE287A29EE088A17EE900A05F034FA4C
:10C8A80032463B4605F0AEFB19EEA88A05F062FD5C
:10C8B800044618EE100A05F027FA32463B4605F002
:10C8C800A1FB05F057FD01E00448044600EE900A7C
:10C8D80000EE104A08B0BDEC048BD0BD0050C34731
:10C8E800F0B58D4B2DED068B93ED001AD3ED011AA3
:10C8F8008FB0F0EE408AB0EE608A8DED060ACDED7D
:10C90800070A30EE410A70EEE10A38EE811A78EE35
:10C91800211A8DED0C1ACDED0D1A8DED0A0ACDED0B
:10C928000B0AFFF798FF8DED040ACDED050A04AA5E
:10C9380092E8030008AB83E80300DDED099A9DED5A
:10C9480008AA69EEA97A4AEE0A7A17EE900A05F063
:10C95800DBF941EC100B07F0FDFC51EC100B05F076
:10C9680009FD09EE100A19EE900A05F0CDF9044602
:10C978001AEE100A0D4605F0C7F945EC104B41ECCC
:10C98800110B07F0D9FB51EC100B05F0F3FC68EE26
:10C99800087A48EEA87AB1EE48AAC8EEA79A5F4B83
:10C9A8005F4D5A691B8B6860EA612B8404468AEEE6
:10C9B80027AA85ED009A19EE100AC5ED028A85EDC1
:10C9C800038AC5ED049A85ED05AA05F09DF94CA3E7
:10C9D800D3E9002305F07CFCDFED527A002818BF6C
:10C9E800B0EE679AB7EE007A79EE077A37EE497AB1
:10C9F8004D4BC7EE877A1B78033BC5ED067A042BAF
:10CA080071D8DFE803F0032738664F0018EE100AE4
:10CA180005F07AF9044618EE900A0D4605F074F907
:10CA280006460F4647EC116B45EC104B07F084FBAC
:10CA380035A3D3E9002351EC100BCDE9004505F0EF
:10CA4800B7F93246CDE902013B463849384809F082
:10CA5800D1FF48E019EE900A05F056F904461AEE9F
:10CA6800100A0D4605F050F92246CDE900012B4683
:10CA78002F4830492AE019EE100A05F045F941EC33
:10CA8800100B07F0E1FB00222B4B51EC100B05F0CB
:10CA98008FF905F06FFC05F037F902460B4624487C
:10CAA80026491EE019EE100A05F02EF90646204622
:10CAB8000F4605F029F916A3D3E9002305F078F904
:10CAC800CDE900011A481E4932463B4609F092FF5B
:10CAD80009E017EE900A05F017F902460B461448CC
:10CAE800184909F087FF124C00230220CA21224668
:10CAF800F9F7DAF9002323700FB0BDEC068BF0BD0F
:10CB0800AE47E17A14AEEF3F6666666666A64C40AD
:10CB1800F6285C8FC2A54C402C360020BC3700207C
:10CB2800AC390020A4707D3F242C002035AB0508CB
:10CB3800C83500204FAB0508000034C05FAB0508BE
:10CB480071AB05088DAB050800B560EEA07A40EE24
:10CB5800007A2DED028B17EE900A87B0B0EE408A6E
:10CB6800F0EE608A8DED020ACDED030A05F0CCF8EF
:10CB780041EC100B07F0EEFB51EC100B05F0FAFB43
:10CB8800DFED117A07EE100A78EEA78A38EE078AE9
:10CB980068EEA87A48EE087AC7EE277A17EE900A68
:10CBA80005F0B2F841EC100B07F0D4FB51EC100B78
:10CBB80005F0E0FB00EE900A20EE880A60EEA80A75
:10CBC80007B0BDEC028B00BD00000000F0B52DEDF4
:10CBD800028BDFED3A1A3A4B8DB030EEA17AF0EEC7
:10CBE800407AB7EE001A8DED020A83ED001A30EE96
:10CBF800010AC3ED011A31EE671A71EEE01ACDEDA4
:10CC0800030AF0EE470A8DED077A8DED081ACDED8F
:10CC1800091A8DED060AFFF71EFE8DED000ACDED0F
:10CC2800010A9DE8030004AB83E803009DED058A33
:10CC3800DDED048A68EE087A48EEA87A17EE900AC5
:10CC480005F062F841EC100B07F084FB18EE100AAF
:10CC580057EC106B05F058F8044618EE900A0D468C
:10CC680005F052F845EC104B41EC110B07F064FA53
:10CC78003946304655EC104B05F07CFB05F044F87E
:10CC880041EC100B07F05AFA002251EC100B0D4B37
:10CC980005F08EF805F06EFB29460646204605F09D
:10CCA80069FB00EE900AF6EE007A60EEA70A00EE45
:10CCB800106A0DB0BDEC028BF0BD00BF0000000093
:10CCC800043A00200000E03FF0EE407A86B020EE03
:10CCD800200A67EE810A06B070472DE9F04F2DED66
:10CCE800028B85B0FCF72AF910EE105AFCF72CF9E4
:10CCF800284610EE104A05F007F880462046894677
:10CD080005F002F841EC100B41EC180B07F0B8F8ED
:10CD180057EC106BB0EE480AF0EE680A07F0B0F96D
:10CD280032463B46404649465BEC10AB05F040F8BE
:10CD380005F020FB9FED138A07EE100ADFED127A4B
:10CD480057EE087A114C5B46C4ED007A52464046CD
:10CD5800494605F02DF805F00DFB07EE900A27EE81
:10CD6800888A04AB84ED018A94E8030003E9030090
:10CD7800DDED030A9DED020A05B0BDEC028BBDE8AE
:10CD8800F08F00BF0000F04200008C42943A00206F
:10CD980030B53F4B2DED088BD3ED008AD3ED019ACA
:10CDA8003C4BD3ED00AAD3ED01BA3B4B93ED008A7F
:10CDB80093ED019A394B93ED00AA93ED01BA38EE41
:10CDC800EA0A79EEEB0A38EE4A1A79EE4B1A93B072
:10CDD8008DED0A0ACDED0B0A8DED0C1ACDED0D1A6D
:10CDE800FFF72CFD8DED000ACDED010A9DE803004B
:10CDF8003AEE6A0A7BEE6B0A04AB38EE681A79EEF3
:10CE0800691A83E803008DED081ACDED091A8DED36
:10CE18000E0ACDED0F0AFFF711FD8DED000ACDEDDD
:10CE2800010A9DE8030006AB83E803009DED040AB0
:10CE3800DDED050A9DED061ADDED071AFFF70BFD7E
:10CE48008DED000ACDED010A9DE8030002AD85E8ED
:10CE58000300134B9DED021A93ED000AD3ED010A6E
:10CE6800DDED031AFFF7EAFC8DED000ACDED010AAE
:10CE78009DE8030012AB03E903006C46DDED110ADF
:10CE880085E803009DED100A13B0BDEC088B30BD9A
:10CE9800C035002018360020883A0020183A0020B3
:10CEA800E0370020F7EE007A77EEC07A20EE022A0B
:10CEB80020EE210A07EEA00AF0EE420A47EE810AA8
:10CEC80088B008B070472DE9F0432DED028B924BE6
:10CED8001B78012B89B08146884646D14FEAC009A4
:10CEE80001291FFA89F92BD809F58065A8B2FAF744
:10CEF8004DFC8A4C0435A8B284ED000AFAF746FCCA
:10CF080009F58645A8B284ED010AFAF73FFC844C7E
:10CF1800043584ED000AA8B2FAF738FCA9F5FC40FC
:10CF280084ED010A80B2FAF731FC7E4CA9F5FA408B
:10CF3800FC3884ED000A80B2FAF728FC84ED010A77
:10CF480008F1FF385FFA88F8B8F1010F00F2DF80C6
:10CF5800A9F57C5080B2FAF719FC734CA9F57A59F7
:10CF680084ED000AA9F17C09CBE0022B40F0CF80C8
:10CF78006E4B6F4A1B68012992ED007A00F2AC8073
:10CF880007EE900AF8EE676A07EE903A46EE877A5F
:10CF9800BDEEE77A17EE104AA4B207EE104A04F184
:10CFA8008005ED00B8EE478AADB2284637EEC88A4C
:10CFB800FAF7ECFB0435A8B204F50665EE008DED32
:10CFC800020AFAF7E3FBB6B230468DED030AFAF728
:10CFD800DDFB043604F58257B0B28DED040AFE007D
:10CFE800FAF7D4FBB6B230468DED050AFAF7CEFB58
:10CFF8000436B0B281348DED060AE400FAF7C6FBB8
:10D00800A4B220468DED070AFAF7C0FB434E04345C
:10D01800A0B286ED000AFAF7B9FB6C1CE400A4B2D2
:10D02800204686ED010AFAF7B1FB3D4D0434A0B263
:10D0380085ED000AFAF7AAFB7C1CE400A4B220469E
:10D0480085ED010AFAF7A2FB364F0434A0B287ED4A
:10D05800000AFAF79BFBD6ED001A96ED012ADDEDE2
:10D06800020AF0EE408A87ED010A9DED031AB0EE40
:10D07800480AFFF717FF8DED000ACDED010A9DE87C
:10D088000300D5ED001A95ED012AB0EE480ADDED52
:10D09800040A86E803009DED051AFFF703FF8DEDEE
:10D0A800000ACDED010A9DE80300D7ED001A85E8D6
:10D0B8000300B0EE480ADDED060A9DED071AB0EE52
:10D0C800682AFFF7EFFE8DED000ACDED010A9DE815
:10D0D800030087E803006C4608F1FF385FFA88F818
:10D0E800B8F1010F13D809F5C1594FEAC9091FFA58
:10D0F80089F94846FAF74AFB0B4C84ED000A09F116
:10D1080004091FFA89F0FAF741FB84ED010A09B016
:10D11800BDEC028BBDE8F083B5010020883A002001
:10D1280018360020183A0020C0350020A02500201D
:10D13800D82500202DE9F04F2DED048B734BC7B097
:10D1480005464FF476701C78FAF7DCFA06464FF479
:10D158007570FAF7D7FA07464FF47470FAF7FAFAC7
:10D16800012C14BF10240024C0B2032D1D9040F0E0
:10D17800A080674A674924A809F03CFCC1B224A8EA
:10D18800FDF7E4FC33463A46634924A809F032FC2B
:10D19800C1B224A8FDF7DAFC604A5E4924A809F068
:10D1A80029FCC1B224A8FDF7D1FC002C14BFD8205B
:10D1B800C820FAF7CFFA0746002C14BFDC20CC2091
:10D1C800FAF7C8FA0646002C14BFE020D020FAF778
:10D1D800C1FA8046002C14BFE420D420FAF7BAFA2A
:10D1E800F31B06EE903AB8EEE67A06EE908AF8EE71
:10D1F800E67A3346C7EE277A3A4601904849CDF891
:10D20800008024A8FDEEE77ACDED027A09F0F2FB62
:10D21800C1B224A8FDF79AFC424A3E4924A809F065
:10D22800E9FBC1B224A8FDF791FCE820FAF792FACD
:10D238000746EC20FAF78EFA0646F020FAF78AFA43
:10D248008046F420FAF786FAF31B07EE903A06EECA
:10D25800908AB8EEE77AF8EEE67A3A46C7EE277A89
:10D2680001902F49CDF80080334624A8FDEEE77AD7
:10D27800CDED027A09F0BEFBC1B224A8FDF766FC29
:10D288001D9A022A08D124A8274909F0DBFB24A803
:10D298001421FDF75BFC29E11D9B012B40F0228145
:10D2A80024A8224909F0CEFB24A81021FDF74EFC42
:10D2B80003E01D9A012A40F01581002C14BFD820E4
:10D2C800C820FAF747FA1B90002C14BFDC20CC20AA
:10D2D800FAF740FA0646002C14BFE020D020FAF7EF
:10D2E80039FA1B9B1C90F61A06EE906AB8EEE67A9D
:10D2F80006EE900AF8EEE67A1026C7EE277A0024A2
:10D30800FDEEE77ACDED1F7AE7E000BFF40D0020CF
:10D318009DAB050898AB0508A7AB0508B4AB050895
:10D32800BAAB050804AC05080AAC05081FAC05082B
:10D338001C9B1B9A2046012103FB042AFFF7C3FD0F
:10D34800944B954A18681768D3ED018A92ED019AB3
:10D35800924B934AD3F80090D3ED019A1368012DAC
:10D36800209392ED018A7ED1F5EEC08AF1EE10FA93
:10D3780054BF4FF0000C4FF0010CB5EEC09ABCF151
:10D38800000F0CBF4FF02B084FF02D08F1EE10FAEC
:10D3980054BF4FF0000E4FF0010EF5EEC09ABEF1EB
:10D3A800000F0CBF2B262D26F1EE10FA54BF0021DA
:10D3B8000121B5EEC08A00290CBF4FF02B0B4FF0AE
:10D3C8002D0BF1EE10FA54BF00220122002A0CBFE7
:10D3D8002B232D231E93BCF1000F01D0F1EE688A98
:10D3E800BEF1000F01D0B1EE499A09B1F1EE699A88
:10D3F8000AB1B1EE488A04F087FCCDE9000118EEC5
:10D40800900ACDF8088004F07FFCCDE90401384685
:10D4180004F07AFCCDE9060119EE100A089604F02A
:10D4280073FCCDE90A01484604F06EFCCDE90C0115
:10D4380019EE900ACDF838B004F066FCCDE9100179
:10D44800209804F061FC1E9ACDE9120118EE100A2A
:10D45800149204F059FC5246CDE9160124A851490A
:10D4680009F0C8FA2FE0022D2ED1FFF791FC8DEDBF
:10D47800220ACDED230A22AB93E8030046AB03E969
:10D488000300DDED457AF5EEC07AF1EE10FA449826
:10D4980005D5F1EE677A17EE906A2D2702E017EEB0
:10D4A800906A2B2704F030FC02460B463046CDE943
:10D4B8000023029704F028FC5246CDE9040124A871
:10D4C800394909F097FAC6B224A83146FDF73EFB60
:10D4D8000120FEF74BF80134A4B21F9BA342BFF60C
:10D4E80027AF70E11D9A022A40F06D81E820FAF713
:10D4F80031F91B90EC20FAF72DF90646F020FAF7DF
:10D5080029F91B9B1C9006EE900AF61AB8EEE68ADB
:10D5180006EE906AF8EEE67A002C14BFD820C820F0
:10D52800C7EE887AFDEEE77ACDED1E7AFAF712F9A2
:10D538000646002C14BFDC20CC20FAF70BF907466E
:10D54800002C14BFE020D020FAF704F9BF1B07EE27
:10D55800100A06EE907AF8EEC77AB8EEE67A1B9AC9
:10D568001F9087EE277A931B012D06EE903ABDEEA9
:10D57800C77A88EE278A0D4B8DED207AB8EEE67AC9
:10D5880087EE277A83ED007A094B83ED008A40F015
:10D59800D0808FE0883A002018360020183A002002
:10D5A800C035002030AC05086BAC0508A02500206C
:10D5B800D82500201F9A002102FB046220462192F0
:10D5C800FFF781FC95ED018AD8ED018AB5EEC08A96
:10D5D800F1EE10FA54BF4FF0000C4FF0010CF5EECD
:10D5E800C08A9AED019ABCF1000F0CBF2B272D279A
:10D5F800F1EE10FA54BF4FF0000E4FF0010EB5EEE9
:10D60800C09ABEF1000F0CBF4FF02B0B4FF02D0B43
:10D61800F1EE10FA54BF002101212868D8F80090D3
:10D62800DAF8003000290CBF2B222D22BCF1000FA4
:10D6380001D0B1EE488ABEF1000F01D0F1EE688A40
:10D6480009B1B1EE499A19921A9304F05DFBCDE93C
:10D65800000118EE100A029704F056FBCDE9040108
:10D66800484604F051FBCDE9060118EE900ACDF8C2
:10D6780020B004F049FB1A9BCDE90A01184604F0D2
:10D6880043FB199ACDE90C0119EE100A0E9204F029
:10D698003BFB219ACDE910014F4924A809F0AAF9CA
:10D6A800C1B224A8FDF752FA01340120FDF75EFF4C
:10D6B800A4B205E0494DDFF83481DFF834A1002435
:10D6C800209BA342BFF676AF0024454D2DE01C9B5E
:10D6D8001B9A2046022103FB0426FFF7F4FB95ED75
:10D6E800018AB5EEC08AF1EE10FA286803D5B1EECA
:10D6F800488A2D2700E02B2704F006FBCDE900011E
:10D7080018EE100A029704F0FFFA3246CDE9040138
:10D71800344924A809F06EF9C1B224A8FDF716FA15
:10D728000120FDF723FF0134A4B21E9BA342CEDAE9
:10D7380049E0022D43D046E01C9B1B9A012120465C
:10D7480003FB0425FFF7BFFBFFF722FB8DED220A41
:10D75800CDED230A22AB93E8030046AB03E90300AF
:10D76800DDED457AF5EEC07AF1EE10FA449806D56B
:10D77800F1EE677A17EE908A4FF02D0903E017EE65
:10D78800908A4FF02B0904F0BFFA06460F46404630
:10D79800CDE90067CDF8089004F0B6FA2A46CDE93D
:10D7A8000401104924A809F025F9C1B224A8FDF7FD
:10D7B800CDF901340120FDF7D9FEA4B200E0002420
:10D7C8001E9BA342B8DA084B1D9A1A7047B0BDECED
:10D7D800048BBDE8F08F00BF7FAC0508883A0020B5
:10D7E800C0350020ADAC0508B50100201836002072
:10D7F800183A0020F0B52DED028B04468DB00028B4
:10D8080000F0D480724B18890419A4B222B2002AFD
:10D8180005DB40F23F139A42C8BF1C4600E00024D3
:10D82800F7F7A6FBA0B24EF29C71F7F7B3FB684B73
:10D838001C81684B186804F067FA5FA3D3E90023DA
:10D8480004F0B6FA04F096FD634B1860634B1B783E
:10D858000A2B054624B23DD107EE104AF8EEC77AE6
:10D8680017EE900A04F050FA5D4B064618680F460A
:10D8780004F038FA02460B4651A1D1E9000104F040
:10D88800C1FB02460B463046394604F091FA06467B
:10D8980028460F4604F038FA02460B463046394609
:10D8A80004F086FA00224F4B04F0ACFB04F062FD52
:10D8B80004F02AFA02460B4604A84B4909F09AF8E4
:10D8C8000020F8F7B9FA0520D72104AA0023F8F7B1
:10D8D800EBFA6BE0454B1888604304F003FA3AA36F
:10D8E800D3E9002304F08EFB04F044FD404B08EE1E
:10D8F800100A1B68FCEEC87A07EE103A17EE905A29
:10D90800F8EEC77A3B4B68EE277A1B68FDEEE77A9C
:10D91800ADB217EE906A28460121F618FFF7D3FA40
:10D92800FFF736FA8DED020ACDED030A02AC94E852
:10D93800030008AB83E80300681C80B20121FFF7ED
:10D94800C2FAFFF725FA8DED020ACDED030A94E835
:10D9580003000CAB07EE105A03E90300B8EEC70A40
:10D96800DDED080A38EE400A9DED091ADDED0A1AC8
:10D978009DED0B2AFFF796FA8DED020ACDED030A0D
:10D9880094E8030006AB83E803004FF6FF730093A7
:10D9980005200023DC213246FEF70AFA164B9DEDDE
:10D9A800060A1878DDED070AFEF79AFF0DB0BDEC00
:10D9B800028BF0BDAFF300807B14AE47E17A843F61
:10D9C800000000A0D954BD410000000000F07340E1
:10D9D800900D0020080300207C3A0020A425002098
:10D9E800302C00200000F43FC0AC0508FC390020B2
:10D9F8000C2C002018260020242C00202DE9F843A8
:10DA0800461F8846B6B200250D4F12E008EB040108
:10DA180089B23046F7F760FA29F814000A20013471
:10DA2800FBF718F8062CF1D116350136F22DB6B2EF
:10DA380004D06FF0040407EB0509E7E7BDE8F883B5
:10DA4800383A00202DE9F04F85B00B1A0193431E98
:10DA58009BB20293431C441F00F1060901F1FF3AEF
:10DA680001F1010B9BB20F461646A4B21FFA89F9C1
:10DA78001FFA8AFA1FFA8BFB039380462046514609
:10DA88003246F7F761FA204639463246F7F75CFA2C
:10DA9800204659463246F7F757FA019B0298E5188F
:10DAA800ADB229463246F7F74FFA40462946324684
:10DAB800F7F74AFA0134039829463246F7F744FA49
:10DAC800A4B20A20FAF7C6FF4C45D7D105B0BDE885
:10DAD800F08F2DE9F843461F8846B6B200250E4F51
:10DAE80012E008EB040139F8142089B23046F7F740
:10DAF8002BFA01340A20FAF7ADFF062CF1D11635BE
:10DB08000136F22DB6B204D06FF0040407EB050914
:10DB1800E7E7BDE8F88300BF383A00202DE9F04375
:10DB28002DED068B70EE007A8DB017EE900AB0EEF0
:10DB3800408A10EE904A20EE009A04F0E5F8064676
:10DB480020460F4604F0E0F8F7EE008A41EC100B8F
:10DB580041EC1A0B06F094F979EE287A55EC104B43
:10DB680017EE900A04F0D0F82246804689462B46E4
:10DB78003046394604F01CF902460B4640464946F1
:10DB880003F062FF04F0F6FBB0EE4A0AF0EE6A0A10
:10DB980009EE900A38EEC99ADFED377A89EE299AAC
:10DBA80029EE279A06F06CFA304653EC102B3946CA
:10DBB80004F0FEF8044619EE900A0D4604F0A4F8A5
:10DBC80002460B462046294604F01CFA00222B4B3D
:10DBD80004F0EEF804F0CEFBB4EE688ADFED287AA4
:10DBE800284BF1EE10FA044619EE100A08BFB0EE01
:10DBF800678A1D6804F088F802460B4603A8224984
:10DC080008F0F8FE204604F07FF802460B4606A806
:10DC18001E4908F0EFFE78EE287A38EEC88A87EEBB
:10DC2800888A18EE100A04F06FF802460B4609A815
:10DC3800174908F0DFFE0520014603AA0023F8F77C
:10DC480033F90520142106AA0023F8F72DF9C82076
:10DC5800052109AA0023F8F727F94FF6E073009386
:10DC68000520DC212A460023FEF7A2F80DB0BDEC02
:10DC7800068BBDE8F08300BF000048420000494021
:10DC8800A4707D3FD8370020C9AC0508D1AC050881
:10DC9800D9AC05082DE9F04F494B2DED048B1D78C3
:10DCA800022D85B080467BD1464E348A012120461C
:10DCB800FFF709F9FFF76CF88DED000ACDED010AC1
:10DCC8009DE8030004AB03E9030028469DED020A22
:10DCD800DDED030AFEF704FE3B4B1A683B4B1B685D
:10DCE80002FB04343A4B1C603A4BDFED3B7A93ED70
:10DCF800008A68EE277A5F6817EE900A04F004F845
:10DD0800824638468B4603F0FFFF41EC100B41EC8E
:10DD1800190B06F0B5F8504653EC102B594604F091
:10DD280047F823A3D3E9002303F090FE04F002FB95
:10DD3800B0EE490AF0EE690A054684B206F0A0F989
:10DD4800504653EC102B594604F032F80B46024665
:10DD580019A1D1E9000103F077FE04F0EBFAB37CD6
:10DD680081461FFA80FA1BB9B08AF18AFFF7B1FE23
:10DD7800002320465146B374FFF740FE2046514623
:10DD88001F22FFF75FFEB0EE480A00EE907AFFF719
:10DD9800C5FE338AB5829844A6F81080A6F8169076
:10DDA80005B0BDEC048BBDE8F08F00BFAFF3008079
:10DDB8000000000000E063400000000000C05D407B
:10DDC800242C0020900D00200C2C00201826002068
:10DDD800D8370020AC3900200000C842124B1B780D
:10DDE800022B10B50CD1114B1B78022B08D1104C0B
:10DDF8002078C0B140B2FFF74DFF0023237010BD5B
:10DE08000C4C237E23B99F20F7F78CF80123237647
:10DE1800064B1B78022B06D1054C94F90000FFF73E
:10DE2800E9FC0023237010BD242C002004380020B6
:10DE3800591A0020900D0020034B00201860034B56
:10DE48001870FDF7B9BC00BF043600200438002064
:10DE5800034B00201860034B02221A70FDF7ACBC7C
:10DE6800043600200438002037B500242546A0B227
:10DE780028213223024601340095F7F767FEB4F5EE
:10DE8800A07FF4D13EBD2DE9F04F2DED088B02287F
:10DE980097B080468DED070AB34B05D0032805D00F
:10DEA800012805D10C2202E0092200E00B221A7099
:10DEB8001878F2F711FE042103914FF00009F3EEF0
:10DEC8000EAA9FEDAABADFEDAABA7DE1A94B1A689E
:10DED800A94B1B6802FB093307EE103A01211FFA10
:10DEE80089F0B8EEC78AFEF7EEFFFEF751FF8DED19
:10DEF800080ACDED090A08AD95E803000AAB83E8E6
:10DF080003009E4B1A6802EBC9030EAF19689C4BBD
:10DF180019600399521812685A60FEF739FF8DED9F
:10DF2800080ACDED090A95E803000CAB83E8030065
:10DF3800DDED0A9A9DED0BAADDED0C8A9DED0D9A9B
:10DF4800B0EE690AF0EE4A0AB0EE681AF0EE491A25
:10DF5800FEF774FC8DED080ACDED090A95E803007B
:10DF6800B0EE691AF0EE4A1A87E80300B0EE680AC4
:10DF7800F0EE490AFEF76FFC8DED080ACDED090AAF
:10DF880095E8030010AB83E803009DED0E0ADDED74
:10DF98000F0AFEF7D9FD8DED080ACDED090A95E8BF
:10DFA800030016AA02E903009DED100ADDED110A2F
:10DFB800149EFEF7C9FD8DED080ACDED090A95E816
:10DFC800030087E80300DDED0F0AF5EEC00AF1EE65
:10DFD80010FA48BFF1EE600A9DED0E0ACDED0F0A6A
:10DFE800FEF7F4FD8DED080ACDED090A08AA92E8BE
:10DFF800030012AB83E803000798129D03F084FE28
:10E008005D4B139FD3F800B05E4BBDEEC87AD3F8D2
:10E0180000A0CDE9040117EE102A58465146FDF735
:10E028008DFD07EE10AAF8EEC77A07EE10BAB4EE27
:10E03800E78AF8EEC77AF1EE10FAB4EEE78A8CBFF9
:10E0480000220122504B0690F1EE10FAD4BF0022B4
:10E0580002F00102B8F1020FDA6012D0B8F1030F32
:10E068003ED0B8F1010F68D1304603F04DFE36A31B
:10E07800D3E9002303F09CFE0022444B03F0E6FCA6
:10E088002AE0284603F040FEDDE9042304460D4655
:10E098002FA1D1E9000103F0B5FF02460B46204647
:10E0A800294603F085FE2CA3D3E9002303F080FE64
:10E0B80004F060F907EE900AC7EEAA7A17EE900A04
:10E0C80003F022FE41EC100B06F0BEF8002251ECE2
:10E0D800100B2F4B03F06CFE04F004F904462CE0FF
:10E0E80018EE100A03F010FE044638460D4603F0F9
:10E0F8000BFE17A3D3E9002303F05AFEDDE904233E
:10E1080003F080FF04F036F903F0FEFD14A3D3E911
:10E11800002303F04DFE02460B462046294603F035
:10E1280071FF04F027F907EE900AB0EE6B7A07EE5C
:10E138008B7AFDEEC77A17EE904A002C2ADBC72CA3
:10E14800A8BFC72427E000BF8716D9CEF753F5BF6D
:10E158008FC2F5285CAF434000000000009070407B
:10E1680000000080DBC48641242C00200000C8C3C6
:10E178000000C8430C2C002018260020F035002091
:10E18800C0350020302C0020900D00200000694090
:10E19800000049C00024114BDB685BB1104B1888A4
:10E1A800104B1988069B4FF6FF759AB2A3B20095DB
:10E1B800F7F7CCFC0B4B039A1C600699084B083206
:10E1C800196009F101090392074B1B884B45BFF6FB
:10E1D8007DAE17B0BDEC088BBDE8F08F900D002028
:10E1E800F83700209C3A0020FC3900202DE9F04344
:10E1F8002D4B85B01878F2F76FFC2C4B0B221A7058
:10E208002B4B1C782B4B1B78012C14BF102400249B
:10E21800012B0BD1002C14BFD820C820F9F79AFA8B
:10E228000646002C14BFE020D02004E0E820F9F7CF
:10E2380091FA0646F020F9F78DFA00240746DFF830
:10E2480084901D4DDFF8808020E007FB04632046A2
:10E2580001216B61A8F82040FEF735FEFEF798FD16
:10E268008DED000ACDED010A9DE8030004AB03E93A
:10E2780003000D4B9DED020A1878DDED030AFEF749
:10E288002FFB6869FDF73EFE0134A4B2B9F80030EF
:10E29800A342DADA094B02221A70094B00221A76D5
:10E2A80005B0BDE8F08300BF242C0020A425002081
:10E2B800F40D0020B5010020BC37002004380020F0
:10E2C800900D0020FC390020AC3900207FB5FDF707
:10E2D8008BF8274A274B1168526819605A60264CF8
:10E2E800264B22681B68264DD31A06EE903AB8EEE4
:10E2F800E67AD5ED006AF8EEE67A0021C7EE277ACD
:10E30800FCEEE77A17EE906AB0B2FEF7DCFDFEF796
:10E318003FFD8DED000ACDED010A9DE8030004AB39
:10E3280003E90300174B9DED020A1878DDED030A97
:10E33800FEF7D6FA144B1868144B1B6836B200FB6C
:10E348000630FDF7DFFD124B226893F900102868AC
:10E3580000FB01200F4A126890421C4605DCFAF7C0
:10E3680071FF0D4B1868FDF701F9002323707FBD7D
:10E37800BC370020C0350020F835002010260020CA
:10E388009C250020242C00200C2C0020182600207E
:10E39800C325002000260020C825002008B5FFF767
:10E3A80095FF0C4B1A680C4B1B689A4210DB4FF018
:10E3B8008040002102F057FD084B1868FAF742FF29
:10E3C800074B02221A70074A00231370064A137675
:10E3D80008BD00BFF83500200026002010260020C8
:10E3E80004380020C3250020900D002010B500211E
:10E3F8004FF0804002F037FD0A4B00241C700A4B96
:10E4080020461C70F7F742FC084B1868FAF71AFF09
:10E41800074B084801221A70074B1C70BDE81040D2
:10E42800F3F78BBAC32500200836002010260020F9
:10E43800242C0020D4170020A425002007EE100A61
:10E44800034BF8EE477A0022C3ED007A5A60704712
:10E458002C36002007EE100A034BF8EE477A00220C
:10E46800C3ED007A5A607047E03700200F4B10491F
:10E478001A68104B1B68D31A06EE903A0E4B1B68AD
:10E48800B8EEE67A06EE903AF8EEE67AC7EE277A24
:10E49800FCEEE77A17EE903A9AB20B80074B188891
:10E4A80090422CBF00200120704700BF302C002074
:10E4B800FC390020182600200C2C002014260020EF
:10E4C80013B502AB011D23ED010A054A89B213F801
:10E4D800014B1454013080B28842F8D11CBD00BFF2
:10E4E8003A3700202DE9F8431F4F0740002F044614
:10E4F8000D4603DA013F67F00F070137BFB2DFF8B7
:10E5080074804FEAC7091FFA89F9484698ED000A4E
:10E5180009F10409FFF7D4FF1FFA89F098ED010A01
:10E52800FFF7CEFF114B10261B8894FBF6F6F60179
:10E538009C42B6B20CD1701980B20D498022FAF70C
:10E5480029FB00B1FEE721B24FF47F70F9F7CCF850
:10E558000F2F07D17519A8B205498022FAF71AFBBF
:10E5680000B1FEE7BDE8F8830F000080FC39002009
:10E578003A370020BC3700202DE9F043744B2DEDCD
:10E58800028B1888FF2898BF4FF4807093B0C000A2
:10E5980007F0BEFE6F4B0546186028B90520B42168
:10E5A8006D4A2B46F7F780FC0024694F6B4E4FF0FD
:10E5B80000086AE0FCF718FF20464FF44141FFF7D6
:10E5C80091FF674B1A685B683260002173602046D0
:10E5D800FEF779FCFEF7DCFB8DED020ACDED030AB0
:10E5E8000DF1080999E803000AAB83E803005D4BC5
:10E5F8009DED0A1A93ED007AD3ED017ADDED0B1A41
:10E6080031EE470A71EEE70A31EE071A71EEA71AE2
:10E618008DED0E0ACDED0F0A8DED101ACDED111A04
:10E62800FEF719F98DED020ACDED030A99E803000A
:10E638000CAB83E80300FF2C4FEAC4032B4404D936
:10E64800C3F80080C3F8048003E00C9A1A600D9A9E
:10E658005A603B8840F23F10604390FBF3F080B271
:10E668004FF4FC630246282100933223F7F76EFA31
:10E678003D4B18683D4B1B68C018FAF7E3FD3C4B4F
:10E688001868FCF773FF0134A4B23B88A34291DAFF
:10E69800012213464FF4807105A804F0E5FE354EBB
:10E6A800DFF8F880294605A805F0C0F9082333707B
:10E6B800314B01241C700020F6F7B6FD2F48F3F704
:10E6C8003CF93078F2F708FA2D4B9FED2E8ADFEDF2
:10E6D8002E8A1C700024D5ED007AB0EE687A07EE19
:10E6E800C87A2046FCEEC77A17EE906A03F0FAFA69
:10E6F800264B002203F05CFB03F01CFEB6B2A3B26B
:10E70800C72E28BFC72687B253B1214BB8F80000DF
:10E7180019884FF6FF7300933A463346F7F716FA0F
:10E728001B4BC8F8007001340835B4F5807F1E60B3
:10E73800D1D1184B1868FAF785FD114B02221A70CF
:10E74800154B00221A7613B0BDEC028BBDE8F0839E
:10E75800FC390020F0350020CEA40508C035002083
:10E76800BC3700202C360020F83500209C250020DE
:10E77800C8250020242C0020510D0020301700202F
:10E7880004380020000016430000C8420000F43F8F
:10E798009C3A002010260020900D0020F837002019
:10E7A800F0B5294B294F2A4D2A4E012285B01A70FF
:10E7B80000243AE0284B1A68336802FB04336B6183
:10E7C800264B1C84FCF710FE20464FF44141FFF70E
:10E7D80089FE234B2A681A606A6820465A6000211D
:10E7E800FEF771FBFEF7D4FA8DED000ACDED010AB4
:10E7F8009DE8030004AB03E903001A4B9DED020AF0
:10E808001878DDED030AFEF76BF86869FDF77AFB07
:10E81800154B1868154B1B68C018FAF713FD144BF5
:10E828001868FCF7A3FE0134A4B23B88A342C1DAFE
:10E83800104B1868FAF706FD034B02221A700E4BAC
:10E8480000221A7605B0F0BD04380020FC390020FB
:10E85800BC370020182600200C2C0020AC390020E2
:10E86800C0350020242C0020F83500209C250020ED
:10E87800C825002010260020900D002038B5FDF78F
:10E88800F9F9124B124D9F221A81124B0124187864
:10E898002C70F2F721F9104B00221A600F4B1B78ED
:10E8A800072B04D00B2B0DD0062B0ED102E0BDE8B0
:10E8B800384075E74FF0804021462C70BDE838405D
:10E8C80002F0D1BABDE8384090E438BD900D002080
:10E8D80004380020242C002004360020A425002021
:10E8E8002DE9F743002581462C46154E154FDFF8D4
:10E8F8005C801FE0FCF778FD49462046FFF7F2FDF3
:10E90800D8F800303868C018FAF79CFC0E4B186825
:10E91800FCF72CFE308895FBF0F080B24FF4FC63D6
:10E928000093282102463223F7F710F905F59E7562
:10E93800013403353388A342DCDABDE8FE8300BF27
:10E94800FC390020F8350020C82500209C2500202F
:10E9580010B5104C4FF47570B4F90010F8F7C4FEF8
:10E968000D4B4FF47670B3F90010F8F7BDFE40F286
:10E97800D230F8F7C7FEB02804D040F2D230B02128
:10E98800F8F7B2FE2088FFF759FD034B1888BDE859
:10E9980010405FE5B0010020AC01002000210A22F0
:10E9A80008B509F077F9D0F1010038BF002008BD9B
:10E9B80073B5041D0E46A4B20C2200234FF6E07571
:10E9C800204601360095F7F765F900230C22B1B20D
:10E9D80020460095F7F75EF90D4B1B78012B16D1F1
:10E9E8000C4E0D4D308829880024043080B20C224A
:10E9F80023460094F7F74EF93088298800940430AC
:10EA0800013180B289B20C222346F7F743F97CBD65
:10EA1800E43500202A360020DC37002008B54FF600
:10EA2800FF70F7F707F90020F7F706FAE12023212E
:10EA38002C4A0023F7F738FAE1204621294A002317
:10EA4800F7F732FAE1206921264A0023F7F72CFA72
:10EA5800E1208C21244A0023F7F726FA2348FFF700
:10EA68009DFF20B121482249012207F0C3FF4B2016
:10EA780023211E4A0023F7F717FA1E48FFF78EFFD7
:10EA880020B11C481A49012207F0B4FF4B20462147
:10EA9800184A0023F7F708FA1748FFF77FFF20B155
:10EAA80015481349012207F0A5FF4B206921124A96
:10EAB8000023F7F7F9F91148FFF770FF20B10F4865
:10EAC8000B49012207F096FF4B208C2100230B4AAB
:10EAD800F7F7EAF90A4B18880A4B1988BDE8084085
:10EAE80066E700BFDEA20508E5AC0508E0250020C2
:10EAF80066A0050804260020162C0020CC2500203E
:10EB0800143A0020DC39002070B5044600200D4678
:10EB18001646F7F791F90020F7F7A2F84FF4FC60D2
:10EB2800F7F788F82046294656BB1E4A3346F7F7BA
:10EB3800BBF91D48FFF732FF20B11B481B490122D2
:10EB480007F058FF04F17006B6B230462946164A57
:10EB58000023F7F7A9F91648FFF720FF20B114485A
:10EB68001249012207F046FF3235ADB22046294648
:10EB7800104A0023F7F798F9304629460C4A07E06F
:10EB88000D4A0023F7F790F932350B4AA9B220460F
:10EB98000023F7F789F9094B1888094B1988BDE84C
:10EBA800704005E7EAAC0508803A002079A405081A
:10EBB800F0390020F2AC050819A50508143A002020
:10EBC800DC39002030B5144D9DF80C402C70134DE5
:10EBD8002880134D02FB04002980124D80B2288042
:10EBE800114D2980114D2A80114A1380114B18802C
:10EBF800114B1980114B1249E2B21A7000230B70A5
:10EC080010490A709DF810200134013254430E4A0D
:10EC180014700E4A137030BD983B0020783A0020DB
:10EC2800BA370020143A0020DC3900203837002099
:10EC3800A43A00202A360020DC370020DE390020E4
:10EC480009360020163A0020E5350020E43500207A
:10EC580038B5054600200C46F7F7EEF80020F6F721
:10EC6800FFFF4FF4FC60F6F7E5FF0B48FFF796FE51
:10EC780028B1094809490A4B002207F0BBFE28467B
:10EC880021460023044AF7F70FF9064B1888064B6C
:10EC98001988BDE838408BE62036002018A90508F9
:10ECA8000000F03F143A0020DC390020114B1B68AB
:10ECB800002B70B505460C4604DA5B420E480F4936
:10ECC8002D2202E00C480D49202207F093FE002077
:10ECD800F7F7B2F80020F6F7C3FF4FF4FC60F6F739
:10ECE800A9FF054A284621460023BDE87040F7F7EA
:10ECF800DBB800BF103A0020E8370020FAAC05085E
:10ED08000F4B10B519684FF4E170F8F70AFD40F29F
:10ED18003D114FF4E070F8F7E7FC0020F7F78CF8A6
:10ED28000020F6F79DFF4FF4FC60F6F783FF054AD5
:10ED3800192064210023BDE81040F7F7B5B800BFDB
:10ED4800103A002002AD050808B54FF4E070F8F756
:10ED5800D9FC40F23D13984205D14FF4E170BDE86B
:10ED68000840F8F7F7BC002008BD38B50546002074
:10ED78000C46F7F761F80020F6F772FF4FF4FC60D5
:10ED8800F6F758FF0B48FFF709FE28B109480A496A
:10ED98000A4B002207F02EFE284621460023054A8A
:10EDA800F7F782F8064B1888064B1988BDE83840F3
:10EDB800FEE500BFFC35002018A905080000F03F5B
:10EDC800143A0020DC39002038B5C501ADB2002462
:10EDD800601980B2F9F786FC0134C0B2FBF7A6FED1
:10EDE800A4B24FF47A70F9F735FE802CF0D138BD13
:10EDF80073B5104D00240E20FBF798FE002609E09D
:10EE08000DF10700FBF7A3FE20B19DF80730AB55C5
:10EE18000136F6B23306F3D5E00180B20549802207
:10EE2800F9F7B8FE00B1FEE70134A4B2B4F5007FEB
:10EE3800E1D17CBD3A37002007EE100AF8EE477A98
:10EE48007FB517EE900A02F05FFF02460B4601A855
:10EE5800054907F0CFFD0A20962101AA0023F7F7FC
:10EE680023F807B000BD00BF09AD0508AFF3008067
:10EE78000EB403B070470A2810B5044602D10D201D
:10EE8800FFF7F9FF064A13681BB103F8014B13603B
:10EE980010BD044B1B680BB12046984710BD00BF3E
:10EEA800B00D00209C3B002010B5044601E0FFF7A0
:10EEB800E2FF14F8010B0028F9D110BD2DE9F04F3D
:10EEC800044685B00D464FF00A0A00E03546207822
:10EED800002800F0C480252801D0013467E060785C
:10EEE800302803D1A0780123033407E02D2802D06D
:10EEF8000234002302E0A078022303344FF0000814
:10EF080005E00AFB080814F8010BA8F13008A0F185
:10EF18003002D2B2092AF4D96C2801D04C2803D186
:10EF280014F8010B43F00403002800F098806028CF
:10EF380086BFA0F12002D2B202464F2A3DD006D8A1
:10EF4800432A2DD0442A09D0422A30D133E0552A09
:10EF580004D0582A29D0532A29D101E00A272DE0C4
:10EF68002E1D2F68002500E001357A5D002AFBD1AF
:10EF780004E02020FFF77FFF4D4601E0980704D406
:10EF8800454505F10109F4D34D463846FFF78CFF96
:10EF980003E02020FFF76FFF01354545F9D395E7DA
:10EFA80028782E1DFFF767FF90E7102706E0FFF788
:10EFB80062FF2E468AE7022700E008272E1D442A12
:10EFC800296804D1002902DA494243F008030022E3
:10EFD80000E02A46B1FBF7FE07FB1E11CDB2092D52
:10EFE800714607D9782814BF4FF0070C4FF0270C4B
:10EFF8006544EDB230350DF80250551CBEF1000FD6
:10F0080002D0102DE5D10F22190705D504A94D19F5
:10F018002D2105F8101C951C13F0010F0CBF4FF0A3
:10F02800200B4FF0300B9B072F4604D508E05846BD
:10F03800FFF721FF4F46474507F10109F7D34F4630
:10F04800013D1DF80500FFF716FF002DF8D103E07C
:10F058002020FFF710FF01374745F9D336E705B001
:10F06800BDE8F08F70B5064D0C462E68286001E0AB
:10F07800FFF701FF14F8010B0028F9D12E6070BDCD
:10F088009C3B00200FB407B504A951F8040B01916B
:10F09800FFF714FFBDE80E4004B070470EB417B573
:10F0A80005A9084C51F8043B206018460191FFF768
:10F0B80005FF2268002313702360BDE81E4003B0DB
:10F0C800704700BFB00D00200EB433B505A9074C3A
:10F0D80051F8043B2568206018460191FFF7EEFEC1
:10F0E8002560BDE83C4003B0704700BF9C3B002052
:10F0F80070B51E4604461C481546FFF7C3FF022E8E
:10F108001FD0042E25D0012E2AD105E0A15D174875
:10F11800FFF7B8FF013600E00026AE42F6DB2020FC
:10F12800FFF7A9FE002609E0A05DA0F12003DBB2ED
:10F138005E2B88BF2E20FFF79EFE0136AE42F3DB22
:10F148000EE034F8021B0A48FFF79CFF013DF8D196
:10F1580006E054F8041B0748FFF794FF013DF8D177
:10F168000A20BDE8704086E610AD050817AD050811
:10F178001DAD050823AD050808B501214FF48070C1
:10F1880001F07CFA4FF480700021BDE8084001F0DE
:10F1980075BA43680A6823F0407323F480731343F5
:10F1A8000A7943EA02234360CA680B6930B51A43F7
:10F1B80084688D68084B2A43234013434A7943EAFD
:10F1C800420383600B7DC26A013B22F47002DBB20A
:10F1D80042EA0353C36230BDFDF7FFC0002303605A
:10F1E800037143718360C360036101230375704732
:10F1F800074A084B516810B50B4090E812002143AC
:10F208008468C068214301430B43536010BD00BFAD
:10F2180000230140E030FCFF00230360436083606B
:10F22800C3607047836811B143F0010301E023F024
:10F23800010383607047436823F4400323F4007399
:10F248000B4343607047416282627047436823F012
:10F258001F030B4343607047044B5A6810B142F4D4
:10F26800000201E022F400025A60704700230140C6
:10F27800044B5A6810B142F4800201E022F4800283
:10F288005A60704700230140092970B50CB20CD9A7
:10F2980004EB44041E3CC6680725A54026EA05057C
:10F2A800A34045EA0304C4600AE0066904EB440489
:10F2B8000725A54026EA050513FA04F42C43046142
:10F2C800062A0CD80523013A5A43446B1F2393405E
:10F2D80024EA0303914043EA0102426370BD0C2A09
:10F2E80012B20CD802EB8202233A046B1F2393401C
:10F2F80024EA0303914043EA0102026370BD02EB72
:10F308008202413AC46A1F23934024EA03039140CE
:10F3180043EA0102C26270BD836843F080438360A0
:10F3280070478068C0F380507047836811B143F418
:10F33800806301E023F4806383607047836811B1C0
:10F3480043F0020301E023F002038360704743683F
:10F35800013923F4604343EA41334360704743680B
:10F3680011B143F4006301E023F400634360704784
:10F37800C06C80B27047014B186870470823014081
:10F38800836811B143F4807301E023F480738360D0
:10F398007047836811B143F4007301E023F40073EC
:10F3A80083607047044B5A6810B142F4005201E080
:10F3B80022F400525A60704700230140092970B5B1
:10F3C8000CB20CD904EB44041E3CC6680725A540C2
:10F3D80026EA0505A34045EA0304C4600AE0066975
:10F3E80004EB44040725A54026EA050513FA04F4AE
:10F3F8002C430461836BC3F30154121B0232D2B253
:10F4080002EB82021F24944023EA040391400B4339
:10F41800836370BD836B013923F4401343EA0153BE
:10F428008363704782B0002301930190019BCB183E
:10F438000193019B1A6002B07047836823F470231C
:10F448000B4383607047836823F440130B43836046
:10F458007047836843F48003836070478068C0F313
:10F4680080507047436811B143F4806301E023F48E
:10F47800806343607047436811B143F4805301E0EF
:10F4880023F480534360704782B0002301930190B6
:10F49800019B28335B180193019B186880B202B066
:10F4A80070470123C9B213FA01F143680AB119433D
:10F4B80001E023EA010141607047036819420CBF6B
:10F4C800002001207047C943016070474368006805
:10F4D80010EA112007D00122C9B212FA01F119422B
:10F4E8000CBF0020012070476FEA112101607047AE
:10F4F800036823F001030360002303604360836013
:10F50800C3600361212343612C4B98421CD02C4BD0
:10F51800984220D02B4B984225D02B4B98422AD08A
:10F528002A4B98422FD02A4B984233D0294B9842E5
:10F5380037D0294B984204D14FF03D5243F8AC2CB8
:10F548007047264B984203D13D2243F8082C704758
:10F55800234B984204D14FF4746243F8202C70472F
:10F56800204B984204D14FF4741243F8382C70475A
:10F578001D4B984204D14FF0746243F8502C7047E9
:10F588001A4B984203D11A4A43F8642C7047194B16
:10F59800984203D1184A43F87C2C7047174B98427D
:10F5A80003D1174A43F8942C7047164B984204BF6E
:10F5B8004FF03D5243F8AC2C704700BF106002403A
:10F5C800286002404060024058600240706002407B
:10F5D80088600240A0600240B860024010640240A7
:10F5E800286402404064024058640240706402404B
:10F5F8003D00002088640240400F0020A0640240C3
:10F6080000003D20B86402400268134B10B5134057
:10F61800CC680A6822434C6922438C692243CC692E
:10F6280022430C6A22434C6A22438C6A22434C6B65
:10F6380022438C6B22431343036042690C6BCB6AF1
:10F6480022F007022343134343610B6943604B686D
:10F6580083608B68C36010BD3F801CF0002303608B
:10F6680043608360C360036143618361C361036274
:10F6780043628362C36203634363836370470368BF
:10F6880011B143F0010301E023F001030360704767
:10F69800036811B143F4004301E023F4004303601D
:10F6A8007047036811B143F0200301E023F0200301
:10F6B8000360704741607047406880B270470368D4
:10F6C80012B143F4002301E023F400230360016135
:10F6D8007047036811B143F4802301E023F48023C9
:10F6E800036070470AB101617047C16070470068E4
:10F6F800C0F3C0407047006800F0010070474069DF
:10F7080000F0380070470A4A0A4B10B50A4CA0426C
:10F7180088BF13468A004CBF5B681B6821F0F02144
:10F7280021F0821119420CBF0020012010BD00BF3A
:10F7380000640240006002400F64024010B5084BAC
:10F74800084A094CA04288BF134611F0005F21F017
:10F75800F02121F0821114BFD960996010BD00BF5B
:10F7680000600240006402400F6402400B0607D5A7
:10F77800436912B143F0800301E023F08003436141
:10F78800802909D001F01E01036812B119430160F4
:10F79800704723EA010101607047124B124A10B505
:10F7A800124CA0428CBF14461C4621F0F02323F0D3
:10F7B800C3132BB1026802F01E0202EAD12202E052
:10F7C800426902F0800288004CBF6368236821F018
:10F7D800F02121F08210184002D0101C18BF01201F
:10F7E80010BD00BF00600240006402400F64024088
:10F7F80010B5084B084A094CA04288BF134611F0BF
:10F80800005F21F0F02121F0821114BFD9609960C6
:10F8180010BD00BF00600240006402400F64024057
:10F82800044B00221A605A609A60DA60024A5A61F0
:10F83800704700BF003C0140FFFF7F00837910B58F
:10F84800002B29D01A4B01681C68CA4314401C605D
:10F858005C6822405A60027902F1804202F59E32C9
:10F8680014682143116002689C68D1430C409C6075
:10F87800DC682140D9604179102906D19968114383
:10F888009960D9680A43DA6010BD01F1804303F535
:10F898009E3319680A4308E00379016803F180433D
:10F8A80003F59E331A6822EA01021A6010BD00BFF0
:10F8B800003C014000230C220360037142718371F4
:10F8C8007047024B1A6902431A617047003C0140B5
:10F8D800034B5B6918420CBF00200120704700BF32
:10F8E800003C0140014B5861704700BF003C01409B
:10F8F800054B1A685B69034004D010420CBF002016
:10F908000120704718467047003C0140014B586180
:10F91800704700BF003C01404FF0204318B943F244
:10F92800DB021A6003E043F2D20243F820204FF0D2
:10F938002042411C6FF0704342F8213002F5827278
:10F9480042F82030704770B584684568C368C16A5A
:10F95800026825431D4303691D4343691D438369A9
:10F968001D43C3691D43036A1D43436A1D43836ADC
:10F978001D43036B0D431D434FF02043082C43F8F0
:10F98800225005D153F8224044F0400443F8224065
:10F99800436B9E691D6835435E6845EA06159E6897
:10F9A80045EA0625DE6845EA06451E695B6945EABB
:10F9B8000655541C45EA03654FF02043B1F5804FC6
:10F9C80043F8245010D1836B98691968014358682B
:10F9D80041EA0011986841EA002118695B6941EA27
:10F9E800005141EA036101E06FF07041014B43F8B7
:10F9F800221070BD040100A0022242604FF4805220
:10FA08004262416B4FF4005210B5826200230F220C
:10FA1800FF2403608360C360036143618361C36142
:10FA28000362C36203630A604A608C60CA600A6149
:10FA38004A618B61816B0A604A608C60CA600A61A6
:10FA48004A618B6110BD4FF0204321B153F820204B
:10FA580042F0010203E053F82010024A0A4043F83A
:10FA680020207047FEFF0F0010280CBF064B074BE5
:10FA78004FF040024FF0180119605A604FF0FC3205
:10FA88009A60DA60704700BF600000A0800000A0A4
:10FA980030B5836844681C43C36844F008041C43B9
:10FAA80003691C43436944EA4324836944EA4334B1
:10FAB800C36999685A68090441EA02211A68DB682F
:10FAC800114341EA0361036A9A685D68120442EAD5
:10FAD80005221D68DB682A4342EA03620368102B8B
:10FAE8000CBF034B034B1C609960DA6030BD00BF4C
:10FAF800600000A0800000A010230360C2690023FA
:10FB080043608360C360036143618361FC231360C6
:10FB180053609360D360026A136053609360D3604C
:10FB2800704741B110280CBF074B084B1A6842F0C8
:10FB380004021A60704710280CBF034A034A044B9A
:10FB480011680B4013607047600000A0800000A09F
:10FB5800FBFF0F0041B110280CBF084B084B1A6877
:10FB680042F040021A60704710280CBF034A044A4A
:10FB7800044B11680B401360704700BF600000A081
:10FB8800800000A0BFFF0F00102802D1024B586967
:10FB98007047024B58697047600000A0800000A0C1
:10FBA800054B18221A6000225A604FF0FC329A6006
:10FBB800DA601A61704700BFA00000A002684368BD
:10FBC80042F0100242EA4322836842EA4332144B6D
:10FBD80010B51A60C26891685468090441EA0421A2
:10FBE8001468D268214341EA02629A600269916806
:10FBF8005468090441EA04211468D268214341EA9F
:10FC08000262DA60426991685068090441EA002199
:10FC18001068D268014341EA02621A6110BD00BF50
:10FC2800A00000A0C2680023036043608360FC2337
:10FC3800136053609360D3600269136053609360EC
:10FC4800D3604269136053609360D3607047054B7B
:10FC580018B11A6842F0040202E01968024A0A4020
:10FC68001A607047A00000A0FBFF0F0062B11028C7
:10FC780001D10E4B03E0B0F5807F03D10C4B5A68DD
:10FC8800114311E00B4BFAE7102804D1074B5A68CF
:10FC980022EA010108E0B0F5807F0CBF044B054B58
:10FCA8005A686FEA0101114059607047600000A06E
:10FCB800800000A0A00000A0102801D1064B04E09D
:10FCC800B0F5807F0CBF054B054B5B680B420CBF42
:10FCD80000200120704700BF600000A0800000A045
:10FCE800A00000A0102804D1074B5A6822EA01019D
:10FCF80008E0B0F5807F0CBF044B054B5A686FEAEB
:10FD08000101114059607047600000A0800000A008
:10FD1800A00000A0102801D1084B04E0B0F5807FB6
:10FD28000CBF074B074B5B6813EA010004D013EACA
:10FD3800D1010CBF00200120704700BF600000A067
:10FD4800800000A0A00000A0102804D1084B5A6829
:10FD580022EAD10109E0B0F5807F0CBF054B064BC4
:10FD68005A684FEAD10122EA01015960704700BF81
:10FD7800600000A0800000A0A00000A008B52C4BE7
:10FD8800984205D10120014600F048FC012048E0D6
:10FD9800284B984205D10220012100F03FFC0220A7
:10FDA8003FE0254B984205D10420012100F036FCA4
:10FDB800042036E0214B984205D10820012100F0AB
:10FDC8002DFC08202DE01E4B984205D11020012162
:10FDD80000F024FC102024E01A4B984205D1202082
:10FDE800012100F01BFC20201BE0174B984205D195
:10FDF8004020012100F012FC402012E0134B9842F1
:10FE080005D18020012100F009FC802009E0104B79
:10FE180098420BD14FF48070012100F0FFFB4FF4A2
:10FE280080700021BDE8084000F0F8BB08BD00BFA5
:10FE3800000002400004024000080240000C02409A
:10FE4800001002400014024000180240001C02404A
:10FE5800002002402DE9F0470023D1F800801A461F
:10FE68004FF0010C03270CFA02F404EA0805A54236
:10FE78002ED1066817FA03F4E443264006600E798B
:10FE8800D0F8009006FA03FA013E4AEA0909012E61
:10FE9800C0F8009014D8866891F8059026408660CE
:10FEA800866809FA03F949EA06068660466826EA7A
:10FEB800050545608D7946689540ADB23543456086
:10FEC800C5682C40C460CC79C5689C402C43C4608C
:10FED80001320233102AC6D1BDE8F0874FF6FF730E
:10FEE80003600023037143718371C371704782B04B
:10FEF8004FF480330193019B0B430193019BC36132
:10FF0800C161019BC361C3690193C369019302B0D5
:10FF18007047036919420CBF00200120704700692F
:10FF280080B27047436919420CBF00200120704716
:10FF3800406980B2704701837047418370470AB1B6
:10FF480001837047418370474161704743694B4063
:10FF58004361704701F00703C908083130B59B00B9
:10FF680050F821500F249C4025EA040440F8214011
:10FF780050F8214012FA03F31C4340F8214030BDE9
:10FF880008B5134B984207D14FF40010012100F037
:10FF980069FB4FF4001014E00E4B984207D14FF460
:10FFA8008000012100F05EFB4FF4800009E00A4B5D
:10FFB80098420BD14FF40000012100F053FB4FF49D
:10FFC80000000021BDE8084000F04CBB08BD00BFA0
:10FFD8000054004000580040005C00407FB50446D3
:10FFE800868868460D4600F06DFA02992C482B6801
:08FFF80026F03F063604B1FBC0
:020000040801F1
:10000000F0F0360C80B20643A680228822F001026E
:100010001204120C2280254A93420AD85B00B1FBDD
:10002000F3F301309BB280B22084032B98BF0423EA
:1000300021E0EE884BF6FF72964205D1032253432E
:10004000B1FBF3F39BB206E019225343B1FBF3F388
:100050009BB243F480431A054FF4967208BF43F0F5
:10006000010350434FF47A7290FBF2F0013080B2FA
:1000700043F400432084A38323886989AA889BB220
:1000800043F001032380238823F4816323F00203D8
:100090001B040A431B0C13439BB223802A89AB89A0
:1000A00013439BB223817FBD40420F00A086010015
:1000B00041F288330360002383804BF6FF72038193
:1000C00043814FF48043C28083817047038819B114
:1000D0009BB243F0010303E023F001031B041B0C5C
:1000E00003807047038819B19BB243F4807303E027
:1000F00023F480731B041B0C03807047038819B121
:100100009BB243F4007303E023F400731B041B0C45
:100110000380704712B141F0010101E001F0FE01DE
:1001200001827047038819B19BB243F4806303E0F6
:1001300023F480631B041B0C0380704783899BB2EC
:1001400001F0FE0123F0FE030B4383817047838996
:1001500019B19BB243F0010303E023F001031B0438
:100160001B0C83817047038819B19BB243F0400395
:1001700003E023F040031B041B0C0380704703883B
:1001800029B16FEA43436FEA53439BB201E05B043A
:100190005B0C03807047038819B99BB243F080035E
:1001A00003E023F080031B041B0C03807047B1F5B0
:1001B000804F838B04D023F480431B041B0C02E08C
:1001C0009BB243F4804383837047B1F5006F03888B
:1001D00003D19BB243F4006303E023F400631B04E8
:1001E0001B0C03807047B1F5005F038803D19BB2FD
:1001F00043F4005303E023F400531B041B0C03805F
:100200007047038819B19BB243F0100303E023F059
:1002100010031B041B0C0380704701827047008A87
:10022000C0B27047038819B19BB243F4805303E016
:1002300023F480531B041B0C03807047B1F5006F3F
:10024000038803D19BB243F4006303E023F400630B
:100250001B041B0C03807047038819B19BB243F049
:10026000200303E023F020031B041B0C03807047D2
:10027000008BC0F307207047838819B19BB243F409
:10028000006303E023F400631B041B0C83807047AE
:10029000838819B19BB243F4805303E023F4805365
:1002A0001B041B0C8380704782B0002301930190D4
:1002B000019BCB180193019B188880B202B0704754
:1002C00083889BB20AB1194301E023EA01018180CE
:1002D0007047838A008B9BB243EA0040084020F0BD
:1002E0007F40431A584240EB03007047838A008BDB
:1002F0009BB243EA004020F07F40704782B0002369
:10030000009301930B0F01900093009B21F07F411C
:1003100013B1019B143302E0019B090C18330193C4
:10032000019B1B6819420CBF0020012002B07047DE
:10033000C94389B2818270478388808A80B208402D
:100340009BB206D001F0E06113EA11410CBF00201E
:1003500001207047C94389B2818270470A4B1A68ED
:1003600042F001021A6000229A60196821F084713B
:1003700021F48031196005495960196821F4802100
:100380001960DA60704700BF003802401030002466
:10039000024B00221A701870704700BF02380240EA
:1003A000034B1A6822F0F80242EAC0021A60704752
:1003B00000380240014B1860704700BF0000474200
:1003C000064B002201281A701A7002D0042804D1AA
:1003D00001E01870704705221A70704770380240AB
:1003E000014B1860704700BF800E4742014341EA4D
:1003F000821200995B08013B42EA016141EA034134
:10040000014B5960704700BF00380240014B186033
:10041000704700BF600047428001034B40EA017112
:10042000C3F88410704700BF00380240014B1860C9
:10043000704700BF68004742014B1860704700BF1B
:100440004C004742034B9A6822F0EC6202430A4395
:100450009A60704700380240034B9A6822F0784255
:1004600002430A439A60704700380240034B9A687F
:1004700022F0030202439A60704700BF0038024036
:10048000024B986800F00C00704700BF0038024033
:10049000034B9A6822F0F00202439A60704700BF53
:1004A00000380240034B9A6822F4E05202439A60FB
:1004B000704700BF00380240034B9A6822F4604244
:1004C00042EAC0029A607047003802401E4B9A68A8
:1004D00002F00C02042A10B503D0082A03D01B4BEB
:1004E00018E01B4B16E059685A6811F4800F5968E0
:1004F00014BF174B154B02F03F02B3FBF2F3124A45
:100500005268C2F30142C1F3881101324B435200D9
:10051000B3FBF2F30C4903608B680E4A0468C3F323
:100520000313D35C34FA03F343608C68C4F382246E
:10053000145D33FA04F484608968C1F34231525C7B
:10054000D340C36010BD00BF003802400024F40057
:1005500000127A001003002000F44073B3F5407FCE
:10056000084B08D1996820F0704221F4F81122F468
:1005700040720A439A601A6F000542EA10501867E9
:10058000704700BF00380240014B1860704700BF41
:100590003C0E4742014B1860704700BF400E474277
:1005A000014B1860704700BF5C014742044B1A6B57
:1005B00009B1104301E022EA00001863704700BF50
:1005C00000380240044B5A6B09B1104301E022EAA3
:1005D00000005863704700BF00380240044B9A6B1C
:1005E00009B1104301E022EA00009863704700BFA0
:1005F00000380240044B1A6C09B1104301E022EAB2
:1006000000001864704700BF00380240044B5A6C69
:1006100009B1104301E022EA00005864704700BFAE
:1006200000380240044B1A6909B1104301E022EA84
:1006300000001861704700BF00380240044B5A693F
:1006400009B1104301E022EA00005861704700BF81
:1006500000380240044B9A6909B1104301E022EAD4
:1006600000009861704700BF00380240044B1A6ACE
:1006700009B1104301E022EA00001862704700BF90
:1006800000380240044B5A6A09B1104301E022EAE3
:1006900000005862704700BF00380240044B1A6DDA
:1006A00009B1104301E022EA00001865704700BF5D
:1006B00000380240044B5A6D09B1104301E022EAB0
:1006C00000005865704700BF00380240044B9A6D27
:1006D00009B1104301E022EA00009865704700BFAD
:1006E00000380240044B1A6E09B1104301E022EABF
:1006F00000001866704700BF00380240044B5A6E75
:1007000009B1104301E022EA00005866704700BFBB
:1007100000380240044B1A7809B1104301E022EA84
:1007200000001870704700BF0D3802404309012BCC
:10073000074A01D1136803E0022B0CBF136F536FFC
:1007400000F01F0033FA00F000F00100704700BF16
:100750000038024007B5002301933120FFF7E6FF80
:10076000019B01330193019BB3F5A06F01D00028D9
:10077000F3D03120FFF7DAFF003018BF01200EBDA3
:10078000024B5A6F42F080725A677047003802403D
:10079000034BDB6818420CBF00200120704700BFEC
:1007A00000380240014B1870704700BF0E380240FD
:1007B00008B5154B98420BD101214FF48050FFF73B
:1007C00061FF4FF480500021BDE80840FFF75ABF99
:1007D0000E4B984207D14FF480400121FFF746FFAE
:1007E0004FF4804009E00A4B98420BD14FF400408F
:1007F0000121FFF73BFF4FF400400021BDE8084016
:10080000FFF734BF08BD00BF003001400038004092
:10081000003C00400B88028810B54C8823438C882C
:100820002343CC8823430C8923434C8923438C895D
:100830002343CC8902F44152234313439BB20380E8
:10084000838B23F400631B041B0C83830B8A0382BA
:1008500010BD838B23F47B6323F00F031B041B0C5D
:100860008383022303848B68F0B5858B022BADB2A2
:1008700038D0294A8E889468002E14BF022601269B
:10088000240203D5946824F400049460D2F88440D0
:10089000D2F884705268DFF884C002F03F02BCFBDB
:1008A000F2F2C4F388145443C7F30272B4FBF2F4B7
:1008B000CA88B2F5007F4FF00A0201D1240A02E093
:1008C0007601B4FBF6F46243B2FBF3F305330A227C
:1008D0009BB2B3FBF2F303F001021202C3F34F0326
:1008E00092B200E000229C1EA4B2FE2C28BF00227F
:1008F000CC8828BF0223134323439BB203840B8875
:100900004A882B4343F4006313438A8813438A893C
:1009100013439BB28383F0BD0038024000127A007B
:100920000023038043808380C380038143818381CC
:10093000C381072303827047002302220380438080
:100940008380C380826083817047038819B19BB222
:1009500043F0400303E023F040031B041B0C03801F
:100960007047838B19B19BB243F4806303E023F497
:1009700080631B041B0C83837047038823F400638C
:100980001B041B0C038003889BB20B43038070473E
:10099000B1F5804F038803D19BB243F4804303E059
:1009A00023F480431B041B0C038070474FF6FF6346
:1009B0009942038803D09BB243F4807303E023F48D
:1009C00080731B041B0C03807047838819B19BB292
:1009D00043F0040303E023F004031B041B0C838097
:1009E0007047838819B19BB243F0100303E023F0F2
:1009F00010031B041B0C83807047838B23F47B63E1
:100A000023F00F031B041B0C8383022303840B8836
:100A1000828BB3F5007F10B592B205D0002B0CBFCE
:100A20004FF48073002301E04FF480734C8822431D
:100A30008C88898942F4006222430A4392B21343AC
:100A4000838310BD808980B270478181704703889D
:100A500019B19BB243F4005303E023F400531B0489
:100A60001B0C0380704703889BB243F480530380C0
:100A70007047012902D0008B80B27047808A80B213
:100A80007047008A80B2704783889BB20AB11943CD
:100A900001E023EA010181807047090901238B40AD
:100AA0009BB21AB1828892B2134303E0828892B259
:100AB00022EA030383807047038919420CBF002098
:100AC00001207047C94389B20181704710B58488FD
:100AD0000089012301F00F0280B213FA02F21040E4
:100AE000A4B205D009098B401C420CBF0020012094
:100AF00010BD01F00F0101238B40DB439BB203814A
:100B0000704700BF08B501214FF48040FFF7BAFDE0
:100B10004FF480400021BDE80840FFF7B3BD014B12
:100B2000186070470038014001F0030289080A4B41
:100B3000023130B5920053F821500F24944025EA39
:100B4000040443F8214053F8214010FA02F2144300
:100B500043F8214030BD00BF00380140014B186010
:100B6000704700BFDC002742014B1860704700BF90
:100B700000042742024B186AC0F30020704700BFF0
:100B80000038014030B5048C24F001042404240C06
:100B90000484058B048CADB2A4B225F0F305154393
:100BA00024F00A0445EA031544F00104ADB20C43F5
:100BB0000583048430BD30B5048C24F01004240473
:100BC000240C0484048B058C24F44074ADB22405F9
:100BD000240D25F0A00544EA022445F0100544EA5E
:100BE000033445EA0115A4B2ADB20483058430BDD7
:100BF00008B5474B984205D101200146FFF742FD59
:100C000001203DE0B0F1804F05D101200146FFF702
:100C10002DFD012076E03F4B984205D102200121B5
:100C2000FFF724FD02206DE03B4B984205D10420E4
:100C30000121FFF71BFD042064E0384B984205D1E9
:100C400008200121FFF712FD08205BE0344B984299
:100C500005D110200121FFF709FD102052E0314B92
:100C6000984205D120200121FFF700FD202049E016
:100C70002D4B984209D102200121FFF703FD0220EC
:100C80000021BDE80840FFF7FDBC284B984207D182
:100C90004FF480300121FFF7F5FC4FF48030EFE78F
:100CA000234B984207D14FF400300121FFF7EAFCB3
:100CB0004FF40030E4E71F4B984207D14FF48020F7
:100CC0000121FFF7DFFC4FF48020D9E71A4B98424F
:100CD00005D140200121FFF7C9FC402012E0174B4D
:100CE000984205D180200121FFF7C0FC802009E057
:100CF000134B98420BD14FF480700121FFF7B6FCE3
:100D00004FF480700021BDE80840FFF7AFBC08BD7C
:100D1000000001400004004000080040000C0040BA
:100D20000010004000140040000401400040014059
:100D3000004401400048014000180040001C0040F1
:100D4000002000401C4A038890429BB212D002F55A
:100D5000806290420ED0B0F1804F0BD0A2F580326D
:100D6000904207D002F58062904203D002F5806283
:100D7000904203D14A8823F0700313430F4A9042F4
:100D800008D002F58062904204D023F440730A89AF
:100D90009BB2134303804B68C3620B880385064BE9
:100DA000984203D003F58063984201D18B7A038681
:100DB00001238382704700BF000001400010004003
:100DC0004FF0FF334360002303800381438083722D
:100DD0007047018582827047038823F070031B04EB
:100DE0001B0C0B430380704741627047C162704720
:100DF000406A7047008D80B27047038819B19BB27A
:100E000043F0020303E023F002031B041B0C0380E6
:100E10007047038819B19BB243F0040303E023F049
:100E200004031B041B0C03807047038819B19BB299
:100E300043F0800303E023F080031B041B0C0380BA
:100E40007047038823F008031B041B0C03800388EE
:100E50009BB20B4303807047038823F440731B0449
:100E60001B0C038003889BB20B43038070470388ED
:100E700019B19BB243F0010303E023F001031B040B
:100E80001B0C03807047038C23F001031B041B0C15
:100E9000038470B5038C8488028B0D884E8822F001
:100EA00073021204120C2A438D8923F002031B04DF
:100EB00035431B0CADB22B430E4DA842A4B203D058
:100EC00005F58065A8420ED1CD894E8A23F008032E
:100ED0002B438D8823F004032B430D8A354324F4E0
:100EE0004074ADB22C43848002838A6842630384D9
:100EF00070BD00BF00000140038C23F010031B04F1
:100F00001B0C0384038C828830B5048B0D8824F479
:100F1000E6442404240C23F0200344EA05241B04A3
:100F20008D891B0C43EA05134D8843EA0513134DC5
:100F3000A84292B2A4B29BB203D005F58065A84244
:100F400015D1CD8923F080039BB243EA05134FF6F8
:100F5000BF751D408B8845EA03130D8A22F4406259
:100F600042EA85024D8A42EA85029BB292B28280B1
:100F70008A6804838263038430BD00BF000001409F
:100F8000038C23F480731B041B0C0384038C828862
:100F900030B5848B0D8824F073042404240C23F4CE
:100FA00000731B042C438D891B0C43EA05234D88D9
:100FB00043EA0523124DA84292B29BB203D005F535
:100FC0008065A84215D1CD8923F400639BB243EA22
:100FD00005234FF6FF351D408B8845EA03230D8A14
:100FE00022F4405242EA05124D8A42EA05129BB2AF
:100FF00092B282808A688483C263038430BD00BF5A
:1010000000000140038C23F480531B041B0C038459
:10101000038C30B58488828B0D8822F4E64212045A
:10102000120C23F4005342EA05221B048D891B0C89
:1010300043EA05334D8843EA05330B4DA842A4B279
:1010400092B29BB203D005F58065A84205D10D8A06
:1010500024F4804444EA8514A4B2848082838A689C
:101060000264038430BD00BF000001400023038000
:101070004380838083608381C3810382438270477E
:1010800030B5058C0124ADB28C4025EA040400F192
:101090001803048409B1082907D149084FF68F7055
:1010A000CC582040C850C8580AE00439C1F34E015A
:1010B00048F6FF70CC582040C8501202C85892B26F
:1010C0000243CA5030BD4163704781637047C163BA
:1010D000704701647047038B23F070031B041B0CE3
:1010E0000B4303837047038B23F4E0431B041B0C67
:1010F00043EA01239BB203837047838B23F0700381
:101100001B041B0C0B4383837047838B23F4E04346
:101110001B041B0C43EA01239BB283837047038BA0
:1011200023F008031B041B0C0B4303837047038B42
:1011300023F400631B041B0C43EA01239BB20383CB
:101140007047838B23F008031B041B0C0B43838322
:101150007047838B23F400631B041B0C43EA0123B9
:101160009BB283837047038B23F004031B041B0C87
:101170000B4303837047038B23F480631B041B0C16
:1011800043EA01239BB203837047838B23F004035C
:101190001B041B0C0B4383837047838B23F48063F6
:1011A0001B041B0C43EA01239BB283837047038B10
:1011B00023F080031B041B0C0B4303837047038B3A
:1011C00009025B0441EA53439BB203837047838B5C
:1011D00023F080031B041B0C0B4383837047838B1A
:1011E00009025B0441EA53439BB283837047038C3B
:1011F00023F002031B041B0C0B4303847047038C76
:1012000023F008031B041B0C0B4303847047038C5F
:1012100023F020031B041B0C43EA01139BB203843D
:101220007047038C23F080031B041B0C43EA01135B
:101230009BB203847047038C23F400731B041B0CC4
:1012400043EA01239BB203847047038C23F40063B9
:101250001B041B0C43EA01239BB203847047038CDD
:1012600023F400531B041B0C43EA01339BB2038499
:10127000704710B5048C01238B40A4B224EA030309
:101280000384038C12FA01F10B439BB2038410BD5B
:1012900010B5048C04238B40A4B224EA0303038416
:1012A000038C12FA01F10B439BB2038410BD00239F
:1012B0000122038043808280C38003817047406B9A
:1012C0007047806B7047C06B7047006C7047038B32
:1012D00023F00C031B041B0C0383038B9BB20B43F7
:1012E00003837047038B23F440631B041B0C0383AD
:1012F000038B9BB243EA01239BB203837047F8B58B
:101300000C464988A288B4F800E0238905460029E4
:101310000CBF02270027012A14BF01260226BEF1B6
:10132000000F10D1FFF72EFC2846E188FFF7CFFF12
:101330002846394632462389FFF73DFCE188284696
:10134000BDE8F840CEE7FFF736FC2846E188FFF716
:10135000C9FF2846394632462389FFF713FCE18846
:101360002846BDE8F840B2E7838B23F00C031B044A
:101370001B0C8383838B9BB20B4383837047838BCC
:1013800023F440631B041B0C8383838B9BB243EACF
:1013900001239BB283837047F8B50D460B88AA885A
:1013A000498804463BB92B89FFF7ECFBE9882046C6
:1013B000BDE8F8408BE7042B07D12B89FFF7FBFB37
:1013C000E9882046BDE8F8408CE7082BB5F808C04E
:1013D000078C1DD127F480773F043F0C0784868B50
:1013E000038CB6B29BB226F0F30623F4206346EAE0
:1013F0000C1C43EA01211FFA8CFC89B24CEA020260
:1014000041F4807182830184E988BDE8F840ABE74C
:1014100027F480573F043F0C0784868B038C26F407
:10142000407623F4005336055B04360D5B0C46EA28
:10143000022243EA013342EA0C329BB2E98892B2BB
:1014400043F4805382830384BDE8F84097E74A88D9
:101450000B8813438A881343CA8813430A891343AA
:101460004A8913438A8913439BB2A0F844307047DA
:101470000023038043808380C38003814381838171
:101480007047B0F8443029B16FEA43436FEA5343E1
:101490009BB201E05B045B0CA0F84430704783888A
:1014A00019B19BB243F0040303E023F004031B04CF
:1014B0001B0C83807047838819B19BB243F00103F2
:1014C00003E023F001031B041B0C83807047838916
:1014D0009BB20AB1194301E023EA010181817047FF
:1014E00081827047038A19420CBF00200120704797
:1014F000C94389B201827047038A828911EA0300D5
:1015000092B203D011420CBF002001207047C943A2
:1015100089B2018270470A43A0F848207047838946
:101520009BB20AB1194301E023EA010181817047AE
:10153000838819B19BB243F0080303E023F008034A
:101540001B041B0C83807047038923F007031B04D3
:101550001B0C03817047038923F070031B041B0CD1
:101560000B43038103899BB243F007030381704758
:1015700038B50D4611460122602D044602D1FFF711
:101580001AFB01E0FFF7FEFA238923F070031B0426
:101590001B0C1D43258123899BB243F00703238144
:1015A00038BD038923F070031B041B0C0B4303811C
:1015B0007047838823F070031B041B0C838083888F
:1015C0009BB20B4383807047038923F007031B04FE
:1015D0001B0C038103899BB20B4303817047038972
:1015E00023F080031B041B0C038103899BB20B4374
:1015F0000381704710B50489E4B20C43144344EAF4
:101600000324A4B2048110BD10B50446FFF7F2FF15
:1016100023899BB243F48043238110BD10B5044657
:10162000FFF7E8FF238923F077031B041B0C43F02B
:101630007703238110BD70B50489068B058C26F4D1
:101640004076ADB226F0030624F00704360425F0F8
:1016500022052404360C1543240C46F4807645EA12
:101660000315214346F00106ADB2018106830584CE
:1016700070BD838819B19BB243F0800303E023F06F
:1016800080031B041B0C83807047A0F85010704728
:1016900008B5234B984205D110200121FEF7F2FF37
:1016A000102037E01F4B984207D14FF40030012142
:1016B000FEF7DCFF4FF4003009E01B4B98420BD1E2
:1016C0004FF480200121FEF7D1FF4FF4802000214C
:1016D000BDE80840FEF7CABF144B984207D14FF44B
:1016E00000200121FEF7C2FF4FF40020EFE7104B6E
:1016F000984207D14FF480100121FEF7B7FF4FF455
:101700008010E4E70B4B984209D120200121FEF71D
:10171000B9FF20200021BDE80840FEF7B3BF08BD97
:10172000001001400044004000480040004C0040D0
:101730000050004000140140038ACA889BB223F481
:10174000405330B513430D46038283890989AA8823
:1017500023F4B0530A43698923F00C031B040A43A2
:101760001B0C92B213438381838AAA899BB223F410
:101770004073134385B0838204466846FEF7A6FE95
:101780001A4B9C4203D003F580639C4201D1039B1A
:1017900000E0029BA28912B2002A4FF019012A68C8
:1017A00001FB03F101DA520000E092006423B1FB77
:1017B000F2F1B1FBF3F21201100903FB1011A08941
:1017C00000B2002806DAC9003231B1FBF3F303F0AE
:1017D000070305E009013231B1FBF3F303F00F0316
:1017E0001A4392B2228105B030BD00BF0010014003
:1017F0004FF4165303600C2200238380C3800381BF
:101800004281838170470B88028A10B54C8823433C
:101810008C88C988234392B20B4322F470629BB236
:101820001343038210BD0023038043808380C38061
:101830007047838919B19BB243F4005303E023F44A
:1018400000531B041B0C83817047038B03F47F43FD
:101850000383038B9BB20B4303837047838929B1B6
:101860006FEA43436FEA53439BB201E05B045B0CB6
:1018700083817047838A19B19BB243F4006303E00C
:1018800023F400631B041B0C83827047C905C90D38
:10189000818070478088C005C00D7047038A23F09F
:1018A0000F031B041B0C0382038A9BB20B430382AE
:1018B0007047838919B19BB243F0020303E023F020
:1018C00002031B041B0C83817047838923F400638C
:1018D0001B041B0C838183899BB20B43838170475C
:1018E000038A23F020031B041B0C0382038A9BB290
:1018F0000B4303827047038A19B19BB243F48043C0
:1019000003E023F480431B041B0C0382704783898C
:101910009BB243F0010383817047838A19B19BB264
:1019200043F0080303E023F008031B041B0C83822D
:101930007047038BDBB20383038B9BB243EA012323
:1019400003837047838A19B19BB243F0200303E0FD
:1019500023F020031B041B0C83827047838A19B178
:101960009BB243F0100303E023F010031B041B0C95
:1019700083827047838A23F004031B041B0C838239
:10198000838A9BB20B4383827047838A19B19BB2CF
:1019900043F0020303E023F002031B041B0C8382C9
:1019A0007047838A9BB20AB1194301E023EA01011F
:1019B00081827047C1F3421310B501F01F01012469
:1019C00014FA01F1A34201D10C3004E0022B01D141
:1019D000103000E0143003680AB1194301E023EA33
:1019E0000101016010BD038819420CBF00200120D5
:1019F0007047C94389B201807047012210B501F0D8
:101A00001F03C1F342149A40012C01D1838903E0E2
:101A1000022C0CBF038A838A9BB21340028892B2C5
:101A200043B1090A012313FA01F111420CBF00204E
:101A3000012010BD184610BD090A01238B40DB436D
:101A40009BB20380704700BF81F0004102E000BFFD
:101A500083F0004330B54FEA41044FEA430594EA6E
:101A6000050F08BF90EA020F1FBF54EA000C55EAA9
:101A7000020C7FEA645C7FEA655C00F0E2804FEA7A
:101A80005454D4EB5555B8BF6D420CDD2C4480EA5C
:101A9000020281EA030382EA000083EA010180EA8C
:101AA000020281EA0303362D88BF30BD11F0004FDA
:101AB0004FEA01314FF4801C4CEA113102D0404210
:101AC00061EB410113F0004F4FEA03334CEA13334B
:101AD00002D0524263EB430394EA050F00F0A78063
:101AE000A4F10104D5F1200E0DDB02FA0EFC22FA5E
:101AF00005F2801841F1000103FA0EF2801843FA52
:101B000005F359410EE0A5F120050EF1200E012A42
:101B100003FA0EFC28BF4CF0020C43FA05F3C01880
:101B200051EBE37101F0004507D54FF0000EDCF1F9
:101B3000000C7EEB00006EEB0101B1F5801F1BD3A2
:101B4000B1F5001F0CD349085FEA30004FEA3C0CA6
:101B500004F101044FEA445212F5800F80F09A809C
:101B6000BCF1004F08BF5FEA500C50F1000041EBA0
:101B7000045141EA050130BD5FEA4C0C404141EBA4
:101B8000010111F4801FA4F10104E9D191F0000FCB
:101B900004BF01460020B1FA81F308BF2033A3F14E
:101BA0000B03B3F120020CDA0C3208DD02F1140C45
:101BB000C2F10C0201FA0CF021FA02F10CE002F180
:101BC0001402D8BFC2F1200C01FA02F120FA0CFC79
:101BD000DCBF41EA0C019040E41AA2BF01EB0451C2
:101BE000294330BD6FEA04041F3C1CDA0C340EDCC0
:101BF00004F11404C4F1200220FA04F001FA02F303
